:1000000000400020E57700002578000027780000F8
:1000100000000000000000000000000000000000E0
:10002000000000000000000000000000297800002F
:1000300000000000000000002B7800002D78000078
:100040002F780000CD570000917B00002F78000032
:100050002F780000000000002F7800002F780000AB
:1000600095360000657F00002F7800002F78000093
:100070002F7800002F7800002F7800002F780000E4
:100080002F780000157C00002F7800002F780000EA
:100090002F7800002F7800002F7800002F780000C4
:1000A0002F7800002F780000000000000000000002
:1000B0000000000000000000000000000000000040
:1000C00010B5064C2378002B07D1054B002B02D02E
:1000D000044800E000BF0123237010BD700200201F
:1000E00000000000B4EB0000044B10B5002B03D05F
:1000F0000349044800E000BF10BDC04600000000F6
:1001000074020020B4EB0000164B002B00D1144BFE
:100110009D46402292029A1A924600218B460F4633
:100120001348144A121A0BF051FD0F4B002B00D04C
:1001300098470E4B002B00D0984700200021040068
:100140000D000D48002802D00C4800E000BF0BF065
:10015000FDFC2000290007F06DFD0BF0D1FCC0462E
:100160000000080000400020000000000000000027
:1001700070020020D02F00200000000000000000CE
:1001800002000120104011D1042A0ED91368180969
:1001900080B2002809D001388000031D11180979A8
:1001A000002902D001309842F8D170470020FCE7C6
:1001B0000378002B03D05AB2002A01DB01307047CC
:1001C0003F229343C03B59424B41C01803789343AD
:1001D000802BF4D10130F9E710B500240378002B0F
:1001E00001D1200010BDFFF7E3FF0134F6E770B541
:1001F000002204000D00411C092003F073FD0028BB
:1002000006D001236200134343600023A34200DBB6
:1002100070BD9A00A958821891600133F6E770B555
:10022000012803DC1C2001F027F970BD01230D68B3
:1002300011201D42F7D04868184206D1042804D97D
:100240000F2302681340042B01D00E20EBE703F0CC
:10025000A7FB6D100400002D03DDFFF7BDFFA842D2
:1002600006DA1220DFE72000FFF7A2FF0400013DBD
:10027000012DF8D120787F2809DDDF280BDCF82359
:100280003F22DB00800118406378134018430123AC
:1002900040001843C9E7EF280BDCFC226378120109
:1002A0009B0113403F220007000C0343A07810403D
:1002B000ECE7F72812DCFC22637892021B03134060
:1002C000E0228004520310403F221843E378134099
:1002D000FC220343A07812018001E8E7012040429C
:1002E000D5E7F8B54D680F00EB0706D4042D04D907
:1002F0000F232E683340092B03D00B2001F0BCF8EC
:10030000F8BD6B683609B6B25C10731EA3420FD8F5
:100310000321200009F016FB6421642803DC01009E
:10032000032800DA03212800891903F00DFD0500D8
:100330002B6800201B099BB2013B9C42E0D23A682B
:10034000A31C9B005A510123013464001C436C60C0
:10035000D6E7F0B585B0012803DC1C2001F08CF84D
:1003600012E001274B683A000093022806D08B6800
:100370003B4203D05F10002F00DC17000125009BDB
:100380002B4203D00120404205B0F0BD009B042B5E
:10039000F8D91B680C680F261900314004292AD1AE
:1003A0002C4205D1042C03D923681E40042E01D011
:1003B0000E20D3E70098FFF7E3FEB842E2DB009897
:1003C00003F0EEFA0600200003F0EAFA0100781EBE
:1003D00030180BF0B1FF041ED4D03378002B01D0BD
:1003E000A64202D36800012521E03000FFF7E0FEBD
:1003F00001350600F1E709293ED1009B5B685B10DF
:1004000001939F42BEDC2C422ED1042C2CD92368B0
:100410003340042B28D1200003F0C2FA0396029047
:100420007E1C009AB300D058844202D17800284341
:10043000AAE728420ED104280CD90368039A134076
:10044000042B07D103F0ACFA010002980BF03EFF39
:100450000028EBD0019B37009E42E1DD92E71F00B0
:10046000019B9F4200DD8DE77B1C00999A008A5812
:10047000A242F4D17800B6E7032900D082E71A0936
:1004800092B25B0F92000B40D31A01939F4200DDA2
:1004900078E72C4229D1042C27D922681640032E54
:1004A00019D1100980B2520F80003240251D801AE8
:1004B000019B2E181B1A0193009B781E0433019A8E
:1004C000904200DD5EE72A001918B2420FD316D120
:1004D0000130400087E7042E07D1200003F060FAC6
:1004E00005002000FFF74CFEE2E70F2036E70C780E
:1004F000A4461478A44502D101310132E5E7013068
:10050000DDE710B503F030FA43000120184310BDB9
:10051000C30711D404280FD90F2302681340032BFB
:100520000AD119400133591AC0234907DB05194084
:10053000024B1A40114301607047C046FFFFFF9F06
:10054000F7B507000E001C20012F06DD4C680123C3
:1005500022001A40009203D10D2000F08DFF53E0DD
:10056000022F02D08A681A42F6D0012335681D4254
:1005700000D0A9E0042D00D8A6E01C41002C00DC2E
:100580001C000F2029680840092828D16B685B10DF
:100590000093022F05D0B368009A5B109A4200DDE9
:1005A0000093009B01221D1B0135EB43DB171D400F
:1005B000691C092003F096FB071E09D001236D007A
:1005C0001D4303003268083345600099A14201DAF7
:1005D0003800FEBD0134A100515802C3F5E70428DC
:1005E00045D1280003F0DCF9FFF7F6FD0190022F5A
:1005F00004D0B3685B10984200DD0193019BA342D5
:1006000004DA002003F0E0FB0700E1E7280003F034
:10061000C7F90700009BA34221DB2800009703F0E5
:10062000BFF905003800FFF7C3FD019B0134070047
:10063000A342F7DA009BC41A200003F0C5FB071E93
:10064000C6D003F0ADF90190306803F0A9F922009B
:10065000009B591B411801980BF09CFAB8E7380031
:10066000FFF7A6FD009B070001330093D2E70328A4
:100670002AD10B099BB2490F9B000140591A022F46
:1006800004D0B2685210914200DD1100A14205DA97
:1006900000220320110003F025FBB5E703200E1B09
:1006A000331DD9170140C9188910002203F01AFB25
:1006B000071E00D18CE7013631000334FFF728FF15
:1006C000381D29193200C7E7212046E7F8B5002870
:1006D00005DC1C2000F0D0FE05002800F8BD012636
:1006E0000C6826400FD06410E343DB171C40E11C6C
:1006F00089100022032003F0F5FA051EEDD0210039
:10070000FFF706FFE9E7042C01D80025E5E70F23F2
:1007100022681340042B1BD12000FFF731FDC31CBE
:1007200007000320D9170140C9188910320003F0CF
:10073000D9FA051ED1D03900FFF7EAFE200003F0F8
:100740002FF92B1D01003A0018000BF023FAC4E723
:10075000092BDAD10320636832005F10FB1CD91724
:100760000140C918891003F0BDFA051ECDD039002B
:10077000FFF7CEFEFF20BE42AFDA0122B300E3183E
:100780009B68134208D01341FF2B00DD0300D943BF
:10079000C917AA190B4013710136ECE710B57F2970
:1007A00002DC0170013010BD1A4B99420CDC402371
:1007B0008A115B42134303703F230B40802149425F
:1007C000194341700230EEE7134B994210DC2023AD
:1007D0000A135B4213433F24802203708B11524261
:1007E0002340214013430A43437082700330DAE709
:1007F0000A4B9942D7DCF0230370603B4370113BF6
:100800008A11FF3B1A4382703F2211401943C17085
:100810000430C8E7FF070000FFFF0000FF0F0100E2
:10082000F0B50D0085B0002803DC1C2000F024FE8C
:100830000DE009680122080010400AD002AC114105
:100840002000FFF7ABFF011B200003F0C9FA0400F2
:100850001AE004293FD90F230C682340092B3AD111
:100860004B685B10019303239C46019B9A420EDD6B
:1008700003F0AAFA041E07D02E68012503F090F8B1
:100880002F00019B9D421DDD200005B0F0BD01320F
:100890009300CC580123234001D10D20C6E76410FA
:1008A0007F2C0DDD0D4E0223B44209DD0C4E634654
:1008B000B44205DD00270B4EE30FA6427B419B00AF
:1008C000C018D2E70135AB00F1583942E5D04910E4
:1008D000FFF764FFD5E72120A8E7C046FF07000027
:1008E000FFFF0000FF0F010010B5040001200840C9
:1008F00010D104290DD90F230A681340042B08D105
:10090000080003F04DF8010020000BF0DFFC43422B
:10091000584110BD0020FCE7F7B50F00012803DCAB
:100920001C2000F0A9FDFEBD01264D682E4006D119
:10093000042D04D90F222B681A40092A01D00B205C
:10094000EFE76A681B099BB25410A34200D85C1EF3
:1009500039681E48FFF7C8FF01230190002813D112
:1009600039681B48FFF7C0FF002811D0002C0DD0BC
:100970000123621C013C9C409200535123436B6055
:1009800004E00136B200AB50B442FADA0020CAE704
:100990003B680D20DA07C4D55B10002B11DD9C42AB
:1009A0000FDB9B00A200291DEB1889180433994224
:1009B00009D10123013C9C40AA181C4353606C6080
:1009C000E4E71220ADE758681860EFE75FD2000057
:1009D00063D20000002310B50C000B70C30705D5CF
:1009E0000D49421020000BF035FC08E00B490028AF
:1009F00002D0042804D10A4920000BF04BFC10BDA2
:100A00000428FCD90F2302681340042BF7D102F00D
:100A1000C7FF04490200E5E7F4DC000068D20000EB
:100A20006ED2000073D20000F0B593B006000291C0
:100A30001C20012E1DDD029B01251B681C002C4083
:100A400000D0ADE0042B00D8E6E01A680F231A406E
:100A5000092A4AD10394039A029992008A581700EE
:100A60002F4005D1042A03D910681840092806D060
:100A7000222000F001FD0190019813B0F0BD5268F2
:100A80005210A418039A013203929642E3D1611CDA
:100A9000012203F027F90190002802D100230193DD
:100AA000EAE7019B6400190025435D600831029A62
:100AB000BB00D05802684368120992B25B109A4298
:100AC00000D8531E0022934209DCDA43D2171340A8
:100AD0009B00C918039B01379F42E8DBCCE79400D9
:100AE0000519AD6801320D51EDE72700032A59D1F0
:100AF0000193029ABB00D3582B42B9D1042BB7D92A
:100B0000186801990140032939D1020992B2430FB3
:100B100092000B40D31A1C190137BE42E9D10320C1
:100B2000E31CD9170140C9188910002203F0DAF834
:100B300001900028B2D000252100FFF7E9FC019BBD
:100B40001E1D029AAB00D45801231C421FD1042C55
:100B50001DD90F2123681940032918D1180980B223
:100B60005B0F80000B40C01A0023834213DBC3439A
:100B7000DB17184001353618BD42E2DB7CE704295B
:100B800000D075E71800FFF7FBFA2418C4E720002F
:100B9000FFF7F6FAE8E7E2181279F2540133E4E7D6
:100BA00000273C000F25029ABB00D35801221342B4
:100BB00034D1042B32D9186801002940042935D1D9
:100BC0001800FFF7DDFA24180137BE42EBD12000F0
:100BD00003F0FAF80190002800D15FE7029FB60009
:100BE000BB19041D029301233D681D4229D1042D28
:100BF00027D90F262B681E40042E37D12800FFF777
:100C0000BFFA0600280002F0CBFE010020003200EF
:100C10000AF0C0FFA41922E02700C3E7180005A9C5
:100C2000FFF7D8FE05A80BF05BFBCCE7032900D04B
:100C30001EE7020992B2430F92000B40D31A1C190F
:100C4000C2E705A92800FFF7C5FE05A80BF048FB81
:100C500005A90500020020000AF09CFF6419029B10
:100C60000437BB42BFD10023237005E7032EF6D122
:100C70001A0992B25B0F92001E40961B291DC5E710
:100C8000F0B50D0097B0002806DC1C2000F0F4FB46
:100C90000700380017B0F0BD0C68012123000B409D
:100CA000009306D1042C04D922680F331A40092A74
:100CB00001D00B20EAE7626852100392002A03DC9D
:100CC000009803F081F8E3E7504A019201280BD025
:100CD0006868084208D1042806D902681340042B2A
:100CE00002D102F05DFE019001980BF0F9FA0600C6
:100CF0000F27039B0834013B05935E43039B02903F
:100D00009B00E318049301232068184273D1042840
:100D100071D901680B003B409C46042B03D1FFF7BF
:100D20002FFA861909E0032B6CD162460B099BB29E
:100D3000490F9B0011405A1A9619049B0434A34290
:100D4000E1D1300003F040F8071EA2D02B680793D2
:100D5000029B002B03D0686802F022FE019038004D
:100D600002F01EFE0400009B079A9B00D3189E68A9
:100D7000300002F015FE0123334005000693002BDE
:100D800001D1042E04D809A93000FFF723FE09ADD4
:100D900028000BF0A5FA069B0490002B0ED1042E20
:100DA0000CD90F2133681940032907D11A0992B2CF
:100DB0005B0F92000B40D31A351D04932000049A58
:100DC00029000AF0E7FE049BE418029B002B0AD0DE
:100DD000059B009A934206DD2000029A01990AF0D1
:100DE000D9FE029BE418009B01330093009A039BF9
:100DF0009342B8D14DE709A9FFF7ECFD09A80BF024
:100E00006FFA8EE702F0CCFDF9E7C04613D7000079
:100E100010B50024A04207DD0B6801341C4003D04C
:100E20005C10E343DB171C40611C0122092002F027
:100E300059FF002803D0012364001C43446010BD07
:100E40000A6870B510000125284034D1042A32D92F
:100E50000F24136849681C40092C17D154681B09DA
:100E60009BB22C41A34200D85C1E844205DC0220C8
:100E70000133984206DB00200FE085005519A96078
:100E80000130F2E7840011510130F2E7032C12D156
:100E9000294203D1132000F0EFFA70BD4910FF2959
:100EA000F8D81B099BB204329B00D3189342E2D9B5
:100EB00011700132FAE70B2000F0DEFADBE70000E8
:100EC000F8B5012700254E680C003740AF420ED11F
:100ED0003D00042E0BD90F2233681A40092A10D185
:100EE00072681B099BB25510AB4200D85D1E216889
:100EF000CB0716D54C10002C01DDA5421CDA1220C0
:100F000030E0042A04D13000FFF73AF90500EEE79B
:100F1000032AECD11D09ADB25B0FAD001340ED1AF1
:100F2000E5E72748FFF7E0FC002813D00BF02EF987
:100F3000290008F0EDFD4C1C002F3ED1042E3CD9B9
:100F40000F2332681340092B10D10134A400A45997
:100F50002000F8BD21681B48FFF7C6FC2C000028C4
:100F6000EAD1113000F088FA0400F1E7042B1CD11B
:100F7000300002F015FD0500012C0EDCFFF718F91A
:100F8000461B300002F020FF041EE1D002F008FDF5
:100F9000320029000AF0FEFDDAE72B78013C002B35
:100FA000ADD02800FFF704F9E5E7032B05D134198C
:100FB000E37801245B001C43CAE70B20D2E7C0465C
:100FC00058D2000063D20000F7B54D680F002A0028
:100FD00001210A402FD1042D2DD90F242B68BE6882
:100FE0001C40092C14D169681B099BB24C1001925A
:100FF000A34200D85C1E39682A48FFF775FC002818
:101000002DD00F232A681340092B1DD1012317E08F
:10101000032C10D10E4203D1132000F02DFAFEBD97
:1010200072100192FF2AF7D81A0992B25B0F920050
:101030001C40141BDFE70B20EFE701339A00AE5092
:101040009C42FADA0020EAE7032BFBD12B000133A4
:101050005A1BA242F6DC6A461279DA70F7E7396861
:10106000CB0706D54910002901DD8C4209DA122090
:10107000D3E70D48FFF738FC2100002801D11130DB
:10108000CBE70F232A681340092B03D101318900D4
:101090004E51D7E7032BD5D16B461B796D18EB70FA
:1010A000D0E7C0465FD2000063D2000070B50124D3
:1010B0000868204207D1042805D90F2501680D4092
:1010C000092D02D14468200070BD032D08D10A0902
:1010D00092B24B0F92002B40D31A5B001C43F2E7F5
:1010E000042DF0D102F05CFCFFF776F840000443D9
:1010F000E9E7000010B5034A0B21034804F03AFC6D
:1011000010BDC04600D20000F8D10000002070479A
:10111000042070470120704710B5002002F054FEF3
:1011200010BD00207047002070470020704700204D
:101130007047002070470020704700207047002053
:101140007047000010B5034A0C21034804F012FC5C
:1011500010BDC046E8D2000048D3000070470378B5
:10116000002B03D05AB2002A01DB013070473F2226
:101170009343C03B59424B41C01803789343802BA3
:10118000F4D10130F9E70000F8B50127060014009A
:101190000800394227D104293FD90F230A681A4091
:1011A000042A3AD13C4213D1042C11D922681340AD
:1011B000042B0DD102F0F4FB0500200002F0F0FB3F
:1011C000010028000BF082F800282EDB1FD127E059
:1011D000E30722D502F0E4FB0A2200210BF048F9D4
:1011E0000500601010E0174015D1042A15D90F230F
:1011F00012681340042B10D120004D1002F0D0FBD8
:101200000A2239000BF034F985420EDB08DD002E8E
:1012100009DC00200CE04D10E3E70F22054B1A70AB
:101220000136022EF5D8042002E004207617304063
:10123000F8BDC046B0020020F8B506000024294BD6
:10124000E500ED182B79032B06D00134FF2CF6D1E5
:10125000013CFF3C2000F8BD30000BF041F8E3B248
:1012600002003100180004F0BFFB0028F2D12A6808
:1012700051688842E9D08300D3189B680130F02B75
:10128000F7D101238000083012181A42DDD1042A58
:10129000DBD90F21136819400429D6D11B0998B254
:1012A00001230130800010181842CED10428CCD977
:1012B0000F2203681340042BC7D102F071FB0327F0
:1012C0000500092128000AF0F3FF0028BDD0013FE6
:1012D000451C002FF5D1310028000BF02DF8854278
:1012E000B8D0B2E7A425002010B50124044002D0F4
:1012F0004410200010BD042810D90F2302681340A9
:10130000042B07D102F04CFB21000A220BF0B0F8AD
:101310000400EEE7032B01D10430F5E70D22014B69
:101320001A70E6E7B0020020012210B5024018D181
:10133000042802D903681A0992B201230B4012D182
:10134000042902D90B681B099BB20024934206D1E1
:1013500004309B000431C318984206D301242000B6
:1013600010BD0022E9E70023EFE704780A78002C9B
:1013700001D1002AF2D0013001319442ECD0002496
:10138000EDE70000F7B50700009101933049314BBC
:10139000002A02D002220A70013A00261A601B6855
:1013A000CE54BE4200DBF7BD009AB300D058294BA3
:1013B000274D1C68C8239B0065191C1B012318427C
:1013C00006D0254A4310210028000AF011FF09E049
:1013D000224A002802D004281BD1214A21002800DB
:1013E0000AF006FF1A4C20000AF07AFF194A019B06
:1013F0001060002B0BD07B1EB34208DD194B9842C6
:1014000005D8431C1360202222540022E2540136E6
:10141000C7E7042819D90F2301680B40042B04D116
:1014200002F0BEFA104A0300CDE7092B03D143684E
:101430000E4A5B10C7E7032B08D10A0992B2490F85
:1014400092000B40D31A0A4ABDE70123094ABAE7C2
:10145000B1020020D4050020F4DC000068D20000B6
:101460006ED200001F0300001FE30000B8D500008B
:10147000C7D50000D2D50000014B1870002070477E
:10148000B002002070B501F0E1FF094C0100251DFC
:101490001F2228000AF03CFF28000AF021FF042345
:1014A00004308008000118432060200070BDC04651
:1014B0008C020020C368F0B59D00836889B05D1977
:1014C0000300183306930369069A9F00069B029057
:1014D000DF19436901939B00D3180393CF4B1B780B
:1014E000002B26D17F222B68CD491C1213409B0074
:1014F0005B58043501929F46029B587804F084FEA5
:101500000023029A137027E0C44B1B78002B10D1E4
:101510002B68019A1C121340C14A9B009B5804354A
:10152000E9E7069B3A1DD11ABC4BD82928DD1A22BF
:101530001A70029BB94C9B6821780193EA1A029BAE
:1015400092109B7812021A43029B587804F064FEB2
:101550000023029A23701370029B069A9B680193E2
:10156000ED1A029BAD10DD60069BFE1A029BB610C1
:101570001E61039B9B1A029A9B10536109B0F0BD38
:1015800039001B7817000C60002BD2D12B68019A10
:101590001C121340A24A9B009B580435ABE7069BE4
:1015A0003A1DD11A9D4BD82902DD1A221A70C0E7C4
:1015B00038001B7817002A68291D0260002B01D013
:1015C0000D00B6E76B68019A1C121340944A9B0009
:1015D0009B5808358FE7069B3A1DD11A8F4BD829A7
:1015E00002DD1A221A70A4E73900A4001B782C1916
:1015F00017000C60002B9CD12B68019A1C12134021
:10160000874A9B009B58043575E7069B3A1DD11A03
:10161000824BD82902DD1A221A708AE73900170096
:10162000804AA400A2581B780A60002B00D080E7F3
:101630002B68019A1C121340794A9B009B58043571
:1016400059E7043F774B3A68A400E250734B1B788C
:10165000002B00D06DE72B68019A1C121340704AD2
:101660009B009B58043546E76E4BA400E058FFF7FB
:101670003BFE043F06003868FFF736FE01233618AC
:1016800076001E43674BE650644B1B78002B00D05E
:101690004FE72B68019A1C121340614A9B009B582C
:1016A000043528E7069B391DCA1A5C4BD82A02DD8F
:1016B0001A221A703DE70698039C0122A04202D22A
:1016C00022000C3A126838001B780F000260002BD1
:1016D00000D02EE72B68019A1C121340504A9B0041
:1016E0009B58043507E7069A3B1D991A4B4AD8299F
:1016F00002DD1A2313701CE706990398814219D260
:1017000002000C3A1068484A4010A418241A039AA0
:10171000A400A2583A601F00404B1B78002B00D059
:1017200007E72B68019A1C1213403D4A9B009B5807
:101730000435E0E6182111700022EBE7069B039ABE
:10174000934219D213000C3B1868374B043FE4183E
:1017500013004010241A3A68A400E2502F4B1B7863
:10176000002B00D0E5E62B68019A1C1213402C4A8E
:101770009B009B580435BEE61822284B1A70EDE7F3
:10178000069B039A934228D2274B043FE618140085
:101790000C3C23685B10F31A9B009858FFF7A4FDDC
:1017A00004903868FFF7A0FD2468049B6410341B84
:1017B0001E18012376001E43039BA400E650174B1E
:1017C0001B78002B00D0B4E62B68019A1C12134042
:1017D000134A9B009B5804358DE618220F4B1A7054
:1017E000EDE7069B3A1DD11A0C4BD82902DD1A22CF
:1017F0001A709EE639001700039AA400A2581B78BD
:101800000A60002B00D094E62B68019A1C1213404A
:10181000034A9B009B5804356DE6C046B002002089
:10182000B8D300009C2D0020FDFFFF3F043F039B29
:101830003A68A400E250D64B1B78002B00D078E623
:101840002B68019A1C121340D24A9B009B58043506
:1018500051E6039BA4001C192368043F38685E10FE
:10186000FFF742FD0123361876001E43C84B266061
:101870001B78002B00D05CE62B68019A1C121340E9
:10188000C44A9B009B58043535E6069BA4003F1BC9
:10189000BF4CBB420CD82378002B00D049E62B6804
:1018A000019A1C121340BB4A9B009B58043522E648
:1018B000B94802F065F82378002B00D039E62B6890
:1018C000019A1C121340B34A9B009B58043512E640
:1018D000A300ED18002C00DA3EE6AD4B1B78002B80
:1018E00000D026E62B68019A1C121340A94A9B00DF
:1018F0009B580435FFE5043F3B68042B04D1A3004B
:10190000ED18002C00DA27E6A14B1B78002B00D045
:101910000FE62B68019A1C1213409E4A9B009B58AD
:101920000435E8E5043F3B68042B04D0A300ED1820
:10193000002C00DA10E6964B1B78002B00D0F8E55F
:101940002B68019A1C121340924A9B009B58043545
:10195000D1E501233E1F306818420AD018410138F2
:10196000002809DB01234000A40018432D19306032
:10197000F2E5FFF7B9FCF2E7854B1B78002B01D0AD
:101980003700D6E52B68019A1C121340814A9B0050
:101990009B5837000435AEE5FF2061004000014050
:1019A000FE38FF380143396002993B0089682412F0
:1019B00004916D1A0299AD1089782D020D4385406E
:1019C00005437D6006991700039A521A92108240CF
:1019D00002439A60029B029A9C70E4B26F4BE4004F
:1019E000E35893606A4A1278002A03D008331D0036
:1019F00003979EE51D00019A9B680C351C1213404D
:101A0000644A9B009B58039775E53B1F1C68039A2B
:101A1000069B934232D10A20E30711D4042C18D933
:101A20000F2322681340042B16D1200001F0B8FFC9
:101A30000AF056FCC8239B00984200D918000630D3
:101A4000643004F005F800280FD1043D069B039391
:101A500082E50720042CF3D02000431E9841FA238E
:101A60004042FF3318400730EAE7029B21005878D4
:101A700004F0E4FB0023029A1370E7E7039B039A48
:101A80000C3B1B6802995B109B00D31A0C3B1C603B
:101A90001F1D1300083B1B685A108A70D2B23F49C1
:101AA000D2005B0055589B0A029A9B009560ED1886
:101AB000039B069A043B1B685B109B00D31803939F
:101AC000334B1B78002B00D033E52B68019A1C1296
:101AD0001340304A9B009B5804350CE53B1F1868A7
:101AE000FFF702FCA40006003F1B1E2827DC00288D
:101AF0000DDC274B1B78002B00D01AE52B68019AD0
:101B00001C121340234A9B009B580435F3E401F058
:101B100083FC033E361801F07FFC214B801B98426A
:101B2000F9D81B4B1B78002B00D002E52B68019ADB
:101B30001C121340174A9B009B580435DBE4012319
:101B4000029A137001F068FC029B0A3886195E60E5
:101B500002E53B1F1868FFF7C7FBA40006003F1B08
:101B600000280DDC0A4B1B78002B00D0E1E42B6829
:101B7000019A1C121340074A9B009B580435BAE493
:101B8000084B984210DD1D22014B1A70D1E4C0466B
:101B9000B0020020B8D30000E4D50000A425002046
:101BA0003F420F0080EE36000123029A137001F0CD
:101BB00033FCFA239B005E430A3E3018029B5860B8
:101BC000CAE4A300FF1A002320001A003900FFF71F
:101BD000D9FBD74ED74C3168200002F001F9D64B23
:101BE00031681860200004F0EFF93168200004F03B
:101BF0002CFBD24B1B78002B00D09AE42B68019A67
:101C00001C121340CE4A9B009B58043573E4CB4B07
:101C1000A4001B783F1B002B00D08AE42B68019A9C
:101C20001C121340C64A9B009B58043563E402987B
:101C300003F072FFC14B1B78002B00D079E42B68B6
:101C4000019A1C121340BE4A9B009B58043552E473
:101C50003B1F1B68002B58D13B0001260C3B18682A
:101C600006402FD046103A0001217300083A0B437A
:101C70001360002E00DC95E0012173000B433A1F36
:101C800013603B00083B1B680B419B1B04933B000C
:101C90000C3B186808423BD0049BA4005B188B40A7
:101CA0000B43039AA350A54B1B78002B00D040E4B4
:101CB0002B68019A1C121340A14A9B009B580435C3
:101CC000FFF719FC04281BD90F2302681340092BC6
:101CD00002D143685E10C6E7042B08D101F060FE14
:101CE0000378002BBFD0FFF73AFA0136F8E7032B51
:101CF00006D11609B6B2520FB6001340F61AB2E773
:101D000019228E4B1A70FFF714FC5B105E1EB0E7B1
:101D1000042842D90F2302681340092B05D1049BE4
:101D2000A40002339B001B58BBE7042B2BD1039B61
:101D3000A4001B19079301F033FE0600049C013434
:101D4000012C10DC3000FFF70AFA831B1800049303
:101D500002F03AF8041E0ED001F022FE049A31007F
:101D600009F018FF07E03178013C002906D1122262
:101D70000C00724B1A70079B1C6094E73000FFF751
:101D8000EEF90600DCE7032B07D10122049BA40037
:101D9000C3181B795B00134383E71922674B1A7042
:101DA000FFF7C7FB04357EE7A300069AFB189B1AD2
:101DB000D82B08DD1A22614B1A70FFF7BAFB0122FB
:101DC0001C003A600437631E002CF8DC5B4B1B7868
:101DD000002B01D0FFF7ADFB2B68019A1C121340BA
:101DE000574A9B009B580435FFF785FB069A3B1D1D
:101DF0009B1A524ED82B03DD1A233370FFF799FB41
:101E0000069B039AA40093422AD23B1F1868FFF74F
:101E10006BFA011E21DD039B0C3B1A6852108242B3
:101E20001BDB9007801A474B4018C018039B8000AB
:101E3000C2583B1B1A60414B3F1B1B780437002BD9
:101E400001D0FFF776FB2B68019A1C1213403C4A25
:101E50009B009B580435FFF74EFB20233370EAE7C5
:101E60001823FBE7344BA4001A683B1B1F001A60C1
:101E7000324B04371B78002B01D0FFF75AFB2B683D
:101E8000019A1C1213402E4A9B009B580435FFF701
:101E900032FB3A1F1368042B02D13A00A4002D191B
:101EA000264B1B78002B02D01700FFF742FB2B6854
:101EB00001991C120B4022499B005B581700043506
:101EC000FFF719FB043F3B68042B04D00023A40058
:101ED0003B602D190437194B1B78002B01D0FFF7FD
:101EE00028FB2B68019A1C121340154A9B009B5833
:101EF0000435FFF700FBA3009C46F81A002C23DCF6
:101F00001C2200260D4B1A706346FF1A0B4B06600D
:101F10001B780437002B01D0FFF70BFB2B68019ACD
:101F20001C121340064A9B009B580435FFF7E3FA46
:101F3000D4050020B102002008000020B0020020DB
:101F4000B8D30000FCFFFF3F002103685B100126AF
:101F50008A008258164003D10D22D54B1A70D3E760
:101F60005210934200DD130001318C42EFDC5E0021
:101F700001231E43C8E7A3009C46F81A002C17DC77
:101F80001C220026CA4B1A706346FF1AC84B066013
:101F90001B780437002B01D0FFF7CBFA2B68019A8E
:101FA0001C121340C34A9B009B580435FFF7A3FA49
:101FB000002103685B1001268A008258164003D175
:101FC0000D22BB4B1A70DFE75210934200DA130068
:101FD00001318C42EFDC5E0001231E43D4E73B005D
:101FE0000122083B1968A40011421DD03B1F1B6849
:101FF000134219D0114113410022994200DA0432F0
:102000003B1B1A60AA4B3F1B1B780437002B01D0E7
:10201000FFF78FFA2B68019A1C121340A54A9B0008
:102020009B580435FFF767FA02203B1F1A684042AD
:10203000FFF7AAF83E1B3060E4E73B000120083BB5
:102040001968A40001421ED03B1F1A6802421AD030
:1020500001415010CB0FD217884253413A1B9B00CD
:102060001360934B3F1B1B780437002B01D0FFF705
:1020700060FA2B68019A1C1213408E4A9B009B58F1
:102080000435FFF738FA01203B1F1A684042FFF77A
:102090007BF83E1B3060E4E73B00083B18683B1FC1
:1020A0001968A600BE1B0423814202D0042802D86E
:1020B0000023336016E001231842F9D10F23026890
:1020C0001A40042AF4D1033A1142F1D10429EFD97C
:1020D0000A681340042BEBD1FFF726F9431E984101
:1020E00080003060724BA4001B783F1B0437002B2C
:1020F00001D0FFF71EFA2B68019A1C1213406D4A9B
:102100009B009B580435FFF7F6F93B00083B186825
:102110003B1F1968A600BE1B0023814202D0042881
:1021200002D80423336016E001231842F9D10F23AB
:1021300002681A40042AF4D1033A1142F1D1042969
:10214000EFD90A681340042BEBD1FFF7EDF84342B7
:10215000584180003060564BA4001B783F1B043769
:10216000002B01D0FFF7E5F92B68019A1C121340F0
:10217000504A9B009B580435FFF7BDF93B000122F4
:10218000083B1968A40011421ED03B1F1B68134274
:102190001AD05B104A10D80FC9179A4241413B1B15
:1021A00089001960424B3F1B1B780437002B01D07C
:1021B000FFF7BFF92B68019A1C1213403D4A9B00A0
:1021C0009B580435FFF797F93B1F1A680120FEF76B
:1021D000DBFF3E1B3060E5E73B000122083B19684E
:1021E000A40011421DD03B1F1B68134219D011419E
:1021F00013410022994200DD04323B1B1A602C4B34
:102200003F1B1B780437002B01D0FFF792F92B6896
:10221000019A1C121340274A9B009B580435FFF774
:102220006AF93B1F1A680220FEF7AEFF3E1B3060C2
:10223000E5E73B1F1B68A400043B5A1E93413A1B71
:1022400017009B0013601A4B04371B78002B01D03A
:10225000FFF76FF92B68019A1C121340154A9B0077
:102260009B580435FFF747F93B00083B1868FFF718
:102270003BF83B1F06001868FFF736F80121A40061
:102280003B1B1F00321852000A431A60084B0437E8
:102290001B78002B01D0FFF74CF92B68019A1C1218
:1022A0001340044A9B009B580435FFF724F9C046AD
:1022B000B0020020B8D300003B00083B1868FFF7CD
:1022C00013F83B1F06001868FFF70EF80121A40061
:1022D0003B1B1F00321A52000A431A60E44B0437BA
:1022E0001B78002B01D0FFF724F92B68019A1C12F0
:1022F0001340E04A9B009B580435FFF7FCF83B0075
:10230000083B1868FEF7F0FF3B1F06001868FEF751
:10231000EBFF02000121A4003B1B1F00724352008F
:102320000A431A60D24B04371B78002B01D0FFF709
:1023300000F92B68019A1C121340CE4A9B009B584F
:102340000435FFF7D8F83B1F1868FEF7CDFF061ECF
:1023500017D11F23C64A1370A4003B1B1F001E6029
:10236000C34B04371B78002B01D0FFF7E2F82B6832
:10237000019A1C121340BF4A9B009B580435FFF77B
:10238000BAF83B00083B1868FEF7AEFF310007F0D3
:10239000D9FA012346001E43DEE73B1F1868FEF70B
:1023A000A3FF061E17D11F23B14A1370A4003B1BC5
:1023B0001F001E60AE4B04371B78002B01D0FFF7C7
:1023C000B8F82B68019A1C121340AA4A9B009B582C
:1023D0000435FFF790F83B00083B1868FEF784FFD0
:1023E000310007F095FB01234E001E43DEE73B1F43
:1023F0001868FEF779FFC11743184B400121A4006C
:102400003A1B17005B000B431360994B04371B7892
:10241000002B01D0FFF78DF82B68019A1C12134096
:10242000944A9B009B580435FFF765F8A300FE1AF9
:102430003068012C25D1FEF757FF01230790049344
:1024400009F0A4FE0799002900DC012107F060FBD8
:10245000049BA400C918012349001943844B3F1B66
:102460001B7831600437002B01D0FFF762F82B682E
:10247000019A1C1213407F4A9B009B580435FFF7BA
:102480003AF8FEF731FF04907068FEF72DFF049BC9
:102490000130C31A0793D3E7A300FE1A31002000CE
:1024A000049301F023FE049B3060FF1A704B043745
:1024B0001B78002B01D0FFF73CF82B68019A1C1207
:1024C00013406C4A9B009B580435FFF714F83B00FF
:1024D000083B1868FEF708FF3B1F06001868FEF768
:1024E00003FF02000121A4003B1B1F0032405200E9
:1024F0000A431A605E4B04371B78002B01D0FFF7AC
:1025000018F82B68019A1C1213405A4A9B009B58DA
:102510000435FEF7F0FF3B00083B1868FEF7E4FEC9
:1025200006003B1F1868FEF7DFFE32000121A40001
:102530003B1B1F00024352000A431A604C4B0437F6
:102540001B78002B01D0FEF7F4FF2B68019A1C12B8
:102550001340484A9B009B580435FEF7CCFF3B00D4
:10256000083B1868FEF7C0FE06003B1F1868FEF720
:10257000BBFE32000121A4003B1B1F004240520061
:102580000A431A603A4B04371B78002B01D0FEF740
:10259000D0FF2B68019A1C121340364A9B009B58AF
:1025A0000435FEF7A8FF3B1F1868FEF79DFEC343E6
:1025B0000121A4003A1B17005B000B4313602C4B56
:1025C00004371B78002B01D0FEF7B3FF2B68019A6C
:1025D0001C121340274A9B009B580435FEF78BFFC3
:1025E0003B00083B1868FEF77FFE06003B1F18689B
:1025F000FEF77AFE320082400121A4003B1B1F003F
:1026000052000A431A601A4B04371B78002B01D082
:10261000FEF78FFF2B68019A1C121340154A9B008E
:102620009B580435FEF767FF3B00083B1868FEF730
:102630005BFE06003B1F1868FEF756FE32000241A3
:102640000121A4003B1B1F0052000A431A60084BE3
:1026500004371B78002B01D0FEF76BFF2B68019A23
:102660001C121340034A9B009B580435FEF743FF9E
:10267000B0020020B8D300003B000C3B1868FEF706
:1026800033FE3B00083B06001868FEF72DFEF117ED
:102690000200C317300007F08DFA3B1F049005912C
:1026A0001868FEF721FE02000498059907F036FA33
:1026B0000123A4003E1B370040001843E54B306067
:1026C0001B780437002B01D0FEF733FF2B68019AEB
:1026D0001C121340E04A9B009B580435FEF70BFF89
:1026E000A300FE1A310020000493FEF791FB049B27
:1026F0003060FF1AD74B04371B78002B01D0FEF750
:1027000018FF2B68019A1C121340D34A9B009B5858
:102710000435FEF7F0FEA300FF1A39002000FEF793
:102720008FFBCC4B1B78002B01D0FEF702FF2B68F0
:10273000019A1C121340C84A9B009B580435FEF7AF
:10274000DAFEA300FE1A310020000493FEF7B8FB66
:10275000049B3060FF1ABF4B04371B78002B01D05D
:10276000FEF7E7FE2B68019A1C121340BA4A9B0041
:102770009B580435FEF7BFFEA300FF1A3900200066
:10278000FEF722FCB34B1B78002B01D0FEF7D1FEE5
:102790002B68019A1C121340AF4A9B009B580435CA
:1027A000FEF7A9FEA300FE1A310020000493FEF7F5
:1027B0007DFC049B3060FF1AA64B04371B78002B6E
:1027C00001D0FEF7B6FE2B68019A1C121340A24AF4
:1027D0009B009B580435FEF78EFE3B1F186801F0E6
:1027E000DFF83A000121083A12680300A4000A4207
:1027F00029D1042A0CD910680F221040013808286A
:102800000FD807F00BF8052026220E0E0E0E24001E
:102810009249180009F05AFD434258413B1B800081
:1028200018608C4B3F1B1B780437002B01D0FEF740
:1028300080FE2B68019A1C121340874A9B009B580C
:102840000435FEF758FE8649E3E78649E1E7864905
:10285000DFE78649DDE7069B3E1DF31A7D4CD82B4A
:1028600003DD1A232370FEF764FE00F0DFFD012272
:102870003B0040001043186023783700002B01D044
:10288000FEF757FE2B68019A1C121340724A9B00F8
:102890009B580435FEF72FFE069B3E1DF31A6D4C28
:1028A000D82B03DD1A232370FEF743FE00F0B4FD9E
:1028B0006F4A4000104001223B001043186023780B
:1028C0003700002B01D0FEF734FE2B68019A1C1252
:1028D0001340614A9B009B580435FEF70CFE069A94
:1028E0003B1D9B1A5B4CD82B03DD1A232370FEF78C
:1028F00020FE00F09BFD5F4B1A68831A904201D2C4
:102900005D4A9B1801213A005B000B43136023785A
:102910000437002B01D0FEF70CFE2B68019A1C1225
:1029200013404D4A9B009B580435FEF7E4FD00F030
:102930007DFD504BA4001860464B3F1B1B78002BBD
:1029400001D0FEF7F6FD2B68019A1C121340424A93
:102950009B009B580435FEF7CEFD00F075FDA300EB
:10296000002810D1FF1A3B4B1B78002B01D0FEF73B
:10297000E0FD2B68019A1C121340374A9B009B58BC
:102980000435FEF7B8FD3E00FF1A012320001A00AF
:102990003900FEF7F7FC394C2068643003F058F832
:1029A000002803D1043D3700FEF7D6FD029B2168C5
:1029B0005A78334803F05BFC0123029A137000F04D
:1029C0002BFD304B22681B68063253431818FFF763
:1029D000F5F800F039FDA300002810D1FF1A1D4BB7
:1029E0001B78002B01D0FEF7A4FD2B68019A1C1266
:1029F0001340194A9B009B580435FEF77CFD3E00AE
:102A0000FF1A2000012300223900FEF7BBFC1B4CFB
:102A10002068643003F01CF80028C3D0184803F085
:102A2000C3F9C9E7A4003E1BFEF72CFD3700094B94
:102A300030601B780437002B01D0FEF77AFD2B683D
:102A4000019A1C121340044A9B009B580435FEF760
:102A500052FDC046B0020020B8D30000F4D50000FB
:102A6000FCD5000003D600000AD600000FD60000F7
:102A7000FEFFFF7FDC05002037894100D4050020E0
:102A8000B102002004000020FB4BA4001B783F1B78
:102A9000002B01D0FEF74DFD2B68019A1C1213404C
:102AA000F64A9B009B580435FEF725FDA4003E1B0B
:102AB000300000F0F6FC3700EF4B30601B78043735
:102AC000002B01D0FEF735FD2B68019A1C12134034
:102AD000EA4A9B009B580435FEF70DFDA4003E1BFF
:102AE000300000F0E0FC3700E34B30601B78043727
:102AF000002B01D0FEF71DFD2B68019A1C1213401C
:102B0000DE4A9B009B580435FEF7F5FCA300FE1A35
:102B100031002000049300F0C9FC049B3060FF1AD0
:102B2000D54B04371B78002B01D0FEF702FD2B6834
:102B3000019A1C121340D14A9B009B580435FEF7A2
:102B4000DAFCA4003F1B380000F0E2FCCA4B1B7803
:102B5000002B01D0FEF7EDFC2B68019A1C121340EC
:102B6000C64A9B009B580435FEF7C5FCA300FE1A1D
:102B700031002000049300F0F3FC049B3060FF1A46
:102B8000BD4B04371B78002B01D0FEF7D2FC2B681D
:102B9000019A1C121340B94A9B009B580435FEF75A
:102BA000AAFCA4003F1B380000F01CFDB24B1B78B0
:102BB000002B01D0FEF7BDFC2B68019A1C121340BC
:102BC000AE4A9B009B580435FEF795FC012120007E
:102BD00000F0F0FCA84B1B78002B01D0FEF7A9FCFD
:102BE0002B68019A1C121340A44A9B009B58043581
:102BF000FEF781FC0021200000F0DCFC9E4B1B78DE
:102C0000002B01D0FEF795FC2B68019A1C12134093
:102C10009A4A9B009B580435FEF76DFCA4003E1BAE
:102C2000300000F001FD3700934B30601B78043713
:102C3000002B01D0FEF77DFC2B68019A1C1213407B
:102C40008E4A9B009B580435FEF755FCA4003E1BA2
:102C5000300000F0FDFC3700874B30601B780437F4
:102C6000002B01D0FEF765FC2B68019A1C12134063
:102C7000824A9B009B580435FEF73DFCA4003F1B95
:102C8000380000F0BFFC7C4B1B78002B01D0FEF716
:102C900050FC2B68019A1C121340784A9B009B58E9
:102CA0000435FEF728FCA4003F1B380003F0E8FEC3
:102CB000714B1B78002B01D0FEF73BFC2B68019A6F
:102CC0001C1213406D4A9B009B580435FEF713FC01
:102CD000A4003E1B300003F07BFF3700664B3060E2
:102CE0001B780437002B01D0FEF723FC2B68019AD8
:102CF0001C121340614A9B009B580435FEF7FBFBF6
:102D0000A4003F1B380003F055FE5B4B1B78002BE3
:102D100001D0FEF70EFC2B68019A1C121340574A93
:102D20009B009B580435FEF7E6FBA4003E1B3000D9
:102D300003F05AFE3700504B30601B780437002BED
:102D400001D0FEF7F6FB2B68019A1C1213404B4A88
:102D50009B009B580435FEF7CEFBA300FF1A3900F9
:102D6000200001F025FD444B1B78002B01D0FEF71D
:102D7000E0FB2B68019A1C121340404A9B009B58B1
:102D80000435FEF7B8FBA300FF1A3900200001F05C
:102D900023FB394B1B78002B01D0FEF7CAFB2B68B5
:102DA000019A1C121340354A9B009B580435FEF7CC
:102DB000A2FBA300FF1A3900200001F031FC2E4BCA
:102DC0001B78002B01D0FEF7B4FB2B68019A1C1274
:102DD00013402A4A9B009B580435FEF78CFBA30046
:102DE000FF1A3900200001F043FC234B1B78002B15
:102DF00001D0FEF79EFB2B68019A1C1213401F4A5C
:102E00009B009B580435FEF776FBA300FE1A3100A9
:102E10002000049303F074FF049B3060FF1A164BEC
:102E200004371B78002B01D0FEF783FB2B68019A37
:102E30001C121340114A9B009B580435FEF75BFBA4
:102E4000A300FE1A31002000049303F061FF049BED
:102E50003060FF1A084B04371B78002B01D0FEF7B7
:102E600068FB2B68019A1C121340044A9B009B5874
:102E70000435FEF740FBC046B0020020B8D3000086
:102E8000A300FE1A31002000049303F049FF049BC5
:102E90003060FF1A984B04371B78002B01D0FEF7E7
:102EA00048FB2B68019A1C121340944A9B009B58C4
:102EB0000435FEF720FBA300FE1A31002000049326
:102EC00003F04AFC049B3060FF1A8B4B04371B78DD
:102ED000002B01D0FEF72DFB2B68019A1C1213402A
:102EE000864A9B009B580435FEF705FBA300FF1A9A
:102EF0003900200001F0A8FA7F4B1B78002B01D08D
:102F0000FEF717FB2B68019A1C1213407B4A9B00AB
:102F10009B580435FEF7EFFAA300FF1A3900200092
:102F200001F0CEFB744B1B78002B01D0FEF701FBA8
:102F30002B68019A1C121340704A9B009B58043561
:102F4000FEF7D9FAA300FE1A31002000049301F025
:102F500033FB049B3060FF1A674B04371B78002B50
:102F600001D0FEF7E6FA2B68019A1C121340634A5F
:102F70009B009B580435FEF7BEFAA300FF1A3900E8
:102F8000200001F0E1FA5C4B1B78002B01D0FEF72A
:102F9000D0FA2B68019A1C121340584A9B009B5888
:102FA0000435FEF7A8FA002C55DD3B1F1E68012CE6
:102FB0000CD1264207D1042E05D90F2332683000E8
:102FC0001340042B11D00120404212E0022CFAD110
:102FD0003B00083B186801231842F4D10428F2D9B9
:102FE00002680E331340042BEDD100F0D9FCFEF73C
:102FF00023F9A300FF1A00282DDB0022022C11D197
:1030000001233340934222D1042E20D931680F325C
:103010000A40092A1BD172685210D2B2910099421B
:1030200010D17F180002104304003A00069B0C32B6
:10303000D31AD82B01DCFEF7AFFC1A222E4B1A70E4
:10304000FEF777FAF418A468FC500433E7E73E6013
:1030500001220437E6E700233B60274B3A1D1B782B
:10306000002B02D01700FEF764FA2B6801991C129E
:103070000B4022499B005B5817000435FEF73BFAD2
:10308000069B029AFB1A9B101361A300FF1A3900DA
:10309000200002F0C7FE184B1B78002B01D0FEF772
:1030A00048FA2B68019A1C121340144A9B009B5843
:1030B0000435FEF720FA069B029AFB1A9B10136157
:1030C000A300FE1A31002000049302F0ABFE049B23
:1030D0003060FF1A084B04371B78002B01D0FEF735
:1030E00028FA2B68019A1C121340044A9B009B5833
:1030F0000435FEF700FAC046B0020020B8D3000045
:103100000023F7B55A1E0192002B07DA01F066FB87
:1031100002F094FF03F00AF919230193002630000E
:10312000194B1968B14212DD184B1A6801328A42F4
:103130000FDAF0241A601D68154F6C43E35D002B15
:103140001FD0E419022B06D12000FEF7B3F9019B32
:10315000D8E70022EDE7012B0DD1002801D100F0C6
:103160005BF9F0226A43BB185B680A49C31A8B42B9
:1031700001D80223BB54F0235D43054BEB5C022BCB
:10318000E2D00136CCE7C046D80500200000002080
:10319000441C00203F420F0080220B4B52001A605B
:1031A0000121A822A920094BD20019649A58C00015
:1031B00005321A5006481A50C122C020920000035E
:1031C0009850044B1970704700E100E00080004007
:1031D0004C0500000306002004207047F8B550C9D4
:1031E000012322001A40101E2DD03340181E2AD071
:1031F000641000201C2C26D81D4B761035009E42F2
:1032000000DD1D001B4F3B5D012B05D0012120007F
:1032100004F0F4FE01233B55174B1B78002B01D122
:10322000FFF7BAFF0023154A9E420DDCFF25144923
:103230001448D65CB44202D15E007052D5540133BA
:10324000042BF6D10420F8BDD15C8C4203D10C4A8A
:103250005B009D52F6E70133042BF5D10023D15CCE
:10326000FF2901D1D454F2E70133042BF7D1E9E768
:1032700088130000E4050020030600201C00002045
:103280000E000020DC05000070B530C901232200CB
:103290001A40101E1BD02B40181E18D064101C2C76
:1032A00000D90024154E335D012B05D001212000EB
:1032B00004F0A4FE0123335569100800104A1038A9
:1032C000104B904204D9012252421A60042070BD72
:1032D0001C600D4806F036FB0C4B040018800C4BAC
:1032E0001B78002B01D1FFF757FF0122094B9A648D
:1032F000A922D200995864189C50E7E7E405002001
:10330000908601001800002020A107000C0000207A
:103310000306002000800040F8B501260D68340047
:10332000B04200DD4C682B003340181E0BD0230048
:103330003340181E07D06D10002D05DCA12300209E
:103340001E4ADB00D650F8BD641000201C2CFAD8B1
:103350001B4F3B5D012B04D00121200004F04EFEE9
:103360003E552900174806F0EDFA0A21053006F00F
:10337000E9FA154BA400E258144B12021343A2229F
:103380001349D2008B50134C0C4B9C50124C1951CA
:10339000012412495C50124B196900219950114ABD
:1033A000904200DD1000A8228021D2009850012216
:1033B00089005A5004201A60C5E7C04600F0014059
:1033C000E405002000B4C40474E600000300030018
:1033D0000060004040A1004014050000040500000A
:1033E00000A00040FFFF0000030010B50120002BEB
:1033F00002DC1B30FEF740F810BD0420704710B50A
:10340000002803DC1C20FEF737F810BD0B680020F5
:10341000DB07FAD40D30F6E70122034B1A64A82229
:10342000D20098587047C046008000400122054BEA
:1034300010B51A64A822FA21D2009858890006F023
:10344000F7F910BD00800040012070470048704728
:1034500074D600001D20704770B5054E0400335C23
:103460000D008B4202D004F0C9FD355570BDC04639
:10347000E405002070B50024084D635D012B09D1DF
:103480000021200004F0D8FD0021200004F0B6FD4A
:103490000023635501341D2CEED170BDE4050020DE
:1034A00070470D2070473B2070470000F8B501249D
:1034B0000B6806000D00234204D10D20FDF7DCFF50
:1034C0002000F8BD5B102000052BFAD80E4A9B00A7
:1034D0009C580E4F3B5D002B05D00021200004F0CE
:1034E0008DFD00233B55012E06DD6B68042B03D1B7
:1034F0000221200004F082FD200004F02DFC0124B4
:1035000040002043DDE7C0465CD60000E405002013
:10351000F8B501260568354202D04468344203D12B
:103520000D20FDF7A9FFF8BD6D101C2DFBD80A4F2B
:103530007B5D012B04D03100280004F05FFD7E5537
:10354000064964108C4202DCE143C917214028007F
:1035500004F088FCE7E7C046E4050020FF03000014
:1035600070B501240D68254204D10D20FDF784FFBC
:10357000200070BD6D101C2D17D80024012804DD1B
:103580004C68043C63425C416400094E735DA34295
:1035900004D02100280004F031FD7455280004F007
:1035A00061FD03000420012BE3D00020E1E7C046C9
:1035B000E405002070B504000D001C280ED8084E4C
:1035C000335C012B04D0012104F018FD0123335595
:1035D000290020004D1EA94104F02EFD70BDC046FB
:1035E000E4050020036810B5DA0703D40D20FDF7C9
:1035F00043FF10BD4168581004394A425141FFF75A
:10360000D9FFF6E737B569460A00064B30CB30C222
:1036100003680220042B02D101F002F837BD01F04B
:1036200027F8FBE71CD6000010B5084C6379002B87
:1036300005D00021052004F0E1FC00236371052082
:1036400004F010FD43425841800010BDE405002005
:1036500010B5084CE37A002B05D000210B2004F0B4
:10366000CDFC0023E3720B2004F0FCFC43425841E4
:10367000800010BDE4050020A02200230349D200F1
:103680008B50034910328B507047C04600F0014008
:1036900000600040F7B52F4D2F4EEB6C002B14D07F
:1036A000A9240023E4003759EB642C4B1868002848
:1036B0000BDB2B4B19784A425141C9B2197004F007
:1036C000BBFC284B1B88DF1937512B6D002B38D0E2
:1036D0000021254B254FF45829653A780193244D54
:1036E0008A4206D02B68032B03D8224AD05C04F010
:1036F000A3FC2B68204A0133134004D50422013B6C
:103700005242134301331B4900228C462B60042B89
:1037100018D06046C05C591CFF2802D10B00012262
:10372000F5E7002A00D02B60012104F085FC01237D
:103730003B702B68114A5B009B5A0C34E418019BC8
:10374000F450F7BD01235B422B6000233B700C4B10
:10375000F4E7C046FC8000400080004018000020D4
:10376000020600200C0000204C050000010600208D
:10377000E00500201C000020030000800E00002057
:103780005C460000084B094AFF201A805A809A8044
:10379000DA800023064A07491370074A0870487008
:1037A0008870C870136070470E000020DC050000B0
:1037B000010600201C000020E00500200122024B31
:1037C00052421A607047C0461800002010B5034AE4
:1037D0000721034802F0CEF810BDC04624D60000F1
:1037E00026DE0000E12170B54902194804F02AF8EC
:1037F000002401220320174B17491A615C50043141
:1038000058508018083158501A60063004F09EFA5B
:10381000FF21124AA15401341D2CFBD101220020AA
:103820000F4B01001A6004230E4A0F4D1468002C40
:10383000FCD02C680002013B20431160002BF5D125
:1038400001220A4B1A6004F0B9F901F013F970BDB6
:10385000CC1B00200080004004050000E40500208F
:1038600000D0004000D1004008D5004004D0004006
:10387000F8B50B4E070030000D0004F02BF80400E3
:10388000A84200DD2C003D00EB1B9C4205DD300012
:1038900004F02AF828700135F6E72000F8BDC0468C
:1038A000CC1B002010B50100014803F0D3FF10BD70
:1038B000CC1B002010B5054C200003F0D9FFE121FE
:1038C0002000490203F0BEFF10BDC046CC1B002003
:1038D000C3070CD4064B1B68834208D8054B1B68F2
:1038E000984204D8031F1B68002B00D018007047B3
:1038F0000C060020080600200023012210B50A480B
:10390000990001334250642BFAD1084C084B002136
:103910001A602000074A08F059F9074B074A63600C
:10392000074B1A6010BDC0469C2D002010060020D9
:1039300008000020D40900003027000014060020F1
:103940000406002010B5044B044A1A60044B054AD3
:103950001A60FFF7D1FF10BD0C06002010060020F2
:1039600008060020E40F0020044B1B6818680009BB
:1039700080B20238C343DB171840704704060020AA
:1039800000B59BB00200054901A808F063FC01A83E
:1039900002F026FA02F0CAFCFCE7C04603D700009A
:1039A0000B4BC20704D4042804D80A4B00D00A4B9E
:1039B000180070470F2203681A40031D042AF7D02D
:1039C000064B092AF4D0064B032AF1D0054BEFE74A
:1039D000DDD600006ED2000068D20000E7D60000FD
:1039E000F7D60000EED600000020064A0649131F55
:1039F000186013681B099BB202339B00D2188A42DD
:103A0000F5D3704714060020E40F0020F7B50F240B
:103A10000126314B314A1968314B324D1868136811
:103A20001F002740072F26D813681B099BB20233BB
:103A30009B00D218AA42F2D300242B4EA500AD1948
:103A40002868FFF745FF01342860642CF6D1274C25
:103A50002068FFF73DFF2060254C2068002802D039
:103A6000FFF736FF20600025224B1B680093009B68
:103A70009D4214DBF7BD1B099BB29B00D3189A42F1
:103A8000D2D01F68374208D1B94206D2B84204D317
:103A9000043F3F68002F00D01F60043BEFE7F02396
:103AA0006B43154A9B181A78002A01D10135DEE7CD
:103AB0001F693C2300266B43DB199B0001930136F1
:103AC000BB1BF3D4019BB4001C1B0B4B1C19A0693E
:103AD000FFF7FEFEA061F2E70C06002014060020AE
:103AE00008060020E40F00209C2D00200800002084
:103AF000E40F0020D8050020441C0020F7B5012465
:103B0000204246D1234B1B689C46984241D3224B0E
:103B10001B68019398423CD8031F1B68002B38D1C7
:103B20000200036800941B099BB2002B0FD100997F
:103B3000131F196090422CD015682B1F1B68990029
:103B400069180C68013B14600A602A00EDE79D00CB
:103B500055192968009C214219D18C4517D8019C20
:103B60008C4214D30E1F3468002C10D10F680F3410
:103B70003C40072C08D92F60151F2B600B680A608A
:103B80001B099BB20A00D0E700993160CDE7013BE9
:103B9000CBE7F7BD0C060020080600200D4970B5E4
:103BA0000A000D4D1368141F1B0926689BB2981C50
:103BB000002E0BD000238A4200D00B00236083002C
:103BC000C91880001218AA42ECD370BD1B01136003
:103BD000F7E7C04614060020E40F0020F8B5124CA9
:103BE00027000F223B681D09ADB213420DD06E1C99
:103BF000B600A74204D032003900200007F0D3FFFE
:103C00000022A3190436A4191A600235AD00074B2F
:103C10007F199F42E5D31B1B9B10013B1B012360B7
:103C2000034B1C60F8BDC04614060020E40F0020C2
:103C300004060020F0B59BB0FFF7EEFB0024070060
:103C4000214AA300D0580134FFF758FF642CF7D164
:103C50001E4B1868FFF752FF1D4B1868002801D053
:103C6000FFF74CFF00261B4B1B689E4217DBFFF73C
:103C700095FFFFF7CBFEFFF7B1FFFFF7CDFB164B2C
:103C8000C21B1B6815491B6801A81B099BB2023B9C
:103C900008F0E0FA01A802F0A3F81BB0F0BDF0258F
:103CA00075430F4BED182B78002B01D10136DAE765
:103CB0002B695C1E002CF9DBA300EB189869FFF759
:103CC0001DFF013CF6E7C0469C2D002008000020A7
:103CD000E40F0020D805002004060020BDD6000017
:103CE000441C0020F7B5174D4F1C2B6806001B68BD
:103CF0000C001B099BB201929F420BDBFFF79AFF5E
:103D00002B681B681B099BB29F4203DB0A20FDF74F
:103D1000B3FBFEBD2868A71CBA00DB1B81181B0182
:103D20000B6029600021031F19600F231E40030050
:103D30002401264340C3083A9A189A42E9D90199C6
:103D400002C3FAE704060020F7B50300012213407E
:103D500004000D000193002B2BD1174B1B688342ED
:103D600027D8164B1B68834223D90F23144F386082
:103D700000681840FFF7B6FF019B3C68061E3B60D9
:103D800017D0236804301B099BB29D4200DD1D0043
:103D9000AA00211D251F07F0FDFEFFF725FE2E605E
:103DA000FFF734FE00232B602268064B134023608C
:103DB00034002000FEBDC0460C060020080600208E
:103DC000E40F0020F0FF0F000323043010B5C117EB
:103DD00019400918891000220420FFF783FF10BD45
:103DE00070B5050008000C00FFF7EEFF0023002867
:103DF00004D170BDE95CC21811710133A342F9DB33
:103E0000E343DB171C40002304192371F1E7F0B5ED
:103E10000C009BB0022804DC1C20FDF72DFB1BB01E
:103E2000F0BD01230868184206D1042804D90F26E2
:103E300001683140042901D00E20EEE761680D00D1
:103E40001D40F9D10429F7D90A683240042AF3D178
:103E5000A2681A4201D10D20DFE7FFF7A1FD06009D
:103E60006068FFF79DFDA768010001AC7F1030007E
:103E7000257003F037F939006423220003F097F925
:103E8000200008F02DFA01002000FFF7A9FFC6E787
:103E900010B51C4CA544041E02D1FFF795FF0BE0A2
:103EA00003F038F80138062828D805F0B7FC0909CE
:103EB00011182904240000208023DB009D4410BD3C
:103EC000200003F0A3F8011B2000FFF789FFF3E7B0
:103ED000200003F049F8430001201843ECE780225A
:103EE0006946D200200003F056F8684608F0F8F959
:103EF00001006846E9E704210348E6E70020CCE733
:103F00000420D9E700FCFFFF4CD7000070B50C007F
:103F1000022803DC1C20FDF7AFFA70BD01230868FE
:103F2000184206D1042804D90F2501682940042924
:103F300001D00E20EFE761681942FAD10429F8D9BF
:103F40000A682A40042AF4D1A2681A4201D10D203D
:103F5000E1E7FFF725FD05006068FFF721FDA46894
:103F600001006410280003F0BDF8210003F0FAF806
:103F7000FFF78EFFD1E770B50D00012803DC1C2090
:103F8000FDF77AFA70BD01240868204206D10428A2
:103F900004D90F2102680A40042A01D00E20EFE75D
:103FA0006A682242FAD1042AF8D913680B40042B1C
:103FB000F4D1FFF7F5FC06006868FFF7F1FC01009B
:103FC000300003F08FF803F011F940002043D9E7E7
:103FD000F8B507000C001C20012F0BDD0125086837
:103FE000284206D1042804D90F2102680A40042A75
:103FF00003D00E20FDF740FAF8BD62682A42F8D1DE
:10400000042AF6D913680B40042BF2D1FFF7C8FC41
:1040100006006068FFF7C4FC0100022F14D0A468FA
:104020002C4211D06410300003F05CF8050002F05F
:1040300071FF012811D1002C02DD0135012C06D1C0
:104040002800FFF725FFD7E701246442EBE72800AB
:1040500002F0E9FF013C0500F0E70228F0D1002C56
:10406000EEDD0135012CEBD000222800110003F019
:104070000CF802F0D8FF013C0500F3E710B501246D
:104080000868044016D04410200005F0EFFE1549E2
:1040900005F0BAFD07F0A0FC04F0F2F80022124B84
:1040A00006F054FE04F094F807F026FC43000120CB
:1040B000184310BD042810D90F2302681340042BA5
:1040C00007D1FFF76DFC21000A2208F0D1F90400A6
:1040D000DAE7032B01D10430F5E70D20FDF7CCF929
:1040E000D2E7C046D30237390000D040086870B527
:1040F00001240500254006D1042804D90F230268B5
:104100001340042B03D00E20FDF7B6F970BDFFF766
:1041100047FC03782900233B5A4253411022C01820
:1041200008F0A6F980239B05C218044B9A4201D9D6
:104130001420E9E740002043E8E7C046FFFFFF3FC7
:1041400010B5034A0621034801F014FC10BDC04617
:104150001CD7000014D700000020704710B51E20A7
:10416000FDF78AF910BD10B51E20FDF785F910BDC9
:1041700010B51E20FDF780F910BD10B51E20FDF70B
:104180007BF910BD10B51E20FDF776F910BD10B5F6
:104190001E20FDF771F910BD10B51E20FDF76CF95A
:1041A00010BD10B51E20FDF767F910BD10B51E201B
:1041B000FDF762F910BD10B51E20FDF75DF910BDC9
:1041C00010B51E20FDF758F910BD10B51E20FDF7E3
:1041D00053F910BD10B51E20FDF74EF910BD10B5F6
:1041E0001E20FDF749F910BD10B51E20FDF744F95A
:1041F00010BD10B51E20FDF73FF910BD10B5034AE4
:104200001121034801F0B6FB10BDC04688D700005D
:1042100010D800000120034B1860034B1B6883403B
:104220001843704708100020E80F0020F0B5EFF3A6
:1042300010810123194083F31088134C134AA446BC
:104240001268134E013A9340124F134A002B17D0B5
:10425000146803420FD03D682C60C046C046C0467B
:10426000C046C046C046C046C0460C4C15682468CF
:1042700025605B08EAE765462C6014683460F8E75F
:1042800081F31088F0BDC0460805005020000020D2
:104290000C050050F40F0020FC0F0020F00F002050
:1042A00030B585B001AD0C220649280007F072FC3C
:1042B0000024285D01210134FFF7CEF80C2CF8D141
:1042C00005B030BDF9D80000F7B56A463B4B01AEEA
:1042D00013800A2393703A4B33801C23B370FFF78B
:1042E0009BF8384B384DC0182B68984201D20023F8
:1042F0002B602C68002C41D1375D01213800FFF77D
:10430000ABF801340021380003F096FE032CF3D102
:10431000002401276B461E5D39003000FFF79CF832
:1043200001343900300003F087FE032CF2D1C8209D
:104330000138C046C046C046C046C046C046C0461A
:10434000C046C046C046C046C046F1D16B460021BB
:104350001878FFF781F86B4600215878FFF77CF852
:104360006B4600219878FFF777F8FFF755F8FA23A6
:1043700000241B01C01828602000FEBDFFF74CF888
:104380002B6800249842F7D3032003F0E5FC0600D5
:10439000042003F0E1FC36180A2003F0DDFC0B4B8F
:1043A0009B1B181A0A4BA04206DB18600023094A1F
:1043B0002B6013600124DFE71C60F7E703040000B3
:1043C0001A1B00001027000000100020E30300006B
:1043D000E80F0020081000200022054B10B51A60DD
:1043E000044B1B68934201D002F034FD002010BD45
:1043F00004100020F01A002010B5041E10DA00246A
:104400000A4BA400E25801239340094A094913606A
:10441000094A1160094A0A4911600A4A136010BD2D
:10442000FFF718F8A042EADDEAE7C04674E60000AC
:10443000FC0F002008050050F40F0020F00F0020B2
:104440000C05005018050050F0B53B4B85B01B68BB
:104450000C00002B03D101204042FFF7CDFF246860
:1044600001222700174028D0FF236012184033494B
:104470006714661040431F401E4005F063FA0504B0
:1044800038002E49784305F05DFA000205433000FC
:104490002A49704305F056FA294B28431B68202B04
:1044A00006D16400A40E274BA400E3580002184371
:1044B000FFF7BCFE002005B0F0BD042CFAD90F2395
:1044C00021680B40092BF5D1636803925B100193BF
:1044D000019B9F42EEDABB00E3189E68039B1E42DD
:1044E00028D0FF237012184072101A401349751417
:1044F00040431D40009205F025FA030428000F49AF
:104500006843029305F01EFA029D000205430098DD
:104510000A49404305F016FA094B28431B68202B33
:1045200006D17600B60E074BB600F55800022843B8
:10453000FFF77CFE0137CBE7FC0F00205906000097
:1045400020000020E0DA00000200086810B5C30770
:104550000FD540101823012A03DD4A68042A00D130
:104560000833054A1360FEF79BFFFFF745FF002065
:1045700010BD01204042EDE72000002010B50124CD
:10458000044002D04410200010BD042810D90F238D
:1045900002681340042B07D1FFF702FA21000A2218
:1045A00007F066FF0400EEE7032B01D10430F5E7C6
:1045B0000D20FCF761FFE6E70868F8B5C3071AD5D8
:1045C000FFF7DCFF0300203B5E2B25D8052043438B
:1045D00001221D180020114E9D4219D005211024E2
:1045E000F75C3C4200D08018013952006410002969
:1045F000F7D10133F0E704280ED90F2203681A40DF
:10460000042A09D11B099BB2002B05D00379DAE7F4
:10461000012340001843F8BD0120FCE705D9000044
:1046200070B508680D00FFF7A9FF04006868FFF780
:10463000A5FF621E0100042A14D8451E042D11D8BE
:1046400005236B439B18012215009D402B00064853
:1046500005682B430360054B1B68002B02D020002C
:1046600002F0F9FB002070BD04100020F01A0020B9
:1046700070B508680D00FFF781FF04006868FFF758
:104680007DFF621E0100042A13D8451E042D10D898
:1046900005236B439B1801229A4007480368934304
:1046A0000360064B1B68002B03D00022200002F0A1
:1046B000D2FB002070BDC04604100020F01A00207C
:1046C000F0B5050089B008680C00FFF757FF0690A9
:1046D000022D36DD6068FFF751FF0190A068FFF7FB
:1046E0004DFF04000127231D661E0793731C0293D0
:1046F000079B9E4235D0052373430593019B019D83
:1047000005330493049BAB421ED0042E16D86B1EB7
:10471000042B13D80122059B2349013B5B199A40C6
:104720009446224A0B681068069A3A4003920DD0CC
:1047300062461A430A60012200280DD17F0001352C
:10474000E0E701240194CDE7029ECFE76246934360
:104750000B600028F2D0039A0299280002F07BFB3C
:10476000ECE7019B1E1D042E1AD8012C18D1002540
:1047700005273B0021006B439B1999400B000A4A17
:10478000013511689943094B11601B68002B05D056
:10479000019B0022581D290002F05DFB052DE8D188
:1047A000002009B0F0BDC04604100020F01A00201F
:1047B000086810B5C30703D5FFF7E0FE054B186086
:1047C000054B1B68002B03D0024B186802F044FB1A
:1047D000002010BD04100020F01A00207FB5A04C6E
:1047E0002368002B0AD19F4A1268002A06D19E4BEB
:1047F0001B68002B01D0FFF767FD7FBD9B4D2A682A
:10480000002A26D1984A1268002A1BD0FFF75CFDC7
:104810000028F2D0FFF744FD924B24681A681C6010
:10482000002A16D0002C14D101AD0C22904928008A
:1048300007F0B0F9285D00210134FEF70DFE0C2CC5
:10484000F8D1DAE7874A1268002AE5D1002BE3D0D5
:10485000E0E700211A2003F0EFFB00211B2003F00A
:10486000EBFB00211C2003F0E7FB2E68012E5CD03F
:10487000022E00D1A2E0002E50D101363100794C39
:1048800003202368994303F0D7FB042021680140EB
:104890004B42594103F0D0FB102123680A201940F4
:1048A0004B42594103F0C8FB80212368090119409C
:1048B0004B425941062003F0BFFB802123680902C7
:1048C00019404B425941072003F0B6FB8021236871
:1048D000490219404B425941092003F0ADFB8021A8
:1048E0002368890219404B425941192003F0A4FB67
:1048F00080212368C90219404B425941182003F016
:104900009BFB802321681B0319404B425941172010
:1049100003F092FB31001A2003F08EFB2B68032179
:10492000581C05F0F5F8296067E702214D4C172067
:10493000236819404B42594103F07EFB082123684C
:10494000182019404B42594103F076FB802123681F
:10495000C90019404B425941042003F06DFB8021EE
:104960002368490119404B4259410A2003F064FB76
:1049700080212368C90119404B425941032003F0AB
:104980005BFB80212368890319404B425941092070
:1049900003F052FB802321681B0419404B4259410C
:1049A000192003F049FB3100062003F045FB3100DC
:1049B000072003F041FB31001B20ADE72021294CEB
:1049C0001720236819404B42594103F035FB402121
:1049D0002368182019404B42594103F02DFB8021D8
:1049E0002368192019404B42594103F025FB8021CF
:1049F0002368490019404B425941092003F01CFB30
:104A000080212368890019404B425941072003F057
:104A100013FB80212368890119404B42594106202C
:104A200003F00AFB80212368490319404B42594196
:104A30000A2003F001FB80212368C90319404B427F
:104A40005941032003F0F8FA802321685B041940E0
:104A50004B425941042003F0EFFA01211C205BE78F
:104A600004100020F80F002008100020EC0F002098
:104A7000F9D80000012010B54042FFF7BDFC10BD81
:104A800010B5034A0921034800F074FF10BDC04669
:104A9000E0DB000028DC00008023F0B502255B0588
:104AA0001A690A4C0A4BA1261D5103278025F600DE
:104AB000ED00BA43884202D300221A51F0BD5F597B
:104AC000002FFCD098518018F4E7C0460405000080
:104AD00000E0014010B5002806D1C020B0214002FE
:104AE0008902FFF7D9FF10BDB02080218002C902E2
:104AF000F7E7000043425841064B40421840B023BC
:104B00009B02C018036800201A0E532A01D11B0211
:104B1000180A704700C0FEFF30B501248025054B00
:104B2000054AED009C505C59002CFCD0016000212E
:104B3000995030BD00E00140040500004342584157
:104B4000074B40421840B0239B02C018A62310B563
:104B50000902DB05090A1943FFF7DEFF10BDC04655
:104B600000C0FEFFF0B5012480260D4B0D4DF60070
:104B70005C51002902DC00225A51F0BD57781478AC
:104B80003F022743947824042743D4780432240630
:104B90003C439F59002FFCD010C00139E9E7C046C3
:104BA00000E001400405000070B505004B680A00F4
:104BB0009C1C2100A400FFF7D5FF281970BD000040
:104BC000134B1B68002B0CD08022B023D2029B0217
:104BD00000280BD11A1D5B681B0E522B00D1100050
:104BE0007047B022C02392025B02F1E782420DD9E6
:104BF00003681B0E522B09D1436802339B00C01877
:104C0000824203D903681B0E522BE9D00020E7E74C
:104C10000C110020F0B50020B7B00024FFF7D0FF42
:104C2000270005002600002D2ED1284D2868FFF70B
:104C300061FF32003B0001900094254904A807F071
:104C400009FB04A801F0CCF8224B64201C682B68F7
:104C5000A0215A425341204A5B421340B0229202A3
:104C60009B18E41A6043490204F06CFEA022520231
:104C7000030000921949220004A807F0EBFA04A8E7
:104C800001F0AEF837B0F0BDFF226B6829689C4692
:104C90000233FF180B12013613409C4200DA1C004D
:104CA000FF200A14024003926246014001920091E3
:104CB000039A0B4904A807F0CDFA04A801F090F874
:104CC0002800FFF77DFF0500ADE7C0460C1100206E
:104CD00032DD00001011002000C0FEFFDCDC00000F
:104CE0001EDD000070B50020FFF704FF0400012066
:104CF000FFF700FF844200DA04000A4B1D686A4295
:104D0000554128001D60FFF7E5FEA0226B425202CC
:104D10001340054A28009B18044A611C1360FFF7E2
:104D20000DFF70BD0C110020048001001011002047
:104D3000F8B50020FFF7DEFE07000120FFF7DAFEDE
:104D40003E00204D0643204C0DD18021C020C902D9
:104D50004002FFF7A1FE01213000FFF7EFFE1B4BE1
:104D60002E6023601DE0874209DD0023B0212B6007
:104D7000164B8902236023680020012517E00123D8
:104D800080212B60124BC9022360F4E7120E522AD5
:104D900008D0002800D023600E4801F021F8FFF76A
:104DA000A1FFF8BD28005A68023292009B188B427E
:104DB00005D21A68561CE9D10028F2D0D1E721604B
:104DC000EFE7C0460C110020101100200480010004
:104DD00004C00200F7DC000070B50020FFF7F0FE11
:104DE000FF260500002801D1280070BD03681C14AF
:104DF0003440FFF7E5FEDA2CF4D10500F2E70000BD
:104E00008022F0B55200A1B00021674806F0DEFE16
:104E1000802200215200654806F0D8FE644BFF272F
:104E20001B681A00049353425A4110000592FFF781
:104E300051FE049C0020631E9C415E4B64421C405A
:104E40005D4BE418FFF7C8FF0600002E2DD1049833
:104E5000FFF750FE411C0598FFF770FE059A574D6D
:104E6000534B2C601A60FEF725FD514B64201B68E4
:104E7000A0215A4253414F4A5B421340B0222C6852
:104E800092029B18E41A6043490204F05BFDA022E1
:104E90005202030000924A49220007A807F0DAF9FB
:104EA00007A800F09DFF21B0F0BD32681314121264
:104EB0003A403B4003921A000A3A092A49D83A4B31
:104EC000039A995C002931D110223E4806F07EFEFB
:104ED00035002B6803991A123A40914209D11A14ED
:104EE0003A400B2A27D0132A2DD00A2A01D1354B5C
:104EF0001D602800FFF764FE051EEAD1314B1968DA
:104F000000290FD02000FFF74FFE04002D4B5B1946
:104F10005968002903D02000FFF746FE040004353D
:104F20000C2DF3D1204B0121039A99543000FFF747
:104F300047FE060089E73B40022BDADC214A9B0052
:104F4000D3185D60D5E7102200211E4806F03EFE12
:104F5000CFE71A00153A082AE8D8144A0399525C98
:104F6000002AE3D13500152B00D01500300003686E
:104F70001A143A40152A0FD01D2A00D10025FFF738
:104F80001FFE0028F3D1002D04D020002900FFF7D8
:104F90000BFE0400054BC6E7039A1B123B409A42E6
:104FA000EDD10500EBE7C0460C10002014110020E5
:104FB0000C11002000C0FEFF04C0020010110020F0
:104FC000C1DC00002C2F002010B5FFF719FF10BD29
:104FD000F0B585B0039203220333DC17294D14404A
:104FE000E4182B68284F5A42534180225B42D20278
:104FF000A4103B409B18A21C0291244E91000091EA
:105000000190316800980A18934215D2FFF7F8FE14
:105010002B685A42534180225B421F40D202BF1884
:105020003368009A9B189F4206D2194800F0D8FEB8
:105030000025280005B0F0BD029B356819066B46B7
:105040001A7BA423DB051343FF222F00090C19430D
:10505000019B12041B04134019432800FFF75CFD59
:105060000837281D21003760FFF756FD002C04D0BB
:105070000A9A21003800FFF775FD009B083BFF18D6
:105080003760D6E70C11002000C0FEFF1011002091
:105090009BDC000070B59AB0FFF74AFEFF221E4C61
:1050A000D2000021200006F091FDFF25FFF794FEBD
:1050B0000026002814D10200C300E3580130591E15
:1050C0008B41D218FF28F7D1144901A807F0C2F884
:1050D00001A800F085FE124800F082FE1AB070BDF3
:1050E00003681A142A400A2A0AD11A122A40FF2AEF
:1050F00003D0D200A1180B71A050FFF761FDD8E7D3
:10510000132AFAD11B122B40FF2BF6D0DB00E2183A
:105110001671E650F1E7C046A425002067DD0000C7
:105120007BDD00000021094B094A596001315160C3
:1051300059680029FCD000211961012393600222E3
:10514000044B8131FF315A501A607047FC10004007
:105150000010004000E100E00222064B0121DA6766
:105160000022054B5A61054A11615A69002AFCD098
:105170007047C04604E100E0FC1000400010004011
:1051800010B5044C2378002B01D0FFF7E5FF002079
:10519000207010BD15120020802301205B055B6E7E
:1051A0005B001843704700000120024B1B685B0046
:1051B00018437047981200200120024B1B685B00C7
:1051C00018437047240000200120024B1B685B003D
:1051D000184370479C12002070B504000D001600A3
:1051E000FEF724F9802301215B055A6E2670002604
:1051F00053006170E1706272010A5A0A6071A17114
:10520000A272010C5A0C000E5B0EA6702571E171A2
:105210002072E272237370BD10B5044C200007F0B9
:105220005FF801002000FEF7DBFD10BDA112002099
:105230000E4B10B51B680E4C5A1C0FD00D4C002B9A
:105240000CD00D4C012B09D00C4C022B06D0094C74
:10525000042B03D00A4C052B00D1074C200007F08B
:105260003FF801002000FEF7BBFD10BD2800002024
:105270000CDE0000FCD5000017DE000003D60000A5
:1052800011DE000070B5214C2278002A3DD1204B60
:1052900001215A608022D20511605A68002AFCD090
:1052A000002207201B4B1C4901255A500439585035
:1052B00008315A5019481A4958501A491A485A5030
:1052C0001A495A50A622D2009D50082218495A5015
:1052D0000431585002201749585017491748585060
:1052E000174804395850182016495850C1218900D0
:1052F0005A500539FF395858921802435A501249EA
:10530000124A9950FFF70EFF257070BD151200204C
:10531000FC000040001000400C050000746962753C
:105320001C05000024050000200004022C050000DC
:1053300014050000340500003C050000FFFF0000DC
:105340002110010054050000161200200405000081
:1053500070B50E4B06001B78002B01D1FFF792FFB2
:1053600000200B4D2C7884420ED00A4B2022197855
:105370000323091B1940084B4901C918300006F0E6
:1053800009FC0120013C2C7070BDC04615120020A4
:10539000A01200201412002016120020002370B565
:1053A00088B0984235DD0D6801262C0034409C42BF
:1053B0002FD12300042D2CD90F222B681A40230053
:1053C000092A26D16A683F2A23DD6846FFF7C0FF15
:1053D000230000281DD06B4619783300A14203DB5F
:1053E0006B461B5D5B003343A200AA180134936037
:1053F000202CF2D1092169444A780B7812021A4311
:105400008B781B041A43CB781B061343024A1360A4
:105410000423180008B070BD9C12002070B5454BE5
:105420008AB01B78002B01D1FFF72CFF02AC2000C3
:10543000FFF78EFF002802D100200AB070BD23784C
:105440000B2BF9D96378012BF6D1E378012BF3D13B
:1054500000231120384E394D33602B706844237976
:10546000374A4178136002780902114382781204A6
:105470001143C27812060A4332490A60002B0ED14A
:10548000152169444A780B7812021A438B781B0461
:105490001A43CB781B0613433360002318E0012B1B
:1054A0001AD1152169444A780B7812021A438B7875
:1054B0001B041A43CB781A211B06134333600E23B7
:1054C000627C6944934200DD130000229A422CD191
:1054D00000220420EA54B0E7022B03D1627B103390
:1054E0001621EEE7042B0DD11521082269446846E8
:1054F00006F050FB0098019902F0DAFD06F0FCF985
:105500003060CAE7052BC8D11521082269446846D6
:1055100006F040FB0098019902F0CAFD06F0ECF994
:105520003060627D0A231E21CBE7885CA8540132DB
:10553000CCE7C0461512002098120020A1120020CE
:10554000280000209C12002010B5134B04001B788B
:10555000002B01D1FFF796FEFFF7FEFD00200F4A5A
:105560000F49104B545058600130106058680028A3
:10557000FCD0002018610130906018690028FCD030
:10558000094B0A481B785B011B185350FFF7E4FDD9
:10559000FFF7C8FD10BDC0461512002000100040E6
:1055A00004050000FC100040141200201612002018
:1055B00010B588B000281DDD0A68012113000B40DA
:1055C00018D1042A16D90F2014682040092811D1B7
:1055D00050683F280EDD98001018806800240842AB
:1055E00001D04010C4B26846C4540133202BF2D11C
:1055F000FFF7AAFF002008B010BD000010B500287A
:1056000013DD0C68E30710D56410532C0DD8084B3C
:105610001B78002B01D1FFF735FEFFF79DFDA1237D
:10562000044ADB00D450FFF77DFD002010BDC046CA
:10563000151200200010004010B500280EDD0C6887
:10564000E3070BD56410FF2C08D8054B1B78002B03
:1056500001D1FFF717FE034A034BD450002010BDC1
:1056600015120020001000402405000013B500288A
:1056700014DD0C68E30711D5094B64100093094B46
:105680000193072C0AD8084B1B78002B01D1FFF798
:10569000F9FD6B46054A1957054BD150002016BD40
:1056A000E2ECF0F4F8FC00041512002000100040B9
:1056B0000C05000070B588B0002820DD01240868C2
:1056C00004401CD104281AD90F2302681340042B6C
:1056D00015D1FEF765F9060006F002FE0500122856
:1056E00000D912252A0002210D326846FFF774FD09
:1056F0006B465D73A54205DC6846FFF725FF002079
:1057000008B070BD2300325D6B449A730134F1E739
:10571000F0B50D008BB0012832DD086801220400CD
:1057200014402DD104282BD90F2301680B40042BE2
:1057300026D16B68134223D0FEF732F96E6807005A
:105740007310019306F0CCFD05000E2800D90E253C
:105750002A000121113202A8FFF73EFD6A461279A4
:1057600002AB5A7302AA73129373019B76141B0E39
:10577000D67313745574A54205DC02A8FFF7E4FE46
:1057800000200BB0F0BD3A5D02A963189A74013491
:10579000F1E730B589B0002814DD0C68E30711D5B6
:1057A000102268460021FFF717FD6B466A46651018
:1057B0005D73684663122D0E64149373D47315746D
:1057C000FFF7C2FE002009B030BD0000174B184A99
:1057D0005968002903D0002159600131916019698D
:1057E00000291FD0002018618023DB00D358114905
:1057F000012B18D1A923DB00D3585B420B600E4963
:105800000B78032B01D801330B7003200B490B7865
:10581000013303400B700A495B015B18094953507F
:105820000123936070470860FAE7C046FC1000400F
:105830000010004024000020A012002014120020BC
:10584000161200200405000010B5034A1021034879
:1058500000F090F810BDC0468CDD000083DD000034
:10586000044A05491368C85401339B059B0D136016
:105870007047C046D0160020D012002070B5114CE1
:10588000114A2368834202DC0023236016E0155C82
:10589000411C2E00FA3E012E05D899420FDA555CC4
:1058A000013D1F2D01D90800ECE70100151A565CD7
:1058B0006E5401318B42FADC181A206070BD1570ED
:1058C000FAE7C046DC1A0020DC16002010B5FDF710
:1058D000A3FD064B1A68824201D900221A601B6898
:1058E000C31A034898428041404210BDCC120020A8
:1058F000204E000010B5094C094A236812689342F3
:1059000000D110BD074AD05CFDF7CCFF0028F8D0CD
:10591000236801339B059B0D2360ECE7D416002020
:10592000D0160020D012002010B50400064B074A04
:105930001B6812689B1ADB439B059B0DA34200DB8F
:1059400010BDFFF7D7FFF1E7D0160020D4160020D6
:1059500070B5FFF741FAFF250400002801D12000AF
:1059600070BD03681B142B401D2B00D10400FFF7F2
:1059700027F9F2E770B5074E33680B2B08DC0C25CE
:105980005D43054C0133285164196160A2603360A6
:1059900070BDC046D81600203C2F002010B5FBF784
:1059A000A9FBFFF76DF8FBF7CDFBFDF70FFFFEF747
:1059B000C7FBFEF723FCFFF747FF01F035F801F0C6
:1059C0004DFA01F097FC10BD962210B5120100218E
:1059D000034806F0FBF80022024B1A6010BDC046D7
:1059E000441C0020D805002070B514007F22174BFE
:1059F000C000C0580D00836813401C2B01D000204C
:105A000070BDC368190011400429F8D101690A402A
:105A1000192AF4D11B0A01339B000C30C018FDF782
:105A2000BFFF037806000120002BE9D0300006F00C
:105A300057FC0023A042E2D1A34201DB0120DFE7B3
:105A4000F15CEA5C9142DAD10133F5E7A42500204C
:105A5000064B074A1B6812689B1ADB439B059B0D8C
:105A60000122834200DC002210007047D016002083
:105A7000D4160020F8B505000C0016001F1E0ED12C
:105A80000320FFF7E5FF002808D0FA20FFF7E8FE23
:105A9000E8B2FFF7E5FEE0B2FFF7E2FEF8BD501D09
:105AA000FFF7D6FF0028F9D0FB20FFF7D9FEE8B2B8
:105AB000FFF7D6FEE0B2FFF7D3FEF0B2FFF7D0FE5D
:105AC0003012C0B2FFF7CCFE3C00E31B9E42E5DD86
:105AD0002078FFF7C5FE0134F7E7000070B5002419
:105AE000F0250B4B1B68A34202DCFFF76DFF70BD76
:105AF0002B006343074A9B181A78002A05D059786F
:105B0000002311201A00FFF7B5FF0134E9E7C04672
:105B1000D8050020441C0020F8B507000024F0251B
:105B20002B0063430C4A01349E18B74211D03178E0
:105B300000290BD00133D15C002311201A00FFF79C
:105B400099FF2A000021300006F040F80A2CE7D126
:105B5000F8BD024B1C60F9E7441C0020D80500206A
:105B6000F0B5150001222F007A4C1740A544019092
:105B70000291002F11D005AB1A706A105A70120EE4
:105B80001A710522691299706D140299DD70FFF780
:105B900071FFCF239B009D44F0BD042D2AD90F2413
:105BA00028680440042C32D1022304AA280013716F
:105BB000FDF7F6FE050006F093FBC82302009B00EC
:105BC000984200DD1A007C1C97420DD1984206D9FC
:105BD000614804AB03226149C01805F0DBFF2200D5
:105BE00005AB02990198D2E72700611E695C05ACFC
:105BF000E155E8E7042D00D0A7E0032304AA043D03
:105C000013716B425D4105AB55710222E9E7092C26
:105C10007ED1042205AB1A706A6851100091694662
:105C2000521209789A70009A59701F2A01DD2022B9
:105C300000926A46127806ACDA70009BBB4202DC26
:105C400005ABE21ACDE70126BB00EB1898680640C9
:105C500006D1042837D90F210368194002290CD135
:105C6000012323704310637042121B0E4014A27074
:105C7000E070237105340137DFE7042921D10223C5
:105C80002370FDF78DFE039006F02AFBA31C0C2861
:105C900009D86070864201D19C19ECE7039A925DA5
:105CA0009A550136F6E70C226270039A925D9A5576
:105CB0000136092EF9D12E23E372237363730E3458
:105CC000D9E7012907D103230438237043425841FF
:105CD00060700234CFE7092909D104232370436897
:105CE0005A1062705B12A370E6700434C3E7032994
:105CF0000BD1052323700068020992B2430F920072
:105D00000B40D31A63701B12EDE726700134B2E723
:105D1000032C00D03DE7052205AB01091A7089B2BA
:105D2000420F890022408A1A11125A709970642A0F
:105D300000DD64220421DA70081F824201DC043293
:105D40004FE7685C58540131F6E7002D00D020E79A
:105D500053E7C046C4FCFFFF2203000078D20000D6
:105D600070B502000024F0210D4E08006043801938
:105D70004578954203D001340A2CF6D170BDF0224B
:105D8000002105F023FF074A1368013BA34200D11D
:105D90001460002329001A001120FFF76BFEEDE7C5
:105DA000441C0020D805002010B5B2B002236A467A
:105DB0000400137006F094FAC72800D9C720002306
:105DC000984207DC421C6B46FE211420FFF752FE6E
:105DD00032B010BD694601335A1EA25CCA54EFE7C7
:105DE00030B5B3B002236A460500137006F078FAA6
:105DF0000400C72800D9C72400239C420BDC2000E4
:105E00003230FFF791FD621C6B46FF211420FFF733
:105E100031FE33B030BD694601335A1EAA5CCA5404
:105E2000EBE70000F0B5BBB004900C00012803DCE8
:105E30001B20FBF721FB51E02A4B08680293C307A4
:105E400009D4042807D90F2302681340042B02D178
:105E5000FDF7A6FD0290234B60680393C30709D4A6
:105E6000042807D90F2302681340042B02D1FDF741
:105E700097FD039000271C4B1B680693069BBB42B3
:105E80000BDC039B194A0093C821029B08A806F06B
:105E9000AFF908A8FFF7A4FFCAE70C267E43144B0E
:105EA0000299F618306806F011FA051E05D17368DC
:105EB000B6680793079B9D4201DB0137DEE7306838
:105EC0000399059606F002FA0836002808D1210049
:105ED0000498059B083102385B6898473BB0F0BDD9
:105EE0000135E7E713D70000D8160020E8DE0000F0
:105EF0003C2F0020F7B5234B06001B68F0210093D0
:105F00000023009A9A4211DC0024F0231A00624315
:105F1000019201991C4A55182F78002F12D0013494
:105F20000A2CF3D11948FFF75BFF29E00A005A4316
:105F3000154882185078B04202D11278002A1FD139
:105F40000133DEE7F0223900280005F03FFE02238E
:105F50000D4A0199EB6053540D4AF1008A58009B99
:105F60006E70AE70AA602F616F61A34202DC054BB8
:105F700001341C60002331001A001020FFF77AFD65
:105F8000F7BDC046D8050020441C002031E30000C6
:105F9000A425002010B5FFF7A1FDFF24084AE30067
:105FA0005B429B18074AD35C043B012B03D8E043B8
:105FB000C0B2FFF79FFF013C002CEFD110BDC046DF
:105FC000FC070000A4250020F8B505000E00FF2402
:105FD0000C4AE3005B429B180B4AD35C062B01D0B2
:105FE000032B0BD1E743FFB2320029003800FFF743
:105FF000FBFC002802D03800FFF77CFF013C002C9E
:10600000E6D1F8BDFC070000A425002070B505000E
:10601000FF24084AE3005B429B18074AD35CAB426B
:1060200003D1E043C0B2FFF765FF013C002CF0D183
:1060300070BDC046FC070000A4250020F7B5FDF7A1
:10604000EBF9574B1A68824201D900221A601A688C
:106050005449821A8A420DD9FF2253491860D3004D
:106060005248CB1A1B181B78073B022B0CD9013A5C
:10607000002AF4D1F7BD0720FFF7C8FF4C4B27E0FB
:106080000820FFF7C3FF38E0FDF7D0F9071E00D165
:1060900001270020FDF7C8FA01900020FDF7D8FA8B
:1060A000019B0090434C444D002B12D02368002BE1
:1060B0006ED12B682760002B6ED0404B01261B78D9
:1060C000002BD8D10920FFF7A1FF394B1E703B4BA5
:1060D0001E70009B002B12D02B68002B0FD1236861
:1060E0002F60002B1ED0324B01261B78002BC7D10E
:1060F0000920FFF78BFF2E4B1E70304B1E7023685C
:10610000002B0FD02A4E3278002A0BD19F4200D2AA
:1061100027602368FB1A312B04D90720FFF776FF8D
:10612000012333702B68002B0FD0244E3278002AC5
:106130000BD1BB4200D92F602B68FF1A312F04D935
:106140000820FFF763FF012333702368002B0CD076
:10615000019B002B09D1164E3378002B02D107206A
:10616000FFF754FF0023236033702B68002B00D10E
:1061700080E7009B002B00D07CE7104C2378002B9D
:1061800002D10820FFF742FF00232B60237071E744
:10619000009A002AA0D1B5E7009B002B9FD1AEE763
:1061A000C81200200F270000A4250020FC070000D3
:1061B000BC120020B8120020C0120020C41200201F
:1061C00037B500240500FFF789FC01A80194FDF70D
:1061D00019FA21002000FEF7FFF8FEF7FFFAFDF79D
:1061E0004BFAFDF7CFFAFDF7E9FAFEF743FCFDF7AE
:1061F00041F9A54204D0FDF77FFB0248FFF7F0FD0F
:1062000037BDC04622E30000002310B501001A008C
:106210001120FFF72FFC10BD07B56B4619706946BA
:106220005A7013128B701314120ECB700A716B46D6
:10623000010005221320FFF71DFC07BD10B50A0061
:1062400001001220FFF78CFC10BD70B505000C009A
:10625000FDF7FAF8002809D020003230FFF764FB80
:106260002B00220000211B20FFF704FC70BD10B59D
:106270000C000300110014202200FFF7FBFB10BDEF
:10628000012370B5FF24084A41185B42884201D3BC
:10629000D84370BD06781D0A234073409B009B586D
:1062A00001306B40F2E7C04604DF000013B5040084
:1062B000FE2813D80A4BC200D05800280ED04368DD
:1062C00008309900FFF7DCFF01900920FFF72CFB55
:1062D00001AB042221001720FFF7CCFB13BDC04601
:1062E000A4250020F7B50190FFF732FB012504003B
:1062F000FF276D42002C01D12800FEBD2668331413
:106300003B40152B0DD121000198083105F0DEFF2F
:10631000002801D135123D402000FEF751FC040059
:10632000E8E71D2BF8D101256D42F5E7F0B5802790
:106330009FB0FFF7DFFAB54CB54D2068FF00391A62
:106340004019FDF795FA23680600C3182360002B57
:106350000ED11FB0F0BD2068391A2818FDF788FA51
:10636000236806001B182360FDF756F8A94B186038
:10637000002EF0DC2B78FA2B00D00EE12368022BE4
:1063800007DCFFF7A3FA0028E3D00120FFF776FA35
:10639000DFE76B78AC78981E182800D9F2E003F09C
:1063A0003DFA0D2024282B34F13E707A7E94CDDE08
:1063B000F1F1F1F1F1F1F1F1F1F1EC00FF2C0ED07E
:1063C0002000FFF7CDFC0022934BE100CA505B1880
:1063D0001A712100009213001320FEF7F9FD03202B
:1063E000D4E72000FFF786FDF9E72000FFF7B8FCAF
:1063F000F5E7FFF7CFFDF2E7FFF770FB0020FFF7AF
:10640000DFFE8648FFF7ECFCE9E7632CE7D8844B16
:10641000A200D25821001520FFF7A2FBDFE7FFF70B
:1064200097FAFF270400002CD9D025682B143B4095
:10643000152B04D02000FEF7C3FB0400F3E7200077
:10644000083005F04DFF06000530FFF76DFAFB2020
:10645000FFF706FA2D121D20FFF702FAE8B2FFF748
:10646000FFF9F0B2FFF7FCF93012C0B2FFF7F8F90C
:1064700025002B1B9E42DDDD287AFFF7F1F901355F
:10648000F7E700211D2000910B000A00FEF7A0FD98
:10649000FDF732FAA3E72000FFF708FF9FE7FCF7BC
:1064A000D5FF05AC5F4A642100905F4B200005F0EA
:1064B0009FFE02232000237005F012FF230002003C
:1064C00000211620FFF7D6FA89E70026524AF3008A
:1064D0009B181C68002C28D01B7903936368083430
:1064E0009F00B81D0293FFF71FFAFB20FFF7B8F9D2
:1064F00001207D1CFFF7B4F9F0B2FFF7B1F9E8B263
:106500002D12FFF7ADF9E8B2FFF7AAF90398FFF7EC
:10651000A7F9E719A7420CD8FFF7ECF90523029871
:10652000584301F069FBFFF7E5F90136FF2ECDD1A5
:1065300055E72078FFF794F90134EBE70024FFF7E3
:10654000CDFA2200210000942300DA20FEF740FD5E
:10655000FF222100D200304805F038FB98E7012CDB
:1065600002D1FEF757FB3AE7022C02D1FEF72CFDD1
:1065700035E70120FFF724FE31E7002321001A0050
:106580001A209FE71A00C83A052A00D927E70022F7
:1065900018001100FAF7E2FD21E7FB2B00D0F4E62A
:1065A0002268042A00DCECE62E79E8781F4B3602DC
:1065B00006439E4200DDE8E6331D9A4200DCE0E639
:1065C000EB5CFE2B00D0E0E66878AC78771E1B28E9
:1065D00000D17DE02ED8072863D0082838D00128C4
:1065E0002DD1FF2C10D02000FFF7BAFB6D79104A97
:1065F000B31E009221002A000A20FEF7E9FC064B98
:10660000E400E0501B191D71701DBFE6DC1A00206C
:10661000DC160020CC120020A425002004E300009A
:106620009C2D00201BE3000016E30000F603000091
:10663000E21600201D285DD04FD31E2871D0030024
:10664000C83B052BE0D8404A3900FAF787FDDBE765
:10665000632CD9D86A79022A13D0032A1BD0012AC5
:10666000D2D1E979AB79090219432B7AA4001B0432
:1066700019436B7A1B060B435B001343334AA35049
:10668000C2E7002FC0DDB11E3148FDF7A9FB2F4B3B
:10669000A400E050B8E7AB79A4005A1E93419B00D8
:1066A000ECE7632FB0DC05AD3A002749280005F080
:1066B00071FA00232800EB55FFF714FE0028A3DB36
:1066C000224B8000C25821001520FFF749FA9BE7B2
:1066D00039001D48FFF778FC96E7FF2C94D06A79C3
:1066E000022A91D81A490B2000912100B31EFEF70F
:1066F0006FFC89E7632F00DD6327002305A9BB42F8
:106700000ADBFB430022DB173B40CB181A70152035
:1067100000917B1C2100EAE7EA185279CA54013340
:10672000EDE7012C00D06FE7002F00DC6CE76B7900
:10673000002B03D01C00322B00DD322464235C4389
:10674000044B1C6060E7C046E11600209C2D002031
:10675000E2160020040000200122094B1A60094AB9
:106760001368002BFCD00322074B1B68D81710407E
:10677000C018012380100638400018437047C046F7
:1067800000C0004000C1004008C500400120704723
:1067900010B5064C200000F09BFE0549200000F0DB
:1067A000CBFE0122034B1A6010BDC046141B002013
:1067B000801A0600E01A00201FB500210E20FCF709
:1067C0004BFE01210F20FCF747FE01210D20FCF7B5
:1067D00043FE1B4B1B4A1B6812681B49D2B28B42FB
:1067E0000CD880239B04019301AB1A710199029A82
:1067F0000023164800F0E6FD05B000BD14498B42A9
:1068000002D88023DB04EEE712498B4202D88023B2
:106810001B05E8E710498B4202D880235B05E2E7BD
:106820000E498B4202D880239B05DCE70C498B4242
:1068300002D88023DB05D6E780231B06D3E7C046BA
:10684000300000202C00002048E80100F41A00204D
:1068500090D0030020A1070040420F0080841E005A
:1068600000093D0010B5002815DD01240B68234206
:1068700011D023410C4A13600C4AA04209D04B6846
:10688000234206D02341022B09D0032B09D0A34277
:1068900003D002231360002010BD0023FAE7032376
:1068A000F8E71460F7E7C046300000202C00002015
:1068B000F8B501250C682C4203D10D20FAF7DCFD58
:1068C000F8BD64102DD4FCF7C5FDA04229DB0021E2
:1068D0002000FCF7C1FDFA222900D200200001F0BF
:1068E000BDF900281DD0002500270726FA22012126
:1068F0009200200001F0B2F9002812D0282802DD11
:106900000123B3401F43013EF0D20E4EAF55013577
:10691000052DE9D1012206210920FDF7E3F9002820
:1069200001D10020CCE70B23012443600023F25C5B
:10693000990052004118224301338A60052BF6D199
:10694000BEE7C046E41A0020F0B50E0085B000286E
:106950002BDD01230A68134027D1042A25D91768A3
:106960000F221740032F20D1802101AA104D13714F
:106970008904029A28000393019100F023FD3668F0
:1069800033681C095B0F3B403700A4B2A400E41A33
:10699000BB1B9C4206DD3979280000F019FD013748
:1069A000F870F5E7280000F012FD002005B0F0BDFA
:1069B000F41A002010B504680D20E30703D5641015
:1069C000FF2C03D91720FAF757FD10BDFFF7F4FE8F
:1069D000E1B2044C200000F0FBFC200000F0F7FCCA
:1069E0000020F2E7F41A002070B5FFF7E5FE064D2F
:1069F0000021280000F0ECFC0400280000F0E7FC77
:106A000001206400204370BDF41A002010B500205E
:106A100001F0A2F9800810BD10B5FFF7F7FF4300A1
:106A20000120184310BD000010B5034A0D21034892
:106A3000FEF7A0FF10BDC04648E30000B0E3000031
:106A40000D4B70B51B6804000E001500002B01D122
:106A5000FFF79EFEE1B2094C200000F004FEF1B207
:106A6000200000F001FDE9B2200000F0FDFC200054
:106A700000F064FE70BDC046E01A0020141B002028
:106A800010B501240368234205D04168214202D099
:106A90008268224203D10D20FAF7EEFC10BD581097
:106AA000802801D91520F7E74910FF2901D91620C0
:106AB000F2E75210FF2A01D91720EDE7FFF7C0FFD8
:106AC0000020EBE710B5002807DD0B68DB0704D5D5
:106AD000302223211920FFF7B3FF002010BD000052
:106AE000F7B501221400904222DD0D682A421FD022
:106AF0001D4B15411B684C68002B01D1FFF748FE68
:106B0000E9B201272500194E3D40300000F0ABFDF1
:106B1000002D0FD03C413000E1B200F0A5FC300068
:106B200000F00CFE0024A04202D02320FAF7A4FCBF
:106B30002000FEBD042CF2D90F2322681340092B3C
:106B4000EDD163685B100193019BAB42E7DDAB00C5
:106B5000E3189968394204D04910C9B2300000F0F6
:106B600083FC0135F0E7C046E01A0020141B00202A
:106B7000154B70B51B6805000E00002B01D1FFF707
:106B800007FE124CEDB22900200000F06CFDF1B2BE
:106B9000200000F069FC0021200000F06FFD0028BB
:106BA00001D0404270BD72B601222900200000F0E1
:106BB00055FD62B6200000F048FC0028F2D020000D
:106BC00000F048FCEEE7C046E01A0020141B00204D
:106BD00010B501240368234202D04168214203D149
:106BE0000D20FAF749FC10BD5810802801D9152056
:106BF000F7E74910FF2901D91620F2E7FFF7B8FFA0
:106C000040002043EFE7000010B50D211D20FFF7E5
:106C1000AFFF164C5A2809D101222A2122703D3893
:106C2000FFF70EFF0122124B1A6010BD0F21192031
:106C3000FFF79EFF332805D102238F2223702021E6
:106C40001A38EDE70D211E20FFF792FFC7280AD161
:106C5000032300222A21A9382370FFF7F1FE1B220B
:106C60002A211E20DCE700232370DBE7340000200C
:106C7000EC1A0020204B10B51B680400002B01D13A
:106C8000FFF7C2FF1D4B1B785BB2022B0AD0032B10
:106C900029D0012B2CD121001D200124FFF768FFF2
:106CA000644205E0012C13D129211920FFF760FF70
:106CB0007F2801DD0138FF3803007F3301DA7F20B0
:106CC0004042C8237F21584302F03CFE604310BD80
:106CD000032C0BD12B211920FFF74AFF043CE7E7D7
:106CE0002D211920D9E721001E20D6E7052CF7D049
:106CF000012400206442E4E7EC1A00203400002064
:106D000010B50120FFF7B6FF43000120184310BD66
:106D100010B50320FFF7AEFF43000120184310BD5C
:106D200010B50520FFF7A6FF43000120184310BD52
:106D3000144B70B51B68002B02D10120FFF79AFF9E
:106D4000114B1B785BB2013301D1FFF75DFF0120CE
:106D5000FFF790FF04000320FFF78CFF05000520DC
:106D6000FFF788FF6D43644340436419201804F023
:106D7000F9FD01F0CDFA04F0BFFD430001201843F6
:106D800070BDC046EC1A002034000020F8B5012385
:106D90001C0098422BDD0F683B4228D04E6835001E
:106DA0001D4024D1042E22D90F2231680A40092A1D
:106DB0001DD173685C10202C00DD2024144B1B684F
:106DC000002B01D1FFF7E4FC72B67F10F9B2114F2E
:106DD0002200380000F042FC62B6A54214DA380006
:106DE00000F033FB002804D101246D002C43200067
:106DF000F8BD380000F02EFB0122AB004000F31874
:106E000010439860AD18E8E764000125EEE7C0463E
:106E1000E01A0020141B002000207047012070475A
:106E20000020704700207047002070470120704705
:106E300000207047002070470020704700207047F6
:106E400000207047002070470020704700207047E6
:106E500000207047704770477047000010B5034A24
:106E60000F210348FEF786FD10BDC0463CE400003C
:106E7000B4E400000378013B1F2B00D970470130B8
:106E8000F8E710B5FFF7F6FF0378002B0BD00130C1
:106E9000222B11D10378002B03D0421C222B03D1CB
:106EA0001000FFF7E7FF10BD5C2B03D14378002BE8
:106EB00000D0821C1000EDE73A2BF2D02C2BF0D042
:106EC0007B2B0BD1FFF7D6FF0378002BE9D07D2B6E
:106ED00001D10130E5E7FFF7D4FFF5E720225B2B76
:106EE00014D1FFF7C7FF0378002BDAD05D2BF0D069
:106EF000FFF7C7FFF7E7202BD3DD2C2BD3D01900EA
:106F000091435D29CFD0222BCDD001300378002BC7
:106F1000F1D1C6E7002210B5904216D0FFF7AAFFC4
:106F200003780422222B10D0023A7B2B0DD0013A99
:106F30005B2B0AD0190030390232092905D92D2BD3
:106F400005D14178303909290AD8100010BD052231
:106F5000742BFAD00132662BF7D001326E2BF4D0AD
:106F6000581E83415A42F0E770B5FFF783FF03785C
:106F700001222D2B01D18018023A00230A2502E0BC
:106F80006B430130CB1801783039CCB2092CF7D9DA
:106F90005A43100070BDF8B50C001500FFF76AFFEA
:106FA0000378222B02D000232370F8BD0D236A1E24
:106FB000210008250C260A279C4601300378222B45
:106FC00002D100230B70F0E7002BFAD0441C5C2B9D
:106FD0000BD14378841C622B0ED0662B0ED06E2B07
:106FE0000ED0722B0ED0742B0ED0002AE9DD0B7060
:106FF000013A01312000E1E72B00F6E73300F4E726
:107000003B00F2E76346F0E70923EEE710B5040022
:10701000FFF737FFA04203D90378013B1F2B00D9AC
:1070200010BD0138F6E710B5002815D00378002B05
:1070300013D0FFF71FFF2021037802008B430020AD
:107040005D2B09D01000FFF71CFF03782C3B5A4240
:107050005341C018FFF70EFF10BD1800FCE70300F6
:10706000002070B50C0081420EDD1A785B2A0BD12E
:10707000581CFFF7FFFE0125AC4205D0FFF7D3FFF8
:10708000002801D00135F7E770BD70B50C00150080
:10709000002901D000230B70002820D00378002B9A
:1070A0001ED0FFF7E7FE037806002C2B03D101303A
:1070B000FFF7E0FE0600337800207D2B0FD08442DE
:1070C00004D02A0021003000FFF765FF3000FFF7F1
:1070D000D8FE03783A2B02D10130FFF7CBFE70BD0A
:1070E0001800FCE7F0B50D0004009DB02E78002ECE
:1070F00035D02E21280005F0DBF8071E14D0431BE5
:107100000193303E092E14D82800FFF72DFF01000F
:107110002000FFF7A4FF0400002C20D0002F1ED079
:10712000019B0133ED18E1E7280005F0D9F8019043
:10713000E7E723787B2B11D1601C642203A9FFF7BA
:10714000A4FF041E0BD0019A290003A805F0CFF874
:107150000028E1D02000FFF794FEEEE70024200095
:107160001DB0F0BD70B5050000200C0081421DDD92
:107170002800FFF7CFFE0300681C012B14D000206D
:10718000022B13D10022681C1100FFF77EFF012C97
:107190000CD0FFF748FF00221100FFF776FF013CFB
:1071A000F5E7FFF740FF013C012CFAD170BDF8B5BF
:1071B000050000200C0016001F0081420DDD280094
:1071C000FFF7A8FE03000020022B06D1681C3A003E
:1071D0003100FFF75AFF012C00D1F8BDFFF723FF64
:1071E0003A003100FFF751FF013CF4E710B50024ED
:1071F000A04218D0FFF73EFE03787B2B0AD1013066
:1072000000221100FFF741FF00280CD0FFF739FEE4
:107210000134F5E75B2B06D10130FFF704FF0028AE
:1072200001D00134F9E7200010BDF8B5002816DDC3
:107230000D68EB0713D56D10013D0124FDF7CCFD62
:107240000026FF27644200280CD1002E21D03000F8
:1072500005F046F801003000FCF7C2FDF8BD01253D
:107260006D42EAE703681A143A40152A0BD11B1243
:107270003B409C4200DA1C009D4201D106000836CA
:10728000FDF79EFCDFE71D2AFAD1012400266442A7
:10729000F6E70120013464002043DFE710B50868F9
:1072A0000C00FCF77DFBFFF71DF8002803DB62688C
:1072B000024B8000C250002010BDC0469C2D002013
:1072C00010B50868FCF76CFBFFF70CF801230028E9
:1072D00002DB024B8000C358180010BD9C2D00201B
:1072E00010B50868FCF75CFBFEF7FCFFC043C00F5D
:1072F000800010BD10B5034A04210348FEF73AFB95
:1073000010BDC04650E500004AE5000010B5FCF78E
:1073100069FAFCF717FBFEF741FB0448FEF760FD36
:10732000FDF7B8FEFEF736FE10BDC0469FE5000033
:1073300010B5FBF7E5FE10BD70B5002504AC247850
:107340000573A94205D10A4B0A4A25210A4804F0CF
:10735000B3FB01600949920052589B0002715B58CF
:10736000A40083716358856043710223C37170BDAB
:10737000B7E5000016E60000C5E5000074E6000071
:107380001FB50191A02100240068C900D2B2445069
:10739000012A10D0A24209D0032A0AD0074A8350FA
:1073A000074B019AC250012343501FBD02221343D1
:1073B000F4E70422FBE70622F9E7C0465405000083
:1073C000240500001FB5FFF7DBFF05B000BD7047C7
:1073D0000368074A99501A00FC32D1680029FCD092
:1073E000A321C90058580023C0B2D3607047C046DB
:1073F0001C05000007B58022074BD2051A60002249
:107400009A6002321A710F230C3200930349023B37
:107410000348FFF791FF07BD081B00200030004024
:10742000F41A0020F8B505000E0017000024BC4235
:1074300008D02B68315D1B6828009847002801D0D0
:107440000134F4E72000F8BD704710B51C3000F09F
:10745000AFF910BD10B51C3000F09CF910BD10B58F
:107460001C3000F0ABF910BD70B5437E0D00002B51
:1074700001D1002070BD6430040000F0A8F900289C
:10748000F7D12000290000F076F90120F2E7000092
:10749000F7B50193FA23002504009B0083600B4B92
:1074A0004560083303601C300F00160000F058F9E7
:1074B0002000643000F054F96B461B792761667533
:1074C0006576A5762000A375FEBDC04654E6000093
:1074D000012330B5A024C375837D13499B005A58FE
:1074E000437DC132114DFF32E40592009B005B5891
:1074F0001551CC22C133FF339B001D5104690C4B45
:107500005204E25005220469243BE250837D046961
:107510009B005A58A123DB00E250437D02699B0087
:107520005958044BD15030BD74E600000C060000E1
:10753000240500000C050000A022002310B50469FA
:10754000D200A3500A4CA1420FD90A4C8C425B4195
:1075500009495B420B40CD21C9045B180469074906
:10756000635005210369995010BDCC235B04F5E7F6
:10757000A086010090D00300000098FD24050000C3
:10758000F7B5040000200D000193824265D016007B
:10759000402A00D9402627001C37380000F0F6F8B2
:1075A000B1232269DB00D55080220123216992009A
:1075B0008B50A27E002A03D12269136222691360D4
:1075C0000025731EAB4207D1019B002B04D0802203
:1075D0000221236992009950012223691A622369CA
:1075E000FC33DA68002A02D19A6A002AF9D09A6A32
:1075F000002A0BD1DA60A3232269DB00D1583800BE
:10760000C9B2013500F0B7F8B542DAD3019B22695F
:10761000002B0FD11300FC339B6A002B0AD10133DE
:10762000A376D3612369FC33DA6C002AFCD00022F4
:10763000DA640AE000230121A37651611A0023696C
:10764000FC3399680029FCD09A602369FC339A6A5C
:10765000002A01D000229A62E8B2FEBD10B50123D3
:10766000FFF78EFF10BD0300AC3310B50400197096
:10767000643000F08BF80123637610BD0023020014
:1076800070B5AC3243760D001178B1220400006968
:10769000D20081508022216992008B5022690133EF
:1076A00013622269936026006436300000F080F88F
:1076B000002812D0300000F06DF81E4B2269D05027
:1076C0002369FC331A6A002A02D19A6A002AF9D087
:1076D0009A6A002A01D11A62E5E723690122002D86
:1076E0000DD11900FC31896A002908D1DA612369BA
:1076F000FC33DA6C002AFCD00022DA6407E05A611D
:107700002369FC339A68002AFCD000229A6000208A
:107710002369FC339A6A82420BD098622169064A37
:107720008B588B501800022B03D0181F431E984112
:10773000033070BD1C050000C404000010B5012119
:10774000FFF79CFF10BD000010B51323142202495F
:107750000248FFF79DFE10BD00400040141B0020B2
:1077600010B540220021040004F030FA002320006C
:107770002364636410BD10B53F24026C531C234086
:10778000446C9C4201D08154036410BD0023036407
:1077900043647047436C026C934206D03F21C25C45
:1077A00001330B4043641000704701204042FBE767
:1077B000036C406C181A00D540307047436C026C63
:1077C000934201D0C05C704701204042FBE73F225A
:1077D000036C406C01331340181A43425841C0B245
:1077E0007047000003210A4802680A430260094802
:1077F00002680A4302600849084A094B9B1A03DDE4
:10780000043BC858D050FBDC00F012F8F8F77CFCC1
:107810002405004054050040C0EB0000000000209B
:1078200070020020FEE7FEE7FEE7FEE7FEE7FEE768
:10783000014B024A1A607047380000200024F4000F
:107840000120704710B503681322DB69984710BD0B
:1078500070470000054B0269D1500369FC331A6A76
:10786000002AFCD0002201201A6270471C0500008B
:10787000030010B55C331A781F231A401E3B190011
:107880009140114AD167C222042104699200A1509B
:10789000026953600269D360A02300220169DB0002
:1078A000CA5001230169094A5B428B500169084AA9
:1078B0008B5001690C3A8B50016908328B5014309F
:1078C000FFF764FF10BDC04604E100E00C050000B6
:1078D0001405000010B51430FFF76AFF10BD10B595
:1078E0001430FFF76BFF10BD10B51430FFF752FFD7
:1078F00010BD0000030070B55E331A780469724B46
:10790000E25003005D331A780469704BE2500300C3
:1079100061331C7802696E4B012C00D09EE005009B
:107920005F352E78A225ED005651020060321578A1
:10793000A1220669D200B5500269D4509623DB001B
:10794000994200D88CE096231B01994200D88AE026
:1079500096235B01994200D888E096239B019942C7
:1079600000D885E0E1239B01994200D882E096236C
:10797000DB01994200D880E0E123DB01994200D885
:107980007DE096231B02994200D87AE0E1231B0296
:10799000994200D877E096235B02994200D874E0C0
:1079A000E1235B02994200D871E0E1239B029942F6
:1079B00000D86EE0474B994200D86CE0E123DB022F
:1079C000994200D86AE0E122002312038A425B4117
:1079D000414A5B421340802252059B1801693F4A8D
:1079E0008B50A02304220169DB00CA5000210369E7
:1079F000FC33D9600369FC331962012301690B6010
:107A000001698B60C1210469890062501F215C30CB
:107A100002780A4093406231314AFF3153500021CD
:107A2000415600293CDA0F230B40083B2D4C9B08A4
:107A30009B001B1903242140A140FC348C40DD69CC
:107A4000A5432C00C0258D4029002143D9611F2367
:107A5000017819401E3B8B40136070BD00246CE719
:107A60009E23DB02BAE79D231B03B7E71E4BB5E756
:107A70001E4BB3E7EC239B03B0E71D4BAEE71D4B5A
:107A8000ACE71D4BAAE71D4BA8E71D4BA6E71D4B16
:107A9000A4E71D4BA2E78023DB049FE71B4B9DE778
:107AA0008C080F4BA400E41803230B40FF21C025D2
:107AB000DB009940AD0066598E433100C0269E40E0
:107AC00033000B436351C2E70C05000014050000AE
:107AD0006C05000090D0030000D0BEFE240500001D
:107AE00000E100E000ED00E000B0130000502700CE
:107AF00000A04E0000F0750000509D0000F0EB006B
:107B000000903A0100E0D70100B0AF0300705F07BA
:107B1000F7B5009308AB1B7800250193FA23040006
:107B20009B0083600E4B45600833036014300F00E8
:107B30001600FFF715FE23005C3327611E70009BC3
:107B4000084A9B00995823005D331970019B20005F
:107B50009B009A5823005E33DD701A70FEBDC0464C
:107B6000F8E6000074E60000036910B51A00FC3264
:107B7000D2680400002A0AD0A322D20099581430F7
:107B8000C9B2FFF7F8FD00222369FC33DA6010BDAB
:107B900010B50248FFF7E8FF10BDC046CC1B00201F
:107BA000162307B5022200930249013B0248FFF762
:107BB000AFFF07BD00200040CC1B002010B50028FF
:107BC00001D004F0BFFA10BD0849094A094B10B5AD
:107BD0001B688858FA22190A1B06184392000023D2
:107BE00001F0E8FF4904C00B084310BD001001403C
:107BF00004050000301C002070B5041E09D0FFF7FA
:107C0000E3FF050000F014F8FFF7DEFF401BA04281
:107C1000F8D370BD0022044B9A60044A1368013304
:107C2000DBB213607047C046FC100140301C0020DE
:107C30007047704710B500F05FF8FFF7FAFF0120BA
:107C4000FFF7DAFFFFF762FBFFF772FB024B002B37
:107C5000FAD000E000BFF7E700000000F8B54C1EC6
:107C6000A1410125104B114F8000C3584C42386888
:107C70000F499D40160001F0DBFD0A21704301F021
:107C8000D7FD2C400300220029000A4800F016F816
:107C9000FA21094C89004443386801F0C9FD01000C
:107CA000200001F0C5FDF8BD74E60000380000209A
:107CB00040420F00100500501027000030B5046846
:107CC0000C40944206D1013B002BF8D112E0013B5D
:107CD000002B0FD004680C409442F8D100240568B2
:107CE0000D40954204D101349C42F8D1002002E0BD
:107CF000201C00E0181C30BDC420114B80001A5815
:107D000010491140C02212020A431A50C021802299
:107D1000490092025A501A608023A3220021DB05F9
:107D2000D20099500122F9309A60074BFF30195068
:107D3000C120023180001950403019501A6070473C
:107D400000E100E0FF00FFFF00100140014B186060
:107D50007047C04684000020F7B5002320285AD879
:107D6000384B8000C258042A5BD007D8022A54D06E
:107D700055D80423012A09D000234CE0062A54D008
:107D800051D31A2A53D002231B2AF5D12E4A116847
:107D900008294ED909294FD00A240226A0200125FE
:107DA0002A4AC00015502A482A4D07681C20BF00E7
:107DB00007402948019700685759009027481B023F
:107DC00007401F43C02300989B020340FF205751E8
:107DD0005759000207401F43019B1F43009B580156
:107DE0006023184007433E43565101251C4B156044
:107DF00058680028FCD000205860A1230125DB0032
:107E0000D3585560A025ED0050511BB2A14202D0BD
:107E100015D2611ACB401800FEBD0823B6E7102327
:107E2000B4E72023B2E74023B0E78023AEE7012385
:107E3000ACE708240026B1E70C000126AEE7091BD9
:107E40008B40E8E774E600008000002000700040EE
:107E50003C0000200405000040000020FF00FFFF60
:107E6000FC700040F0B520285BD8364B8000C2582B
:107E7000354B1E68002E30D1C227344BBF00D85975
:107E8000334C03250440C02000022043D851C024B5
:107E900080206400800018512E4F18602E4B803CCB
:107EA000D859FF3CA043D8510437D859A8432043A0
:107EB000D8510837D8590C35A84384460720654661
:107EC0002843D851A820C0001E50C1208026800021
:107ED00076021E501C601C4B1C60142500202B00D9
:107EE0001E4C2E0046433659771C1BD14343E250AB
:107EF000A0230325C132FF329200DB05D550184B79
:107F00001A68082A14D114234343E3189A681248C4
:107F10005132FF32920059601150DA68C1239B0040
:107F2000C250F0BD9642E1D001300328D9D1F8E724
:107F3000082A02D9083AD140E5E708239A1A914065
:107F4000E1E7C04674E60000341C002000E100E0D8
:107F5000FF00FFFF040500000090004044000020E7
:107F6000840000202149F0B54A6C2148002A14D031
:107F7000A025A12600230124ED05F600C258571CB8
:107F800006D0C7187F68002F02D027009740AF5156
:107F900014333C2BF2D100234B64A0230121DB05D9
:107FA00000260F009C4614234B43C3181A1F126867
:107FB000104C0E4D920014195219526C002A10D018
:107FC0001A00143A1268551C09D0103B1B68FF2B8D
:107FD00005D03B00934065461A00074BEA50FC343D
:107FE000666401310429DED1F0BDC046FC9000403A
:107FF00044000020009000400C05000000B520283F
:1080000010D80C4A8000835803290BD8A0220800FE
:10801000C133FF33D2059B0001F000FC02090507C4
:108020000021D15000BD0C21FBE70421F9E7032119
:10803000F7E7C04674E6000020280AD8074B800006
:10804000C25801239340A022D205002902D104493D
:1080500053507047A121C900FAE7C04674E60000FA
:108060000C05000003000020202B0AD8A021A2222A
:10807000C905D2008858034A9B009B58D840012369
:108080001840704774E60000F7B506000D000C00BC
:108090008B180193019B671B9C4207D033682178A2
:1080A0001B683000984701340028F3D13800FEBD2A
:1080B000F0B5C64600B5CB0F9846404A4B005B0D65
:1080C0009A1882B00D000400132A2FDC002A49DB25
:1080D0003B4F17413E000E40064323D07F08390036
:1080E00029400C430AD03749BD438C4663445C4267
:1080F0005C418023DB021341E4071D434146CE006F
:1081000031492B008E19220034687568200029003F
:1081100001F0F6FE009001910098019922002B00D9
:1081200003F086F802B004BC9046F0BD332A08DDA7
:108130008023DB009A42F5D102000B0001F0E0FE43
:10814000F0E7224A9446012263445242DA40024256
:10815000E8D052080242D1D094438022D2051A417D
:108160001443CBE74B005B080343DBD00B031B0B33
:108170001C436342234380244D0C24031B0B2340E8
:108180006D042B4319004346DA000F4B9B181C6803
:108190005D6802000B002000290001F0B1FE009094
:1081A00001910098019922002B0003F041F842460A
:1081B0004B005B08D60733431900B3E701FCFFFF10
:1081C000FFFF0F00EEFBFFFF28E70000EDFBFFFFC6
:1081D000F8B5274A4B005B0D9A180C000700132ACC
:1081E00010DC002A36DB234B13410B423AD08024AB
:1081F00024031441002064189C430600250030002D
:108200002900F8BD332A0EDD80230600DB000D00B7
:108210009A42F4D102000B003800210001F070FEF8
:1082200006000D00EBE7144D0600AC460125634443
:108230006D42DD40AC4663460D000342DFD0332380
:108240009A1A323B93401818874200D94C1C634657
:108250009843D2E7C90FCC070020531CCDD1074B60
:108260001C43CAE706000D000028C0D1C7E7C0467E
:1082700001FCFFFFFFFF0F00EDFBFFFF0000F03FE1
:1082800030B5214A4B0087B05B0893421EDD1F4A80
:10829000934205DD02000B0002F0CAFF07B030BDBB
:1082A00002AA00F095F803231840049A059B0128C0
:1082B00013D002281DD0002814D00298039900F092
:1082C0006FFB80231B069C466144E7E700230022E6
:1082D0000093002301F0DEF8E0E70298039900F034
:1082E0005FFBDBE7012402980399009401F0D2F8C8
:1082F000D4E7012402980399009401F0CBF880237D
:108300001B069C466144C9E7FB21E93FFFFFEF7F65
:10831000F0B54746CE4680B58DB004000D0000F0A4
:1083200067FA294B06001B780F005BB298460133B1
:1083300010D022002B002000290003F0C1FA814652
:10834000002807D1002200232000290001F00AFCA8
:10835000002806D1300039000DB00CBC904699467B
:10836000F0BD01230293194B0694079503934B46E6
:108370000A93434604940595002B15D00023002250
:108380001900100002F0D8F8434608900991022B1A
:108390000ED103F0AFFB212303600A9B0193002B56
:1083A0000CD1089E099FD5E7002300240893099467
:1083B00002A801F0C1F90028EFD1EAE703F09AFB27
:1083C0000A9B01930360ECE78800002038E7000077
:1083D000F0B54E464546DE465746E0B5E14B4C000B
:1083E0008FB09046894664089C4200DC87E0DE4BF3
:1083F0009C4222DCDD4A002900DC92E0DC4B02F0EA
:1084000017FFDB4B06000F009C4200D17EE1D94AEA
:10841000D94B02F00DFF02000B00414630000A600C
:108420004B60390002F004FFD34BD24A02F000FF48
:10843000434601259860D9606BE0D04B9C4200DC3C
:108440008FE0CF4B9C4200DD55E1CE4A231592468A
:108450009A4451460905631A19001D00040003F0EF
:108460004BFA03F07FFA02000B002000290008926B
:10847000099302F0DDFE0022C34B02F067FC0F00FF
:10848000060003F039FA03F06DFA04000D00020053
:108490000B00300039000A940B9502F0C9FE00224F
:1084A000B94B02F053FC002200230C900D9101F017
:1084B00053FB002800D192E1002300222000290074
:1084C00001F04AFB434243410133B04A4146019225
:1084D000022208A80092524600F07CFB4B460500A1
:1084E000002B16DA802243461206944642465B6809
:1084F000454263445360D3686344D36009E00B0092
:10850000020041460A604B600022002300258A6079
:10851000CB6028000FB03CBC90469946A246AB46C3
:10852000F0BD934B01F0ECFC914B06000F009C4218
:1085300000D13DE18F4A904B01F0E2FC02000B00BC
:10854000414630000A604B60390002F071FE894AF2
:10855000894B01F0D5FC012543466D429860D960F6
:10856000D7E701F049F88A4A8A4B06000F0002F06B
:10857000EDFB0022884B01F0C3FC03F0BDF90500C0
:1085800003F0F0F9794A7A4B0490059102F0DEFB92
:1085900002000B003000390002F04AFE754A060066
:1085A0000F0004980599744B02F0D0FB02900391E0
:1085B0001F2D00DCC7E0029A039B3000390002F057
:1085C00037FE83468A4653465B0024155B0DE31A4B
:1085D000102B6CDD04980599D322674B520502F0ED
:1085E000B5FB02000B00300039000292039302F049
:1085F0001FFE0A00010013000691079202003900D5
:10860000300002F015FE029A039B02F011FE0600F4
:108610000F0004980599614A614B02F097FB320004
:108620003B0002F005FE069E079F0B00020039008A
:1086300030000292039302F0FBFD4B005B0D83467A
:108640008A46E41A312C32DD04980599B822544B3D
:10865000920502F07BFB03000C00020002930394DE
:108660000B000698079902F0E3FD02000B000600DC
:108670000F000698079902F0DBFD029A039B02F0B7
:10868000D7FD484A0290039104980599464B02F0A1
:108690005DFB029A039B02F0CBFD02000B00300051
:1086A00039000292039302F0C3FD83468A465A467C
:1086B0005346414630000A604B60390002F0B8FD75
:1086C000029A039B02F0B4FD44460B000200A26034
:1086D000E3604B46002B00DB1BE75B4623608023F7
:1086E0001B065344636080231B069C466144A060C4
:1086F000E1606D420DE70B00020002F099FD434678
:1087000000259860D9601860596002E7D3221A4B9F
:10871000520502F08DFD214A214B0D00040002F0AC
:1087200087FD02000B00414620000A604B602900D3
:1087300002F07EFD1A4B194A02F07AFD43460125EC
:108740009860D960E5E602000B003000390002F0C5
:108750006FFD6B1E154A9B009B5883468A46A342B9
:10876000A5D130E7FB21E93F7BD90240000040540E
:10877000FB21F93F3163621A61B4D03DFB213941DD
:10878000FFFFEF7FEAFBFFFF00007041C0E7000042
:1087900083C8C96D305FE43F0000E03F7370032E73
:1087A0008A19A33BC14920259A837B3940E7000001
:1087B000D3220C4B520501F0A3FB0B4A0B4B0400D8
:1087C0000D0001F09DFB02000B00414620000A60F5
:1087D0004B60290002F02CFD034A044BB9E6032349
:1087E00073E6C04661B4D03D7370032E8A19A33B73
:1087F000F8B54746CE46674B80B50A000F00190012
:1088000005003940994200D19BE004000100002F8F
:1088100069DD3F1500D1B4E05F4B12039C46802315
:10882000120B5B0313435B00CA0F67449B184A009B
:10883000F80703D5D20F5B009B188A0079108C468D
:10884000002180201624894680030D189D4202DCF9
:1088500029185B1B8144D50F5B00013C5B1952005A
:108860004008002CF1D100208046802020250027E0
:10887000000609E08B425CD0D40F5B00013DE31899
:1088800052004008002D16D0C4198B42F2DD271883
:108890000E00002C49DB5B1AA242894149425B1A57
:1088A000121BD40F5B00013D80443100E3185200DD
:1088B0004008002DE8D113434ED143465B083749A9
:1088C0004A468846494652104244C90702D580218B
:1088D00009060B4361460F05BD18180029000CBCA2
:1088E00090469946F8BD7B005B0803433900002B96
:1088F000F5D0002F3CD1E30A153A6405002BFAD0DD
:108900008020400303423FD1002700E00F005B00BE
:10891000791C0342FAD0250020208D40401A2900FE
:10892000D71B2200C2401A4376E7FE43F60F8E198A
:10893000B1E79442A0D82718002CF6DB1E000023D4
:10894000AEE702003B002800390002F0FFF92A00E0
:108950003B0001F0D5FAC2E74346013303D043465A
:1089600001335B08ABE7012398460023C144A6E727
:108970003B00020002F05CFC02000B0001F0DCFD99
:10898000ADE713000022BBE70127210020207F4232
:10899000C6E7C0460000F07F01FCFFFF0000E03F9B
:1089A000F0B54746CE4680B587B000920193754B2F
:1089B0004F00814688467F089F4263DC02F09CFF9F
:1089C000002800D1D4E04A4643464846414602F0DA
:1089D000BDF904000D006C4A6C4B02F0B7F96C4A0B
:1089E0006C4B01F08DFA22002B0002F0AFF96A4ABD
:1089F0006A4B02F01DFC22002B0002F0A7F9684A26
:108A0000684B01F07DFA22002B0002F09FF9664AC4
:108A1000664B02F00DFC22002B0002F097F9644A2D
:108A2000644B01F06DFA22002B0002F08FF90290E6
:108A300003910022604B2000290002F087F9029A7E
:108A4000039B06000F002000290002F07FF9009A26
:108A5000019B04000D004846414602F077F90200F0
:108A60000B002000290002F0E3FB02000B003000A5
:108A7000390002F0DDFB02000B0000204F4902F03C
:108A8000D7FB70E002000B0002F060F904000D005B
:108A90003D4A3E4B02F05AF93D4A3E4B01F030FA56
:108AA00022002B0002F052F93B4A3C4B02F0C0FB83
:108AB00022002B0002F04AF9394A3A4B01F020FA21
:108AC00022002B0002F042F9374A384B02F0B0FB8B
:108AD00022002B0002F03AF9354A364B01F010FA29
:108AE0002B00220002F032F9354B029003919F4295
:108AF0009FDD344B00229F423DDC334900207B1830
:108B00002E4916001F0002F093FB049005910022ED
:108B1000294B2000290002F019F932003B0002F035
:108B200087FB029A039B06000F002000290002F039
:108B30000DF9009A019B04000D004846414602F0E1
:108B400005F902000B002000290002F071FB020071
:108B50000B003000390002F06BFB02000B000498A0
:108B6000059902F065FB07B00CBC90469946F0BD34
:108B700000201249F7E7154B002604920593144F85
:108B8000C5E7C046FFFF3F3ED43888BEE9FAA8BD1E
:108B9000C4B1B4BD9EEE213EAD529C804F7E923E4C
:108BA0009015CB19A001FA3E7751C1166CC1563F02
:108BB0004C5555555555A53F0000E03F0000F03F8E
:108BC0003233D33F0000E93F0000E0FF0000E73F01
:108BD0000000D23FF0B5DE464E4645465746E0B56A
:108BE000DC4CA5440D9114001900A49A0993DA4BAA
:108BF0009200D6584D1E03901821E01E069602954D
:108C000000F0A0FEC3430100DB1719404B1C9A0083
:108C10009B1ADB001B190B9105934C1B771918D479
:108C2000A59BA5009C463F1922AE6544013707E08D
:108C3000286802F097FE013403C60435BC4208D010
:108C4000002CF5DA00200021013403C60435BC42B3
:108C5000F6D1069B002B01DA00F0FDFB069B039981
:108C60000133DB009A46099BDA0094460092002209
:108C7000914672AA0492B94A6144934688469AABD7
:108C800063449B44029B002B00DABCE15D46002656
:108C90000027039C4D442A686B6803CC02F056F809
:108CA00002000B003000390001F02AF9083D0600EF
:108CB0000F004445EFD1049B4B441E605F600823C6
:108CC0009C46E144D145DDD10EA8042184464942A9
:108CD00061448C46069A93009C44614684460A91FE
:108CE0000399083B63448C460C93009B00926344B9
:108CF0009B46009A0498D10003008C466344089177
:108D00001E685F68002A33DD954980468C466244C0
:108D1000D300984470AB9A460EAB99460022914B13
:108D20003000390002F012F802F0E6FD02F01AFEFF
:108D300000228D4B04000D0002F008F802000B0029
:108D40003000390002F074FA02F0D6FD4B4601C340
:108D50009946434620001A685B68290001F0D0F864
:108D600008235B429C46E04406000F00D045D5D165
:108D7000059B30001A003900984600F0DFFCFF2305
:108D800000229B0504000D0001F0E0FF00F038FC1C
:108D90000022764B01F0DAFF02000B0020002900D0
:108DA00002F046FA0D00040002F0A6FD814602F032
:108DB000D9FD02000B002000290002F039FA06005C
:108DC00040460F00002800DCEEE0009B18215A1EF0
:108DD00092000EAB9B58091A1D000D41A9448D400D
:108DE0005D1B0EAB9D5017231B1A1D41002D2DDD61
:108DF00001239C46009BE144002B00DC1CE20E9CFE
:108E00000123002C00D0B5E0009A012A09D0990076
:108E10000EAA54580133002C00D0ACE0009A9A42BC
:108E2000F5D1059B002B0EDD012B00D1A8E1022B13
:108E300009D1009B0EA95A1E92000EAB9B580793B6
:108E40009B029B0A8B50022D00D1C1E0002300221F
:108E50003000390000F080FE009B002800D194E231
:108E6000069A591E8A4210DC414A0A9894460EAA74
:108E70006344944600229B0063441C68043B2243E5
:108E80008342FAD1002A00D0C0E0069B0EAA013B23
:108E90009B00D358002B00D0B3E001220C9B043B75
:108EA000596801320029FAD0009B9C4662441100A7
:108EB00007921A0001338B4246DC0B9863468046CA
:108EC000A59C4344A046099C9B00A1464A44984463
:108ED000D30022AA9146049A99449446089BA59AE5
:108EE00063448446614494469A468B0063440093ED
:108EF0004346586802F036FD4B4618605960029BA5
:108F0000002B24DB4D46039C0026002701E0286847
:108F100069680CCC01F01AFF02000B003000390028
:108F200000F0EEFF083D06000F005C45EFD1534610
:108F30009E60DF6004239C460433E0449C46009B13
:108F4000E144E2449845D3D1079B0093D1E6002643
:108F50000027ECE794FDFFFF08E9000018FEFFFF83
:108F6000FFFFFF1F0000703E000070410000204026
:108F7000FFFFFF3F002180225204141B0EAA545011
:108F8000009999420EDD0EA884469B000EAA890026
:108F9000D25861446344CF4800E01A68821A04C37F
:108FA0008B42FAD101243CE7059B002B06D1009BA4
:108FB0000EAA013B9B00D558ED1517E70022C64BC2
:108FC000300000F0EDFD002800D024E100253DE751
:108FD00032003B000020C14902F02AF906000F00D0
:108FE000002C00D132E7059A0020BC4900F0A6FB16
:108FF00002000B003000390002F01AF906000F00E1
:1090000024E7012250E70026002754E64B46059A44
:10901000079388468B000EA9CB58183A08950592FD
:10902000002B0DD18C464146AD4B43449B0063441D
:10903000043B58680139183A0028F9D0884605924F
:10904000059A0020A54900F079FB434604000D0075
:10905000002B00DA05E29E000EAB9C464346DB0087
:1090600066449C46059370AB9946049F67440097FD
:10907000306802F077FC22002B0001F067FE00222E
:1090800038607960974B2000290001F05FFE083FAF
:1090900004000D00043EB945EAD14AAB03939B4658
:1090A00000239A46069B4246994643460132029265
:1090B00004934B46002B00DAAAE080208A4B009DE7
:1090C0009846C005894900260027002408E00823A7
:1090D0009C460835E044544511DC434618685968FD
:1090E0002A686B6801F032FE02000B003000390084
:1090F00000F006FF013406000F00A145E7DA5B46E9
:10910000C0C39B4601239C46009BE244083B00935E
:10911000029B9A45CDD1049B9846A49B022B00DD6F
:109120008EE0002B37DC1FD1059B00271D00039B21
:1091300000249C461E006544083E2A686B6838007F
:10914000210000F0DDFE083D07000C00AE42F4D126
:10915000089B002B03D080231B069C4664443A00E6
:1091600023000D990A604B600720079B18409B2342
:109170009B009D443CBC90469946A246AB46F0BD40
:10918000009B0EA95A1E92000EAB9B5807935B02E0
:109190005B0A8B5057E64346002B00DA70E1002053
:1091A0000021DB004AAAD61848AF32687368083E2F
:1091B00000F0A6FEB742F8D1089B002B00D025E1B5
:1091C0000B0002004A984B990D9C2260636002F0EC
:1091D0002FF8434607000C00002B13DD01254CAE91
:1091E000B14638002E0021004C4601360CCC00F070
:1091F00087FEA146B045F7DA089B07000C00002B5C
:1092000000D015E13A0023000D998A60CB60ABE7EE
:109210000026002773E701239C46009BE1440225BA
:10922000002B00DDEBE532003B0000202B4901F074
:10923000FFFF06000F0009E60024F2E54AAB0393A6
:10924000A49B032B00D08FE74346002B00DC14E1E6
:10925000039ADB009B46130091465B441E685F68DF
:10926000234B43440293DB00994448AB9A464B4658
:109270005C681B681800210032003B0000900191DF
:1092800000F03EFE04000D0002000B000098019962
:1092900001F0CEFF3B00320000F032FE4B469860FA
:1092A000D9601C605D6008235B429C46E144260057
:1092B0002F00CA45DBD14346012B00DCE3E0039AD3
:1092C00013005B441E685F68029BDB0099464A44BA
:1092D000904610E0FFFFFF000000E03F0000F03F7D
:1092E000FFFFFF3F0000703EC8E80000FB21F93F90
:1092F000FFFFFF1F984643465C681B68180021006B
:1093000032003B000090019100F0FAFD04000D00D6
:1093100002000B000098019901F08AFF32003B0027
:1093200000F0EEFD4346039A9860D9601C605D60D2
:10933000083B26002F009A42DCD14D469446002679
:1093400000244746083565442A686B6830002100D0
:1093500000F0D6FD083D06000C00AF42F4D1039B9F
:109360004A9F5D689968D868089B002B65D0802269
:10937000120694460D9B6544604464441F605D6022
:109380009960D8601E615C61EEE69A464B46079391
:10939000059B30005A423900089500F0CFF90022B1
:1093A0003A4B06000F0000F0FBFB002824D0384B9E
:1093B00000223000390001F0C9FC02F09DFA52464B
:1093C0000400950002F0CEFA0022304B01F0BEFC02
:1093D00002000B003000390001F02AFF02F08CFA85
:1093E0000EAA50510122059B524418339046059312
:1093F00093000EAAD45023E65346300039009C0057
:1094000002F07AFA0EAB1851D04619E680230D9A75
:109410001B06CB18106053600B0002004A984B9952
:1094200001F006FF434607000C00002B00DDD5E6E7
:1094300080231B069C466444E4E62B003A000D9D05
:109440002A606B600A000300AA60EB603200230010
:109450002A616B6188E6099BDB00009372AB049381
:1094600032E4A49B022B00DDE8E6002B00DD92E64F
:1094700000D079E6002700246AE6002600246EE783
:109480000020002198E60026340068E700007041C3
:109490000000703EF0B5CE46474680B587B00092DA
:1094A0000193474A4B00814688465B08934207DC9C
:1094B0004146484602F020FA4146031E484666D01F
:1094C0004A4643464846414601F040FC04000D0030
:1094D00002000B004846414601F038FC394A3A4B3D
:1094E00006000F002000290001F030FC374A384BFD
:1094F00001F09EFE22002B0001F028FC354A364B7D
:1095000000F0FEFC22002B0001F020FC334A344B1B
:1095100001F08EFE22002B0001F018FC314B324A84
:1095200000F0EEFC0E9B02900391002B34D00098CB
:10953000019900222D4B01F009FC029A039B049033
:1095400005913000390001F001FC02000B00049885
:10955000059901F06DFE22002B0001F0F7FB009A47
:10956000019B01F065FE224A04000D00214B3000F2
:10957000390001F0EBFB02000B002000290000F095
:10958000BFFC02000B004846414601F051FE07B007
:109590000CBC90469946F0BD02000B00200029004B
:1095A00001F0D4FB124A134B01F042FE32003B00A3
:1095B00001F0CCFB4A46434600F0A2FCE7E7C04678
:1095C000FFFF3F3E7CD5CF5A3AD9E53DEB9C2B8A35
:1095D000E6E55A3E7DFEB157E31DC73ED561C11990
:1095E000A0012A3F1111813FA6F810110000E03FB1
:1095F000495555555555C53F49004B081900704709
:10960000474AF0B54F4691464B005B0D994446469C
:10961000D6464A46C0B505000C000E008846070035
:10962000132A27DC002A4BDB3E4B13419A460B00E2
:1096300052461340034318D03B4A3C4B28002100BC
:1096400000F05EFC0022002300F0A0FA002847D0C2
:10965000002C04DA80234A465B03134198444646B3
:10966000534600279E43380031001CBC9046994663
:10967000A246F0BD332A08DD8023DB009945F4D1F2
:1096800002000B0000F03CFCEFE7294A944601225F
:1096900063445242DA4092460242E6D0224A234BC9
:1096A0002800210000F02CFC0022002300F06EFABC
:1096B000002815D0002C1EDB534646469F430FE082
:1096C000194A1A4B2800210000F01AFC002200233E
:1096D00000F05CFA002803D0002C04DB00270026F1
:1096E00038003100C1E76400640825430027002DDD
:1096F000F6D0104EF4E74B46142B0BD03422D21A7E
:10970000012393405D19BD4208D201239C462F00DE
:10971000E044D1E7133B9C46E044CDE72F00CBE784
:1097200001FCFFFFFFFF0F009C7500883CE4377EC3
:10973000EDFBFFFF0000F0BF002070474B0070B54D
:109740005B0D14000A00002B1AD14B005B08034389
:1097500015D0234B002201F0F9FA224B9C422DDB5D
:109760000A004B005B0D363B1F4DE318AB422ADC71
:10977000002B0DDD1D4C1B0522401A43110070BD4E
:109780001B4DAB42F0D102000B0000F0B9FBF6E735
:109790001D00353519DA174B02009C4209DD0B001C
:1097A0001548164900F032F8134A144B01F0CEFA6E
:1097B000E5E70B001248134900F028F8104A114B56
:1097C00001F0C4FADBE70200E9E7084C3633224037
:1097D0001B051343190000220B4B01F0B7FACEE72B
:1097E00000005043B03CFFFFFE070000FFFF0F806A
:1097F000FF07000050C300009C7500883CE4377EE2
:1098000059F3F8C21F6EA5010000903C30B54A0024
:10981000DB0FDB0752081A43110030BD02B471465A
:1098200049084900095C49008E4402BC7047C046A3
:10983000002243088B4274D303098B425FD3030A8F
:109840008B4244D3030B8B4228D3030C8B420DD3A2
:10985000FF22090212BA030C8B4202D31212090230
:1098600065D0030B8B4219D300E0090AC30B8B426E
:1098700001D3CB03C01A5241830B8B4201D38B031C
:10988000C01A5241430B8B4201D34B03C01A5241C1
:10989000030B8B4201D30B03C01A5241C30A8B4204
:1098A00001D3CB02C01A5241830A8B4201D38B02EF
:1098B000C01A5241430A8B4201D34B02C01A524193
:1098C000030A8B4201D30B02C01A5241CDD2C30905
:1098D0008B4201D3CB01C01A524183098B4201D381
:1098E0008B01C01A524143098B4201D34B01C01A6C
:1098F000524103098B4201D30B01C01A5241C308E4
:109900008B4201D3CB00C01A524183088B4201D352
:109910008B00C01A524143088B4201D34B00C01A3E
:109920005241411A00D20146524110467047FFE7AA
:1099300001B5002000F0F0F802BDC0460029F7D0C4
:1099400076E7704703460B437FD4002243088B42DF
:1099500074D303098B425FD3030A8B4244D3030BB6
:109960008B4228D3030C8B420DD3FF22090212BA7B
:10997000030C8B4202D31212090265D0030B8B42F7
:1099800019D300E0090AC30B8B4201D3CB03C01AE1
:109990005241830B8B4201D38B03C01A5241430BBC
:1099A0008B4201D34B03C01A5241030B8B4201D3AC
:1099B0000B03C01A5241C30A8B4201D3CB02C01A17
:1099C0005241830A8B4201D38B02C01A5241430A8F
:1099D0008B4201D34B02C01A5241030A8B4201D37E
:1099E0000B02C01A5241CDD2C3098B4201D3CB0125
:1099F000C01A524183098B4201D38B01C01A5241D4
:109A000043098B4201D34B01C01A524103098B42D7
:109A100001D30B01C01A5241C3088B4201D3CB00C2
:109A2000C01A524183088B4201D38B00C01A5241A5
:109A300043088B4201D34B00C01A5241411A00D255
:109A400001465241104670475DE0CA0F00D04942BE
:109A5000031000D34042534000229C4603098B422E
:109A60002DD3030A8B4212D3FC22890112BA030AB6
:109A70008B420CD3890192118B4208D38901921138
:109A80008B4204D389013AD0921100E08909C309BD
:109A90008B4201D3CB01C01A524183098B4201D3BF
:109AA0008B01C01A524143098B4201D34B01C01AAA
:109AB000524103098B4201D30B01C01A5241C30822
:109AC0008B4201D3CB00C01A524183088B4201D391
:109AD0008B00C01A5241D9D243088B4201D34B00AC
:109AE000C01A5241411A00D20146634652415B10EE
:109AF000104601D34042002B00D5494270476346CF
:109B00005B1000D3404201B5002000F005F802BD13
:109B10000029F8D016E770477047C046D0400B1CAC
:109B20001141203A03D49C461341184363465242E4
:109B3000934018437047C0468446101C62468C46CA
:109B4000191C634600E0C0461FB501F097F80028D5
:109B500001D40021C8421FBD10B500F0EFFF404204
:109B6000013010BD10B501F089F8002801DB00209C
:109B700010BD012010BDC04610B501F07FF80028CF
:109B800001DD002010BD012010BDC04610B501F060
:109B900011F8002801DC002010BD012010BDC046D6
:109BA00010B501F007F8002801DA002010BD0120EF
:109BB00010BDC046F0B5CE46474615042D0C2E000C
:109BC00080B50704140C3F0C9946030C7E435D439B
:109BD000674363437F19340CE4199C46A54203D9BB
:109BE00080235B029846C4444B4643435143250CB3
:109BF00036046544360C2404A4195B195918200056
:109C00000CBC90469946F0BDF0B54E4657464546C9
:109C1000DE46E0B543025B0A450083B00F1C99465F
:109C20002D0EC60F002D57D0FF2D24D08020DB0035
:109C3000C0041843002381469A469B467F3D7C0220
:109C40007A00FB0F640A120E984623D0FF2A4BD0ED
:109C5000E30080240020E4047F3A1C43AD186B1C11
:109C600047460193534677403A000F2B48D87D4929
:109C70009B00CB589F46002B00D085E008339A46C6
:109C8000063B9B467C027A00FB0FFF25640A120EFE
:109C90009846DBD1002C00D090E0524601231A43B5
:109CA00092460120DBE74C4658461700022824D094
:109CB000032800D1CFE00022002301284DD1580213
:109CC000D205400AFF071043384303B03CBC90461E
:109CD0009946A246AB46F0BD002B5BD104239A46C1
:109CE000033B00259B46AAE7FF35002C60D1524676
:109CF00002231A4392460220B1E7FF220023DEE747
:109D00004B461B0C9C464B462604360C18046146F9
:109D10003300220C6446000C43434E4350435443EB
:109D200080191A0C1218964203D9802149028C46D8
:109D300064441B041B0C1004C01883015E1EB34155
:109D4000800E1843130C1B199B0103431C002301B5
:109D500079D5012362081C401443019A7F32002AFE
:109D60004DDD630704D00F232340042B00D00434BF
:109D7000230103D53C4B019A1C408032FE2ABCDCF7
:109D8000A3015B0AD2B29AE70C239A46093BFF254E
:109D90009B4654E7180001F071FE4A46431F7625A2
:109DA0009A4000236D4291462D1A9A469B4646E7FB
:109DB000524603231A439246032050E7200001F045
:109DC0005DFE431F2D1A9C40763D002047E780230F
:109DD0000027DB03FF2272E7424666E74C4632006B
:109DE000584662E780234A46DB031A4222D01C42CF
:109DF00020D123435B025B0A4746FF225FE7012332
:109E00009A1A1B2A21DC23000199D3409E318C40F1
:109E10001A0023005C1EA34113435A0704D00F22EB
:109E20001A40042A00D004335A0111D49B015B0A62
:109E3000002244E780234A46DB0313435B025B0AAC
:109E40003700FF223BE7019587E70022002336E732
:109E50000122002333E78023DB0323435B025B0AF9
:109E6000FF222CE718E90000FFFFFFF770B500287C
:109E70003DD0C317C5185D40C40F280001F0FEFD9A
:109E80009E22121A962A07DCD2B2082833DD08383F
:109E900085406802400A23E0992A0BDD052329004A
:109EA0001B1AD94003001B339D402B005D1EAB41A4
:109EB00019430D00052801DD431F9D402B000F496C
:109EC0000B406E0709D00F263540042D05D0043312
:109ED0005D0102D59F220B40121A9B01580AD2B293
:109EE0004002D205400AE4071043204370BD00241D
:109EF00000220020F4E76802400AF1E7FFFFFFFBC1
:109F0000F0B54F464646D6460C000903C0B5490A8F
:109F1000470F5E0039431F03DB0F9C4665007B0A39
:109F2000570F1F436D0DE40F760DA146C000B846D4
:109F3000D200AB1B64457BD0002B5FDD002E00D030
:109F4000A4E03E00164300D112E15E1E002E00D0B8
:109F50009EE1871A4346B84280410125C91A404212
:109F6000091A0B0200D431E149024E0A002E00D139
:109F70006EE1300001F082FD0300083B1F2B00DD85
:109F800061E120223900D21A9E40D1409F400E4309
:109F90009D4200DD51E15D1B6B1C1F2B00DD7CE150
:109FA0002021C91A3D0030008F408840DD40791ED5
:109FB0008F41310007222843D940002507433A400A
:109FC000002A09D00F233B40042B05D03B1DBB4288
:109FD000BF417F42C9191F000B0200D426E26A1C50
:109FE000C64B55056D0D9A4200D106E1C44AFF08E3
:109FF0000A40530752023B43120B8EE0002B00D065
:10A00000B8E06B1C5B055B0D012B00DC30E1871AAF
:10A010004346B842B641CB1A76429E1B330200D566
:10A020004CE13B003343A1D100220024002570E025
:10A03000002B00DCE5E0002E00D183E0AF4EB542FE
:10A0400060D0802636043743B846382B00DC3EE12A
:10A05000434613431F007A1E97413F1887428041B1
:10A06000404209180B0200D4B0E0A44B01359D42D8
:10A0700000D1C3E0A24A7B080A4001210F401F43E0
:10A080005108D30707221F433A4099E79B4EB54238
:10A0900038D0802636043743B846382B00DDDCE064
:10A0A0001F2B00DC30E11E004746203EF740BC4637
:10A0B000202B04D04026F31A46469E403243170018
:10A0C00063467A1E97411F43CCE0002B00D104E287
:10A0D0004346134300D159E14B07C008184380237E
:10A0E000C9081B03194208D04546ED081D4204D19A
:10A0F0004346D008590708432900420FC9007F4D45
:10A100001143C0004B07CA087C49C00803438D4275
:10A1100068D012036D05120B6D0D0021120318009B
:10A12000130B0A0D12051A43764B2D0513402B43D2
:10A130005B00E4075B08234319001CBC904699466A
:10A14000A246F0BD3E00164312D05E1E002E00D087
:10A1500000E18718874280414144404209180125A7
:10A160000B0233D5022585E76446330041461000D3
:10A170001D00C7E7002D00D0DAE00C000443F3D047
:10A180005C1C00D19FE15D4CA64200D12FE1DB4376
:10A19000382B00DD66E11F2B00DD83E12024050064
:10A1A000E41A0F00DD40D940A0404346A7405B1AA7
:10A1B000441EA04198462F433843171ABA42924191
:10A1C00043465242991A64463500CAE607223A408D
:10A1D000002A00D0F6E64B07CA084849FF083B436F
:10A1E0008D4296D11900114300D19EE180210903CF
:10A1F0000A431203120B414D8FE715000022002382
:10A200008BE7002B00D0C7E06B1C5F057F0D012F93
:10A2100000DCF1E0394DAB4200D1B9E085180A000D
:10A22000854289414244494251180722CF076D08AF
:10A230002F4349083A401D00C2E607223049ED1A73
:10A2400031403A40BCE63E002838864000279FE671
:10A25000380001F013FC20308EE6434613431F0004
:10A260007A1E9741C71BB84280414042091A78E6DE
:10A270000E003B0006431343002D61D1002E00D099
:10A28000F4E0002B00D11BE164463900100039E7EF
:10A290001A4FBB427AD03300FFE630001F3DE84042
:10A2A000202B03D04021CB1A9E4037437B1E9F4179
:10A2B000072207433A400021002589E7171A434641
:10A2C000BA42B641591A76428E1B64464EE61F2B9F
:10A2D00000DDADE020264746F61AB740B946170024
:10A2E000B246DF404E463E4337005646B240561E09
:10A2F000B24117434246DA408918AEE6FF07000034
:10A30000FFFF7FFFFFFF0F8020264746F61AB7406A
:10A31000B9461700B246DF404E463E433700564628
:10A32000B240561EB24117434246DA40891A99E7B5
:10A330007F4CA6425BD0802424045B42214327E764
:10A34000002E0CD1002B00D1CBE064463900100068
:10A35000774DD7E6764FBB4218D0330075E6002B19
:10A3600014D04B07C00818438023C9081B031942A7
:10A3700007D0FC081C4204D17907D0080843E14605
:10A3800021004C46420FC9001143C000684DB9E698
:10A390001D0000220023C0E6002D5BD10D00054307
:10A3A00000D1E2E65D1C00D1B0E0614DAE421FD0AD
:10A3B000DB43382B71DC1F2B00DD96E020250F00DE
:10A3C000ED1AAF40B9460700AA46DF404D463D436F
:10A3D0002F005546A840D940451EA8418844074350
:10A3E000BF18974292415142414435003AE66446D3
:10A3F00035004146100085E60B000343002D00D0D8
:10A4000063E6002BF5D04346134300D17AE6871864
:10A410008742804107224144404209183A400B02DA
:10A4200000D4D5E6434B01351940C9E5380069E64B
:10A430001E004746203EF740BC46202B04D0402655
:10A44000F31A46469E403243170063467A1E9741F0
:10A450001F4302E6364DAE42CAD080252D045B4232
:10A460002943A6E70843411E8841A6E6002B00D1F8
:10A4700048E6871A4346B842B641CB1A76429E1B3D
:10A4800033024BD5171A4346BA429241591A5242E7
:10A49000891A072264463A4092E501430F00791E6B
:10A4A0008F419DE71C000F00203CE740202B03D08C
:10A4B0004024E31A99400843411E884138437CE612
:10A4C0000022002425E6171A4346BA429241591A3F
:10A4D0005242891A6446350043E541461000144D46
:10A4E00010E680220024120380E61D000F00203DAC
:10A4F000EF40BC46202B03D04025EB1A994008437F
:10A5000007006346781E87411F4369E78718974213
:10A510009B4141445B42C9183500A3E53B003343EE
:10A52000CED0072231003A4052E600231A00F4E56B
:10A53000FF070000FFFF7FFFF0B55746DE464E469F
:10A540004546E0B5834607000E03480085B09246B5
:10A550001C00360B400DCD0F002800D19DE0954B1F
:10A56000984239D08023F6001B041E43924A7B0F89
:10A570003343994694460300634400930023002626
:10A58000FF00029323031B0B98466300E40F52461F
:10A590005B0D019400D1B3E086498B4200D19EE06F
:10A5A0004246D100802212040A435146490F11430A
:10A5B0008B46814952468C4600996344CB1A002150
:10A5C000D20000932B0063409A460F2E00D905E17C
:10A5D0007A4BB6009B599F465B463343994600D061
:10A5E000B8E002230826002700900293CAE7CB4672
:10A5F0003A0002990195019B9A46022927D0032926
:10A6000000D180E2012944D06D49009B8C4663440F
:10A610001C00002C38DD530700D013E2D2085B4643
:10A62000DB0109D55946674B19408B468021C9008B
:10A630008C46009B63441C00634B9C4207DC5B46DA
:10A6400064055F075B0217431B0B620D02E00023EA
:10A650000027584A00211B031C0B0B0D1B0523432D
:10A6600014055A4A380013401C4353466400DB0764
:10A6700064081C43210005B03CBC90469946A246A4
:10A68000AB46F0BD0122524201231B1B382B00DCDC
:10A69000ADE1002200230027DCE75B463343994607
:10A6A0005ED0002E00D18AE1300001F0E7F903000E
:10A6B0000B3B1C2B00DD7BE11D22D31A5A46010007
:10A6C000DA4008398E4013005F46334399468F4085
:10A6D0003F4B00261B1A00930023029352E741468A
:10A6E00053460B433B499B468C46009B6344009377
:10A6F0005B46002B3BD1022300221E43022161E76F
:10A70000434613439B4637D04346002B00D162E1BA
:10A71000404601F0B3F903000B3B1C2B00DD53E175
:10A7200002004146083A914088461D21CB1A514605
:10A73000D9400B0041460B439B46534693401A00B9
:10A74000009B25499C46604403008C46634400936B
:10A75000002137E70323B14600900C26029311E74E
:10A760000023009301330426002702930AE7032302
:10A77000C3461E43032125E701331E430022012166
:10A7800020E700239A46802300271B03094A61E73C
:10A79000802349461B03194200D1E2E05946194281
:10A7A00000D0DEE00B431B0317001B0BA246014A3F
:10A7B00050E7C046FF07000001FCFFFF58E900001A
:10A7C000FF030000FFFFFFFEFE070000FFFF0F80FA
:10A7D0000DFCFFFF01F8FFFFF3030000D94500D98E
:10A7E000CBE000D1C6E03C0048460027009B013B7F
:10A7F00000935B46160E1B021E4313029846330459
:10A800001B0C9946310C0191FFF798F84A464243D8
:10A810000B04210C050019438A4207D98919013D0F
:10A820008E4203D88A4201D9851E8919881A019956
:10A83000FFF784F809048C464A46210464464243E3
:10A84000090C030021438A4204D98919013B8E4235
:10A8500000D8F1E02D041D43AB464346891A424619
:10A86000280C12041D0C5B46140C22001B041B0C4C
:10A870005A4303946B434443029568431B19150CD8
:10A88000EB189C4203D980246402A44660441C0C4B
:10A8900015041B042D0C20185D19814277D373D049
:10A8A0000C1AA24A7D1BAF42BF419446009B7F42D7
:10A8B0006344E01B1C00864200D1DBE00199FFF7F6
:10A8C0003DF84A4642430B04290C070019438A42CB
:10A8D00007D98919013F8E4203D88A4201D9871EC0
:10A8E0008919881A0199FFF729F809044A46894607
:10A8F00029044D464243090C030029438A4207D9E3
:10A900008919013B8E4203D88A4201D9831E8919D5
:10A910003F04891A3A00039F1A43380013041B0CA2
:10A92000584381460298150C6F43434345434846BC
:10A93000000C8446DB1963449F4203D98020400207
:10A940008446654448461F0C00041B04000C7D1916
:10A950001818A94200D284E000D17FE001231A43F5
:10A9600057E680234A461B0313431B031B0BAA46CF
:10A970006F4A6FE6BA4200D935E74B46DC07580804
:10A980007B081C43FF0734E70024AF4289D24744C9
:10A990004745A4415B466442A4196418013BA642A2
:10A9A0001ED2A0426DD800D1B6E0241A9B4678E7AB
:10A9B00003005A46283B9A400027914688E65846AD
:10A9C00001F05CF8203072E603005246283B9A40C2
:10A9D00093460022B4E6504601F050F820309AE643
:10A9E000A642E2D1B845DCD9341A9B4659E71F2B61
:10A9F00065DC504C0099A4465C46614408008C40DC
:10AA000011008240D940501E82410C4314435A46E3
:10AA1000DA401300620709D00F222240042A05D031
:10AA20002200141D9442894149425B181A0262D5E2
:10AA30000122002300270DE68A4200D80AE7831E80
:10AA4000891907E70F231340042B00D1E6E5171DF2
:10AA50009742924153429B44FA08E0E5002800D116
:10AA6000D7E57118531EB14227D3A94215D358D048
:10AA70001A0073E7002B00DC04E6012300229B444C
:10AA8000CDE502234744474589415B429C46494204
:10AA900089190C19E344241A03E743465F0047452C
:10AAA0009B41B8465B429E19023A8919A94200D0DF
:10AAB00054E7404500D051E7ABE51A00F6E71F2107
:10AAC0005F4649420C1BE740202B07D01A49009BE8
:10AAD0008C46634418005B4683401A43501E8241F3
:10AAE0003A4307270023174009D00F2100231140C4
:10AAF0001400042995D122005F075B021B0BD208CA
:10AB000017430022A6E5802359461B030B431B0372
:10AB100017001B0B064A9DE5BD42B2D89B46002498
:10AB2000BFE68045B9D31A00C3E7C046FF03000063
:10AB3000FF0700001E0400003E040000F0B54F4671
:10AB40004646D6468446C0B58046194E18030F03C4
:10AB50004D00000B5C0082463F0B6D0DC90F914606
:10AB6000640DDB0F0120B5420AD0B44203D0A542E8
:10AB700001D157450CD01CBC90469946A246F0BD69
:10AB800066463E43F7D1AC42F5D154461443F2D168
:10AB90000120C845EFD1994207D0002DEBD1634683
:10ABA0001F433800471EB841E5E70020E3E7C046F1
:10ABB000FF070000F0B54F464646D6464D00C0B5EB
:10ABC0000E03C90F8A462C491F035C008046360BD2
:10ABD0006D0D91463F0B640DDB0F8D421ED08C42F4
:10ABE00016D0002D1ED130438446002C01D13A43AB
:10ABF00023D06246002A1AD09A4529D05146022015
:10AC00000139084001381CBC90469946A246F0BD67
:10AC100039001143E5D002204042F4E73043FAD135
:10AC2000AC420FD0002C0FD13A43E7D00CE0012208
:10AC3000013B934318000130E5E763460020002BF9
:10AC4000E1D0DBE73A43E6D19A45D7D1A542D5DC3E
:10AC5000A54205DBBE42D1D808D00020BE42D2D2E8
:10AC600050460123013898430130CCE7C845C5D888
:10AC70000020C845F4D3C6E7FF070000F0B54F46F3
:10AC80004646D6464D00C0B50E03C90F8A462E492A
:10AC90001F035C008046360B6D0D91463F0B640D23
:10ACA000DB0F8D4218D08C4211D0002D18D13043CB
:10ACB0008446002C1ED13A431CD163460020002B51
:10ACC00030D0514602200139084001382AE03900CD
:10ACD0001143EAD0022025E03043FBD1AC4226D01C
:10ACE000002C26D13A4324D1514602200139084094
:10ACF000013817E06246002A0FD09A45E1D1A542FB
:10AD000005DBBE42DDD819D00020BE420AD2504633
:10AD1000012301389843013004E00122013B9343B1
:10AD2000180001301CBC90469946A246F0BD3A433B
:10AD3000D0D19A45C5D1A542C3DCE0E7C845C0D80B
:10AD40000020C845E3D3EDE7FF070000F0B5574604
:10AD5000DE464E464546E0B5834606000F034800F2
:10AD600087B092461D003F0B400DCC0F002800D14C
:10AD70006FE0DE4B984238D08023FF001B041F4356
:10AD8000730F3B430193DA4B0027994600239B4600
:10AD9000F60081442B0369001B0B52469846490D6F
:10ADA000ED0F002900D185E0D04B994200D173E02E
:10ADB0004346DA0080231B0413435246CC48520F0B
:10ADC00084461343524600206144D2008944210046
:10ADD000694000918C46012149448A460F2F00D9D1
:10ADE00090E0C449BF00CF59BF465B463B43019347
:10ADF00000D06AE102230827002681469B46C9E766
:10AE000032005846019B61460091022800D175E04E
:10AE1000032800D1FEE1012800D02CE10023002707
:10AE2000002600253F032A0D3F0BB34812053A4385
:10AE300002401B051343009A5B00D1075B080B43DC
:10AE40003000190007B03CBC90469946A246AB467C
:10AE5000F0BD5B463B43019300D12FE1002F00D1B1
:10AE6000A5E1380000F00AFE03000B3B1C2B00DDBF
:10AE700096E11D22D31A5A460100DA405E4608398F
:10AE80008F4013008E403B4301939C4B00271B1ABD
:10AE9000994600239B467DE7414653460B43934921
:10AEA0008C46E144002B00D01AE102220220174315
:10AEB00000228CE7134300D10DE14346002B00D163
:10AEC00081E1404600F0DAFD02000B3A1C2A00DD69
:10AED00072E10100434608398B4098461D239A1AB7
:10AEE0005346D3401A004346134352468A404946CC
:10AEF000081A824989468144002068E77B4B002775
:10AF000000268EE7140C1204120C1100370C3604C4
:10AF1000350C794328008C462E00604360448346FC
:10AF200056432100300C80465846794340440291F4
:10AF3000844506D98846802149028C46E044414632
:10AF400002913604010C360C00048B4681191E0C4C
:10AF50001B041B0C0391190079438C462800754390
:10AF60006544A8465843050C45447743A94203D994
:10AF7000802149028C466744290C8C463900000424
:10AF8000000C2D042D186144AB44059159460491E1
:10AF900001990F043F0C080C39005143424390467D
:10AFA00002008C46090C8B4662437C4344445C445B
:10AFB000A04503D98021490288464244210C884695
:10AFC00061460904090C8C463900594343437043D8
:10AFD0007E430F0CF6182404BE19644442448C4688
:10AFE000B34203D980235B0298464044029B6146EA
:10AFF0009846049B370443449B46AB45AD416B42A6
:10B000000D0405992D0C8C467F196744FD18A84640
:10B010005D462D19A542A44193466442A446C3440B
:10B02000DC448F42BF4198459B4193459241A445E2
:10B03000A4415B427F421F43360C52426442BF1917
:10B040002243BF18624638184302D20D03991343B6
:10B050006A020A43501E82416146ED0D2A434E02A8
:10B060003243D90100D4B3E00126500832400243F4
:10B07000DE0732435B08224C5444002C62DD51074A
:10B0800009D00F201040042805D0101D9042924195
:10B0900052429B180200D90104D580241948E400CB
:10B0A000034054441848844200DD27E75E075B02F2
:10B0B000D2081F0B630516435B0DB2E600239946C9
:10B0C0000133042700269B4664E60323019781464B
:10B0D0000C279B465EE6012201201743002276E6FC
:10B0E000032303201F43434671E6C046FF070000C9
:10B0F00001FCFFFF98E90000FFFF0F800DFCFFFF40
:10B10000FF030000FFFFFFFEFE0700000023802773
:10B1100000933F030026434B83E6019B3200A44685
:10B12000584670E6AC466EE6802701993F033942E7
:10B130002DD03B422BD11F433F033F0B0095160000
:10B14000384B6EE601252D1B382D00DD66E61F2DE0
:10B1500040DC35481C005044160082408440EE40DC
:10B16000501E824134431443EB40620709D00F2242
:10B170002240042A05D02200141D944280414042FE
:10B180001B181A023ED501230027002649E6802716
:10B19000019B3F031F433F033F0B0094214B40E6BD
:10B1A00003005A46283B9A40002601926DE6584615
:10B1B00000F064FC203057E603005246283B9A40DA
:10B1C0001300002293E6504600F058FC20307BE646
:10B1D000CA4650E71F201E004042041BE640202DB7
:10B1E00003D0124C5444A3401A43501E82413243B0
:10B1F00007260027164009D00F2000231040140016
:10B200000428B9D122005E075B021F0BD208164347
:10B21000002306E680273F031F433F033F0B160032
:10B22000004BFEE5FF0700001E0400003E04000086
:10B23000F8B557464E464546DE460C000903E0B5D4
:10B24000490A460F5F0031431E03DB0F760A9B4617
:10B25000530F3343C84E6500C000E40FD2006D0D9C
:10B26000A24681467F0D9C469046B74200D1B9E088
:10B270005B46012673409B46EE1BA34500D183E04D
:10B28000002E63DD002F00D0B1E06346134300D1F0
:10B2900023E1731E002B00D0BAE1861A6346B04248
:10B2A00080410125C91A4042091A0B0200D447E126
:10B2B00049024B0A98464346002B00D189E140469B
:10B2C00000F0DCFB0300083B1F2B00DD7CE12022AB
:10B2D0003000D21A4146D040994002009E400A43B5
:10B2E0009D4200DD6AE15D1B6B1C1F2B00DD94E1BC
:10B2F000202110003500C91A8E40DA408840DD4018
:10B30000711E8E411100072228430025064332405A
:10B31000002A09D00F233340042B05D0331DB3423C
:10B32000B641764289191E000B0200D43DE26A1C28
:10B33000914B55056D0D9A4200D119E18F4AF608DF
:10B340000A40570752023743120B9BE0002E00D0F1
:10B35000C5E06E1C7605760D012E00DC48E16746DF
:10B36000861ACB1BB042BF417F42B8461F004346FE
:10B37000FF1A3B00B8461B0200D55FE137439AD164
:10B3800000220024002579E0002E00DCFAE0002FE6
:10B3900000D18DE0784B9D4267D0802367461B0427
:10B3A0001F43BC46382E00DC52E1634613435A1E4D
:10B3B00093411E1886428041404209180B0200D476
:10B3C000BEE06D4B01359D4200D1D2E06B4A73085F
:10B3D0000A4001210E401E435108D30707221E4395
:10B3E000324095E71E00164300D045E740E7624B28
:10B3F0009D423AD0802367461B041F43BC46382E2B
:10B4000000DDEBE01F2E00DC3AE133006746203B15
:10B41000DF403B00202E05D04027BF1B6646BE40C4
:10B42000324390464646721E96413343DAE0002B83
:10B4300000D114E26346134300D168E180234E0734
:10B44000C008C9081B030643194208D06046C0085B
:10B45000184204D163460100D2085E071643F30088
:10B460009946C900720F444D11434B46DE08424BCA
:10B470004F073743CA089D4200D16EE012036D05A5
:10B48000120B6D0D00211203130B0A0D12051A4346
:10B490003B4B2D0513402B435B00E4075B08234324
:10B4A000380019003CBC90469946A246AB46F8BD10
:10B4B0006346134311D0731E002B00D007E186189A
:10B4C0008642804161444042091801250B0237D56C
:10B4D00002257BE73E00614691463500C5E75C46A4
:10B4E000002D00D0E1E00B000343F3D0731C00D12A
:10B4F000ACE1214B9F4200D13AE1F343382B00DD10
:10B500006FE11F2B00DD8CE120250E00ED1AAE400F
:10B51000B0460600AA46DE40454635432E00554655
:10B52000D940A8406346451EA8415B1A9C4630435B
:10B53000161AB242924163465242991A3D00B4E64D
:10B5400007223240002A00D0E4E60B4BF6084F07F2
:10B550003743CA089D4200D090E73B00134300D117
:10B56000A6E180231B031A431203120B024D89E745
:10B5700015000022002785E7FF070000FFFF7FFF7F
:10B58000FFFF0F80002E00D0C7E06B1C5E05760D1C
:10B59000012E00DCF0E0C84DAB4200D1B9E08518C7
:10B5A0000A00854289416244494251180722CE0768
:10B5B0006D082E43490832401D00A9E6BF49ED1A27
:10B5C000114007223240A3E632002838824000268C
:10B5D00086E6300000F052FA203073E663461343EB
:10B5E0005A1E9341C61AB04280414042091A5CE695
:10B5F0000E00674606431743002D5ED1002E00D093
:10B60000F3E0002F00D11EE15C46614691462CE735
:10B61000A94FBE427BD01E00F1E610001F3DE8405E
:10B62000202B03D04021CB1A9A401643731E9E4113
:10B630000722064332400021002583E7161A63469D
:10B64000B2428041591A40420B1A98465C4632E693
:10B650001F2E00DDABE02027BB1B9A4663465746F2
:10B66000BB40994613004F46F3401F433B005746EB
:10B67000BA40571EBA4113436246F240891898E611
:10B680002027BB1B9A4663465746BB40994613008A
:10B690004F46F3401F433B005746BA40571EBA413E
:10B6A00013436246F240891A9CE7834B9F425FD066
:10B6B00080252D047342294320E7002E0CD1002F52
:10B6C00000D1D0E05C46614691467B4DCDE67A4F95
:10B6D000BE421CD01E0065E6002F18D0C0084E07E1
:10B6E00006438020C9080003014208D06346DC08F5
:10B6F000044204D12100DA46D2085E071643F30063
:10B70000994601245346C900720F11431C406A4DEB
:10B71000ABE61D0000220027B4E6002D59D10B0036
:10B72000034300D1D6E6731C00D1B2E0624B9F42C6
:10B730001ED0F343382B6FDC1F2B00DD97E0202554
:10B740000E00ED1AAE40B0460600AA46DE40454661
:10B7500035432E005546A840D940451EA8418C448B
:10B760000643B61896429241514261443D0025E697
:10B770003D006146914678E60B000343002D00D062
:10B7800055E6002BF5D06346134300D16DE68618CD
:10B790008642804161444042091800220B0200D4D5
:10B7A000D0E6464B01351940B2E5B1465DE63300BF
:10B7B0006746203BDF403B00202E05D04027BF1BC3
:10B7C0006646BE40324390464646721E964133431B
:10B7D000EFE5394B9F42CBD080252D04734229439E
:10B7E000A8E70843411E8841A2E6002F00D13CE6AD
:10B7F0006346861ACF1AB0429B415B42FB1A9846B9
:10B800001B024ED5161A6346B2429241591A524251
:10B81000891A5C4600227BE501430E00711E8E41B1
:10B820009FE71D000E00203DEE40B046202B04D0C7
:10B830004025EB1A99400843814648464346411E3D
:10B840008841184374E60022002417E6161A63465E
:10B85000B2429241591A5242891A3D0025E5614689
:10B860009146154D01E680220024120379E61D0061
:10B870000E00203DEE40B046202B04D04025EB1AB0
:10B880009940084381464E464346711E8E411E43F1
:10B8900067E7861896429B4161445B42C9183D00A8
:10B8A0008CE547463743CED007224146324049E631
:10B8B00000273A00E6E5C046FF070000FFFF7FFFD4
:10B8C00070B50C4E0D031C0349005B002D0B490D98
:10B8D000240B5B0DB14208D0064900208B4203D1F6
:10B8E00014432000441EA04170BD05430120002DDB
:10B8F000FAD1F1E7FF07000030B5144D0A034B0001
:10B90000120B5B0DC90F0024AB4211DD104CA3429A
:10B9100010DC8024640322430E4CE41A1F2C0CDD3F
:10B920000D48C31ADA4013005C42002900D11C0004
:10B93000200030BD094BCC18FAE7094DE040AC4679
:10B9400063449A4013000343EEE7C046FE03000041
:10B950001D0400003304000013040000FFFFFF7FFC
:10B96000EDFBFFFF70B500282DD0C317C5185D4053
:10B97000C40F280000F082F8154B1B1A5B055B0D05
:10B980000A2815DD0B38854000222D032D0B0021E0
:10B9900010002D030A0D2D0B12052A430D4D1B051A
:10B9A0002A4013435B00E4075B082343190070BD82
:10B9B00002002900153291400A000B21081AC540E7
:10B9C0002D032D0BE3E70024002300250022DEE7F2
:10B9D0001E040000FFFF0F804100090E4B1C70B5D4
:10B9E000DBB24602750AC40F012B14DDE0239B0075
:10B9F0006D07360BCB1800210A0D280012051C4DCF
:10BA000032435B052A405B0813435B00E4075B0895
:10BA10002343190070BD002914D1002D1ED0280029
:10BA200000F02CF80A281CDC0B232A001B1ADA4031
:10BA3000030015339D400F4B12031B1A5B05160BB9
:10BA40005B0DD8E7002D06D0320B802636036D073C
:10BA50001643094BCFE7084B0026CCE7002300260E
:10BA6000C9E703002A000B3B9A400025E3E7C046E4
:10BA7000FFFF0F8089030000FF0700001C21012346
:10BA80001B04984201D3000C10391B0A984201D3C1
:10BA9000000A08391B09984201D30009043902A29F
:10BAA000105C40187047C046040302020101010106
:10BAB000000000000000000030B51C00094B05002C
:10BAC0001B6885B0D868084B002A01D1074B1A00C3
:10BAD0000292019300912B002200054900F026F804
:10BAE00000F0A6FD8C000020D8E9000013D700006C
:10BAF000E5E90000014B18687047C0468C00002043
:10BB0000084B10B50400002B02D0002100E000BF5C
:10BB1000054B1868836A002B00D09847200001F07D
:10BB20005DFBC0460000000014EA00000EB403B53F
:10BB3000010003AB044804CB0068019300F076F8E1
:10BB400002B008BC03B018478C00002070B5002676
:10BB50000C4D0D4C641BA410A64209D1002601F027
:10BB60003FFB0A4D0A4C641BA410A64205D170BDD0
:10BB7000B300EB5898470136EEE7B300EB5898470F
:10BB80000136F2E75C0200205C0200205C0200202B
:10BB90006C020020002310B59A4200D110BDCC5C8D
:10BBA000C4540133F8E710B5884202D98B18984283
:10BBB00003D3002307E08B5C8354013AFBD210BD12
:10BBC000CC5CC45401339A42FAD1F8E7030012184E
:10BBD000934200D1704719700133F9E7936810B5AB
:10BBE000013B9360002B04DA9469A34207DB0A2926
:10BBF00005D01368581C10601970080010BD00F0C3
:10BC00004BFC0100F9E7F8B506000F001400D51849
:10BC1000AC4201D1002007E021783A003000FFF764
:10BC2000DDFF0134431CF3D1F8BD0000F0B59FB037
:10BC300002900F0016000593002805D08369049335
:10BC4000002B01D100F0F4FD7B4B9F425BD1029BA6
:10BC50005F68BB891B0762D53B69002B5FD000235F
:10BC600006AC6361203363761033A37635002B78FE
:10BC7000002B01D0252B5CD1AB1B04930CD03200E0
:10BC800039000298FFF7BFFF431C00D1C4E062698E
:10BC9000049B9446634463612B78002B00D1BBE086
:10BCA000012200235242626002A9543252186E1CD3
:10BCB0002360E360A3601370A365317805225F48B9
:10BCC00000F0D4FE751C002835D12268D30604D5B7
:10BCD000532302A95B1820211970130704D553239D
:10BCE00002A95B182B21197033782A2B2CD0350030
:10BCF00000210A20E3682A786E1C303A092A64D9A8
:10BD000000292ED026E04E4B9F4202D1029B9F6815
:10BD10009FE74C4B9F429CD1029BDF6899E739001B
:10BD2000029800F00FFC002899D0012040421FB07B
:10BD3000F0BD01359BE7414B2268C01A01238340C7
:10BD4000134323602E00B8E7059B191D1B6805915E
:10BD5000002B01DB099304E05B42E3600223134301
:10BD600023602B782E2B0AD16B782A2B35D1059B9B
:10BD700002351A1D1B680592002B2BDB0793324EF0
:10BD800029780322300000F071FE002806D04023FD
:10BD9000801B8340226801351343236029780622E3
:10BDA0002A486E1C217600F061FE00283AD0284B0C
:10BDB000002B25D10722059B0733934308330593B6
:10BDC0006369039A9B18636150E7434301219B1801
:10BDD000350090E701235B42D0E700230A201A00D8
:10BDE0000135636029786E1C3039092903D9002B8D
:10BDF000C5D00792C3E74243012352183500F1E74B
:10BE000005AB00933A00134B2100029800E000BFFD
:10BE10000390039B0133D3D1BB895B0600D584E734
:10BE20000B9884E705AB00933A000A4B2100029877
:10BE300000F080F8ECE7C0466CEA000018EA000069
:10BE40008CEA00004CEA00001EEA000022EA000032
:10BE50000000000007BC0000F7B5150001938A68D8
:10BE60000B6900900C00934200DA130022002B6053
:10BE700043321278002A01D001332B6023689B06DD
:10BE800002D52B6802332B60062723681F4027D07A
:10BE9000230043331B785A1E93412268920630D404
:10BEA0002200019943320098089EB047431C25D0D8
:10BEB000062320682A68E16803400025042B03D18B
:10BEC0008D1AEB43DB171D40A3682269934201DD05
:10BED0009B1AED180027BD4220D1002010E0013749
:10BEE000E3682A689B1ABB42D2DD22000123193283
:10BEF00001990098089EB047431CF0D101204042B0
:10BF0000FEBD3020E1184331087021005A1C453134
:10BF10000978A218433202331170C1E722000123CD
:10BF20001A3201990098089EB047431CE6D00137A9
:10BF3000D1E70000F0B589B004920A0043320593BE
:10BF4000039002920A7E0C000E9B6E2A00D186E0BE
:10BF50001FD8632A33D008D8002A00D18CE0582A91
:10BF60004DD0250042352A7030E0642A01D0692A7C
:10BF7000F7D1196825680A1D280629D508681A60AE
:10BF8000002803DA2D23029A404213706B4E0A27D1
:10BF90004FE0732A74D008D86F2A1FD0702AE0D1DE
:10BFA000202209680A43226003E0752A16D0782A05
:10BFB000D7D12200782145321170614E22E0250050
:10BFC0001A684235111D196013682B70012365E052
:10BFD00008681A606906D3D500B2D1E719682568E8
:10BFE000081D186008682E0605D5544E08276F2ACC
:10BFF0001BD00A2719E06D06F7D580B2F5E7453169
:10C000004E4E0A7018682268011D006819601506F6
:10C0100021D5D30702D520231A43226010270028F8
:10C0200003D1202322689A43226023000022433355
:10C030001A706368A360002B58DB042221689143C7
:10C040002160002854D1029D002B5AD0250033785E
:10C0500042352B7055E05506DBD580B2D9E71A681A
:10C060000D68101D4969186013682E0601D5196006
:10C0700002E06D06FBD519800023029D23614FE08D
:10C080001A68111D1960156800216268280000F007
:10C09000EDFC002801D0401B606063682361002331
:10C0A000029A13703CE023692A0004990398059DC5
:10C0B000A847431C3ED023689B0715D4079BE06824
:10C0C000984239DA180037E0220001231932049926
:10C0D0000398059EB047431C2CD00135E368079AAE
:10C0E0009B1AAB42F0DCE9E70025F7E70028ADD06A
:10C0F000029D3900FDF722FC735C013D2B70002886
:10C10000F7D1082F09D12368DB0706D563682269B8
:10C11000934202DC3023013D2B70029B5B1B2361A9
:10C12000059B07AA00932100049B0398FFF794FE48
:10C13000431CB8D10120404209B0F0BD29EA0000FB
:10C140003AEA00000D4B70B51C680500A36B002B8C
:10C150000FD1182000F06EFC094BA0630360094B5F
:10C1600001224360084B83600B238381002302611B
:10C1700043610022A36B1D615A6170BD8C000020D9
:10C180000E33CDAB34126DE6ECDE0500124B10B56C
:10C190001C68A36B002B0FD1182000F04BFC0F4B39
:10C1A000A06303600E4B012243600E4B83600B23A0
:10C1B0008381002302614361A46B0B4A206961699A
:10C1C0000A4BFDF7F7FC012200238018594120613A
:10C1D00061614800400810BD8C0000200E33CDABDB
:10C1E00034126DE6ECDE05002D7F954C2DF4515890
:10C1F0000CB430B5164B9DB00C1E1D6808DA8B23AD
:10C2000001202B6040421DB030BC08BC02B0184772
:10C21000822302A99B008B810023029008619C422B
:10C2200000D0631E8B604B6101235B42CB81209A5F
:10C2300021AB2800019300F055FD431C01DA8B234C
:10C240002B60002CDFD00023029A1370DBE7C0467E
:10C250008C0000200EB400B50B499CB01DAB0290C1
:10C260000690079104910948094904CB059100689B
:10C2700002A9019300F036FD0023029A13701CB04E
:10C2800008BC03B01847C046FFFFFF7F8C000020AA
:10C290000802FFFF020010B51378541C002B05D1D3
:10C2A000CC5CD4540133002CFAD110BD2200F3E74A
:10C2B000C9B20378002B04D08B4200D17047013003
:10C2C000F7E74B42594149420840F7E702780B78BB
:10C2D000002A03D0013001319A42F7D0D01A7047BA
:10C2E0000023C25C0133002AFBD1581E7047002393
:10C2F00030B59A420AD0013AC45CCD5CAC4204D15C
:10C30000934202D00133002CF6D1631B180030BDDC
:10C3100030B50500002A00D130BD0C78013A6B1C05
:10C320002C700131002C05D19A189A42F4D01C705F
:10C330000133FAE71D00EDE710B50378002B0FD1AC
:10C340000B785A4253415B42184010BD0023CA5C2F
:10C35000002AFAD0C45C944201D10133F7E70130DE
:10C360000378002BF2D11800EFE70000F0B51F00B2
:10C370000E0087B00590019102920C98347800F07D
:10C38000EAFA082200194378751C134036D12D2C87
:10C3900036D1B51C74780126002F62D0102F09D138
:10C3A000302C07D120222B789343582B54D11027BF
:10C3B0006C7802352D4B3900F31818000393FDF704
:10C3C000BDFA049101210023494202008C46180065
:10C3D0002100303909291AD80C00A74223DD591C45
:10C3E00009D06346824206D302D10499A14202DBFE
:10C3F0000123784320182C780135E9E72E00BCE7AB
:10C400002B2C01D01E00C7E7B51C7478FAE7210079
:10C410004139192901D8373CDFE721006139192951
:10C4200001D8573CD9E75A1C08D1059A2333136029
:10C43000029B0398002B09D107B0F0BD002E00D05D
:10C440004042029A002AF7D0002B01D06B1E0193C4
:10C45000029B019A1A60EFE73024002FAAD1082727
:10C46000A8E7302C9ED00A27A4E7C046FFFFFF7F35
:10C4700037B51300064A05001068046A002C00D185
:10C48000044C0A0000942900FFF770FF3EBDC0462F
:10C490008C000020F0000020F8B505000E0014000C
:10C4A000002804D08369002B01D100F0C1F9224B90
:10C4B0009C422DD16C68A369A360A3891B0731D569
:10C4C0002369002B2ED023682269F7B2981A63697A
:10C4D000F6B2834205DC2100280000F03BF9002879
:10C4E00026D1A3680130013BA36023685A1C226057
:10C4F0001F706369834204D0A389DB071AD50A2E13
:10C5000018D12100280000F025F9002812D00FE0F2
:10C510000A4B9C4201D1AC68CDE7094B9C42CAD181
:10C52000EC68C8E72100280000F00CF80028CAD009
:10C53000012676423000F8BD6CEA00008CEA00006B
:10C540004CEA0000364B70B51D6806000C00002D4B
:10C5500005D0AB69002B02D1280000F069F9314BFE
:10C560009C420FD16C680C23E25E93B219072DD464
:10C57000D90611D409230120336037331343A38133
:10C58000404270BD284B9C4201D1AC68EBE7274B81
:10C590009C42E8D1EC68E6E75B0713D5616B0029A4
:10C5A00008D023004433994202D0300000F06AFAE8
:10C5B000002363632422A3899343A3810023636040
:10C5C000236923600823A2891343A3812369002BD5
:10C5D0000BD1A0218022A389890092000B409342B5
:10C5E00003D02100300000F0E1F90123A2891340BB
:10C5F00011D00023A36063695B42A361002023691B
:10C600008342BED10C23E25E1306BAD54023134306
:10C61000A3810138B5E7920700D46369A360EDE711
:10C620008C0000206CEA00008CEA00004CEA00005C
:10C6300010B5062000F090FC012000F0CFFD0000B6
:10C64000F7B58A8905000C00130760D44B68002BEE
:10C6500004DC0B6C002B01DC0020FEBDE76A002F20
:10C66000FAD000232E682B6080235B01216A1A40D8
:10C6700034D0606DA3895B0706D56368C01A636B0D
:10C68000002B01D0236CC01A0200216A002328006D
:10C69000E76AB847A189431C06D12B681D2B30D807
:10C6A0002B4ADA40D3072CD500236360236923602B
:10C6B000CB0405D5431C02D12B68002B00D160654B
:10C6C000616B2E600029C7D023004433994202D009
:10C6D000280000F0D7F900206063BEE7012328009E
:10C6E000B847431CC6D12B68002BC3D01D2B01D0EB
:10C6F000162B01D12E60AFE74023A2891343A381FB
:10C70000ABE740230B430120A3814042A5E70F691B
:10C71000002FA1D00B680F60DB1B01930023920751
:10C7200000D14B69A360019B002B00DC94E7019BC7
:10C730003A00216A2800A66AB047002803DC40239B
:10C74000A2891343DFE7019B3F181B1A0193EAE715
:10C75000010040200B6970B505000C00002B01D1D1
:10C76000002070BD002804D08369002B01D100F0A7
:10C770005FF80B4B9C4209D16C680C22A35E002B26
:10C78000EED021002800FFF75BFFEAE7054B9C4253
:10C7900001D1AC68F1E7044B9C42EED1EC68ECE7C8
:10C7A0006CEA00008CEA00004CEA0000002310B59F
:10C7B000040003604360836081814366C28103613A
:10C7C00043618361190008225C30FFF7FFF9054BD4
:10C7D00024626362044BA362044BE362044B236351
:10C7E00010BDC04699CF0000C1CF0000F9CF0000B6
:10C7F00025D0000010B5024900F08CF810BDC046ED
:10C8000055C7000070B568254A1E55430E00290023
:10C81000743100F081F9041E08D000212A00016063
:10C8200046600C30A0606832FFF7D0F9200070BD80
:10C83000836913B50400002B28D18364C3640365A6
:10C84000134B144A1B6882620193984201D1012361
:10C850008361200000F020F86060200000F01CF8E8
:10C86000A060200000F018F80022E0600421606859
:10C87000FFF79CFF01220921A068FFF797FF022222
:10C880001221E068FFF792FF0123A36113BDC046A8
:10C8900014EA0000F5C70000F8B51C4B07001E683D
:10C8A000B369002B02D13000FFF7C2FF4836B468ED
:10C8B0007368013B04D53368002B07D03668F6E770
:10C8C0000C22A55E002D0DD06834F2E7042138005B
:10C8D000FFF798FF30600028F0D10C2304003B6084
:10C8E0002000F8BD20000A4B656625606560A560E4
:10C8F000E36025616561A561082229005C30FFF7CE
:10C9000065F96563A563A564E564E9E714EA0000D9
:10C910000100FFFFF7B5040007000026019148342D
:10C92000002C01D13000FEBD6368A5680093009B18
:10C93000013B009301D52468F2E7AB89012B08D9AC
:10C940000E22AB5E013304D029003800019B9847CA
:10C9500006436835EBE7EC300068704770B50E00B1
:10C960001D000E23C95E96B01400002907DA0023CB
:10C970002B60B3891B0611D48023DB000FE06A46CD
:10C9800000F088FB0028F2DBF022019B120213402A
:10C99000054A9B185A4253412B60EDE74023002083
:10C9A000236016B070BDC04600E0FFFFF7B5022659
:10C9B0008B8905000C00334206D0230047332360E7
:10C9C000236101236361F7BD01AB6A46FFF7C6FF30
:10C9D00000990700280000F09FF8002808D10C22D9
:10C9E000A35E9A05EFD4032293431E43A681E4E796
:10C9F0000F4BAB628023A28920601343A381009B6D
:10CA000020616361019B002B0DD00E23E15E2800A5
:10CA100000F052FB002806D00322A38993431A009A
:10CA200001231343A381A0893843A081CBE7C046EB
:10CA3000F5C7000010B5034B0100186800F06CF852
:10CA400010BDC0468C00002082B0002900D101A991
:10CA5000101E06D0002B06D013780B601078431EF2
:10CA6000984102B0704702204042FAE7C9B28218EA
:10CA7000904201D10020704703788B42FBD00130F7
:10CA8000F6E7000070B50500002910D00C1F2368E0
:10CA9000002B00DAE418280000F034FB1D4A13686C
:10CAA000002B05D163601460280000F02CFB70BDE2
:10CAB000A34209D9216860188342F3D118685B68E2
:10CAC00041182160EEE713005A68002A01D0A24203
:10CAD000F9D919685818A0420BD1206809185818BC
:10CAE00019608242E0D110685268411819605A609A
:10CAF000DAE7A04202D90C232B60D5E72168601841
:10CB0000824203D1106852684118216062605C6003
:10CB1000CAE7C046381C0020032370B5CD1C9D43D6
:10CB2000083506000C2D1ED20C25A9421DD8300058
:10CB300000F0E8FA254A14682100002919D1244C94
:10CB40002368002B03D1300000F0CAF920602900CF
:10CB5000300000F0C5F9431C2BD10C2330003360AA
:10CB600000F0D1FA03E0002DDFDA0C23336000205F
:10CB700070BD0B685B1B19D40B2B03D90B60CC1851
:10CB8000256003E04B688C420DD11360300000F04B
:10CB9000BAFA200007220B30231D9043C31AE7D0B6
:10CBA0005A42E250E4E763600C00EFE70C0049688A
:10CBB000C3E70323C41C9C43A042E1D0211A3000E8
:10CBC00000F08EF9431CDBD1C7E7C046381C0020BB
:10CBD0003C1C0020F8B507000D001600002905D107
:10CBE0001100FFF799FF04002000F8BD002A03D1CF
:10CBF000FFF748FF3400F7E700F086FA2C00B04258
:10CC0000F2D231003800FFF787FF041EECD0290074
:10CC10003200FEF7BFFF29003800FFF733FFE3E7DC
:10CC2000F0B58E6885B007000C00039201939E4218
:10CC30003CD890238A89DB001A4234D00325096945
:10CC400023685B1A0293636902985D43EB0F5D19D9
:10CC5000019B6D1001331B18AB4200D91D00530519
:10CC600032D529003800FFF757FF061E09D10C23E3
:10CC70003B6040230120A28940421343A38105B0B9
:10CC8000F0BD029A2169FEF785FFA389144A1A4074
:10CC900080231343A381029B2661F61826606561F9
:10CCA000019EED1AA560019B9E4200D9019E3200B3
:10CCB00003992068FEF777FFA36800209B1BA36001
:10CCC00023689E192660DAE72A003800FFF782FF02
:10CCD000061EE0D121693800FFF7D4FEC7E7C04641
:10CCE0007FFBFFFFF0B59FB0029005938B890F008B
:10CCF00016001B0611D50B69002B0ED14021FFF742
:10CD00000BFF38603861002805D10C23029A0138E6
:10CD100013601FB0F0BD40237B61002306AC63614C
:10CD2000203363761033A37635002B78002B01D0A7
:10CD3000252B46D1AB1B04930CD03200390002984E
:10CD4000FFF76EFF431C00D1AEE06269049B94467E
:10CD5000634463612B78002B00D1A5E001220023FE
:10CD60005242626002A9543252186E1C2360E36082
:10CD7000A3601370A365317805225448FFF776FE4F
:10CD8000751C00281FD12268D30604D5532302A99D
:10CD90005B1820211970130704D5532302A95B18CF
:10CDA0002B21197033782A2B16D0350000210A2048
:10CDB000E3682A786E1C303A092A4ED9002918D027
:10CDC00010E00135B1E7414B2268C01A01238340CE
:10CDD000134323602E00CEE7059B191D1B680591A8
:10CDE000002B01DB099304E05B42E3600223134361
:10CDF00023602B782E2B0AD16B782A2B35D1059BFB
:10CE000002351A1D1B680592002B2BDB0793304E51
:10CE1000297803223000FFF729FE002806D040239E
:10CE2000801B834022680135134323602978062242
:10CE300028486E1C2176FFF719FE00283CD0264BAF
:10CE4000002B25D10722059B073393430833059315
:10CE50006369039A9B18636166E7434301219B184A
:10CE60003500A6E701235B42D0E700230A201A0021
:10CE70000135636029786E1C3039092903D9002BEC
:10CE8000C5D00792C3E74243012352183500F1E7AA
:10CE900005AB00933A00114B2100029800E000BF5F
:10CEA0000390039B0133D3D1BB890B985B0600D45D
:10CEB0002FE7012040422CE705AB00933A00074BD7
:10CEC00021000298FFF736F8EAE7C04618EA0000AA
:10CED0001EEA000022EA00000000000021CC000051
:10CEE000002370B5064C05000800236000F060F9CF
:10CEF000431C03D12368002B00D02B6070BDC046BB
:10CF0000CC2F002070B504000D001F2904D9162372
:10CF100003600120404270BD436C002B04D08A00A6
:10CF20009B181A68002A08D1200000F031F82A0066
:10CF30000100200000F01AF8EDE70020012AEAD0F5
:10CF4000511C03D1162301302360E4E7002428009C
:10CF50001C6090472000DEE710B5034B0100186805
:10CF6000FFF7D0FF10BDC0468C000020002370B535
:10CF7000064C050008001100236000F001F9431C75
:10CF800003D12368002B00D02B6070BDCC2F002074
:10CF900010B500F0E5F810BD70B50C000E25495F26
:10CFA00000F0BAF8002803DB636D1B18636570BDE1
:10CFB000A389024A1340A381F9E7C046FFEFFFFFB0
:10CFC000F8B51F008B8905000C001600DB0505D5A0
:10CFD0000E23C95E0022022300F080F8A389054ACF
:10CFE00028001340A38132000E23E15E3B0000F0D5
:10CFF0002BF8F8BDFFEFFFFF70B50C000E25495F61
:10D0000000F06CF8A389421C03D1054A1340A381A8
:10D0100070BD802252011343A3816065F8E7C046CA
:10D02000FFEFFFFF10B50E23C95E00F021F810BD21
:10D030000B1E04D0FF2A04D98A2303608B3B1800FF
:10D0400070470A700123FAE770B505000800110067
:10D050000022064C22601A0000F0B8F8431C03D1ED
:10D060002368002B00D02B6070BDC046CC2F002061
:10D07000002370B5064C05000800236000F060F83E
:10D08000431C03D12368002B00D02B6070BDC04629
:10D09000CC2F0020002370B5064C050008001100BD
:10D0A000236000F055F8431C03D12368002B00D007
:10D0B0002B6070BDCC2F0020002370B5064C0500FE
:10D0C0000800236000F054F8431C03D12368002BB0
:10D0D00000D02B6070BDC046CC2F002070B505007D
:10D0E000080011000022064C22601A0000F050F8DF
:10D0F000431C03D12368002B00D02B6070BDC046B9
:10D10000CC2F0020704770470B1F1B68181F002B87
:10D1100001DA0B58C018704770B5050008001100FF
:10D120000022064C22601A0000F03AF8431C03D19A
:10D130002368002B00D02B6070BDC046CC2F002090
:10D1400058220120014B40421A607047CC2F00202A
:10D1500058220120014B40421A607047CC2F00201A
:10D1600058220120014B40421A607047CC2F00200A
:10D170005822024B00201A607047C046CC2F002076
:10D1800058220120014B40421A607047CC2F0020EA
:10D1900058220120014B40421A607047CC2F0020DA
:10D1A00058220120014B40421A607047CC2F0020CA
:10D1B000044A1368002B00D1034B181810601800A4
:10D1C0007047C046401C0020D02F0020582201206C
:10D1D000014B40421A607047CC2F0020FEE7C0464A
:10D1E000F8B5C046F8BC08BC9E467047F8B5C046C6
:10D1F000F8BC08BC9E467047646174610000000082
:10D200007CD20000EF01000085D20000E3020000A4
:10D210008DD200001909000094D20000290A0000F4
:10D2200099D2000041050000A4D200005303000081
:10D23000A9D20000810C0000B5D200001F0200003E
:10D24000BFD2000021080000CDD20000CD060000B2
:10D25000DAD200000305000072616E646F6D006138
:10D260006C6C006C6173740066616C736500747241
:10D27000756500252E3135732E2E2E006D616B6580
:10D280004C697374006164644C6173740064656C10
:10D29000657465006A6F696E00636F707946726FBE
:10D2A0006D546F0066696E64006A6F696E537472C4
:10D2B000696E677300756E69636F646541740075AC
:10D2C0006E69636F6465537472696E67006E65772B
:10D2D00042797465417272617900667265654D6567
:10D2E0006D6F7279000000004DD300000D11000039
:10D2F00052D300002B1100008DD200002F1100002E
:10D3000058D300001111000062D300003311000057
:10D310006BD300003711000075D300003B110000F3
:10D3200080D300003F1100008CD3000015110000D5
:10D3300095D30000231100009FD3000019110000B5
:10D34000AAD300002711000066696C65006F706544
:10D350006E00636C6F736500656E644F6646696C42
:10D360006500726561644C696E6500726561644256
:10D370007974657300617070656E644C696E6500E8
:10D38000617070656E6442797465730066696C657E
:10D3900053697A650073746172744C697374006EBA
:10D3A000657874496E4C6973740073797374656D34
:10D3B000496E666F00000000F814000008150000B8
:10D3C000221500009E150000D61500000A16000068
:10D3D0004216000068160000A4160000E6160000C1
:10D3E0003C17000080170000E21700002C18000016
:10D3F000521800008A180000D0180000F61800002B
:10D4000024190000521900002A3000000A1A0000F6
:10D41000DC1A0000521B0000C21B00000E1C0000A2
:10D420002E1C0000501C0000A81D0000EC1D000078
:10D43000641E0000921E0000C41E0000F61E0000C4
:10D44000761F0000DE1F00003A2000009820000038
:10D450000A2100007C210000D821000032220000B7
:10D4600068220000B8220000FE22000046230000CF
:10D470009A230000EE2300002C24000098240000D2
:10D48000CE240000162500005E250000A625000021
:10D49000E02500002826000078260000DA2700009A
:10D4A000241900008A180000E0260000F81400008B
:10D4B000162700004227000078270000A42700005C
:10D4C000F8140000F8140000F8140000F81400002C
:10D4D0005628000098280000DE2800002E290000B1
:10D4E0005A290000D2290000242A0000882A0000BE
:10D4F000F8140000F8140000AC2A0000DC2A000038
:10D500000C2B0000422B00006C2B0000A22B000013
:10D51000CC2B0000F42B00001C2C00004C2C000035
:10D520007C2C0000A62C0000D02C0000002D000058
:10D530002A2D0000F8140000F8140000F814000070
:10D54000F8140000F81400005A2D0000862D000089
:10D55000B22D0000DE2D00000A2E0000402E00003B
:10D56000802E0000B62E0000EC2E0000182F0000C8
:10D57000442F00007A2F0000F8140000F814000077
:10D58000F8140000F8140000F8140000F81400006B
:10D59000F8140000F8140000F8140000F81400005B
:10D5A000F8140000F8140000A62F0000A62F0000B9
:10D5B00080300000B63000005B2564206974656D22
:10D5C000206C6973745D002825642062797465732A
:10D5D0002900286F626A65637420747970653A2047
:10D5E00025642900537461636B20756E64657266EF
:10D5F0006C6F7700626F6F6C65616E006E756D6247
:10D60000657200737472696E67006C69737400628E
:10D610007974652061727261790000000700000072
:10D62000030000007ED60000D931000086D600003D
:10D63000893200008FD60000FB33000098D600002E
:10D64000DD310000A1D60000FF330000A9D60000A4
:10D65000E9330000B2D600001933000000000000DA
:10D6600001000000020000000300000004000000B0
:10D670000A0000006D6963726F3A62697400686144
:10D6800073546F6E6500706C6179546F6E650068DD
:10D690006173536572766F00736574536572766F4C
:10D6A00000646163496E69740064616357726974F0
:10D6B0006500737175617265576176650047432037
:10D6C000746F6F6B2025642075736563733B2066F0
:10D6D00072656520256420776F726473003C496E23
:10D6E00074656765723E003C4C6973743E003C4F44
:10D6F000626A6563743E003C42797465417272618E
:10D70000793E000D0A564D2050616E69633A20251E
:10D71000730D0A006D6973630000000051D70000AB
:10D72000ED4000005AD700007D4000005ED70000A9
:10D73000D13F000066D70000773F000070D700009F
:10D740000D3F00007CD700000F3E00006E756C6C32
:10D7500000686578546F496E740073696E006A736F
:10D760006F6E476574006A736F6E436F756E7400F9
:10D770006A736F6E56616C75654174006A736F6E83
:10D780004B6579417400000014D800005941000035
:10D790001CD800005D41000026D800007B4100003D
:10D7A0002FD80000854100003AD800008F410000CA
:10D7B00046D800009941000054D80000A341000061
:10D7C0005CD80000AD41000062D80000B741000005
:10D7D00077D80000C14100008CD80000CB41000088
:10D7E00098D80000D5410000A8D80000DF41000013
:10D7F000B4D80000E9410000C1D80000F3410000A6
:10D80000D0D8000067410000E3D80000714100005B
:10D810006E6574006861735769466900737461725C
:10D8200074576946690073746F7057694669007769
:10D83000696669537461747573006D794950416408
:10D8400064726573730073746172745353494473E3
:10D8500063616E0067657453534944006D794D41AF
:10D8600043006874747053657276657247657452CC
:10D8700065717565737400726573706F6E64546F53
:10D88000487474705265717565737400687474704F
:10D89000436F6E6E65637400687474704973436F90
:10D8A0006E6E65637465640068747470526571753A
:10D8B0006573740068747470526573706F6E73650D
:10D8C00000776562536F636B6574537461727400A3
:10D8D000776562536F636B65744C617374457665ED
:10D8E0006E7400776562536F636B657453656E6425
:10D8F000546F436C69656E74001A1B1C03040607A1
:10D90000090A171819000000000008080800080A92
:10D910004A4000000A5FEA5FEA0ED92ED36E193240
:10D920004489330C924C924D08080000000488088A
:10D9300008040804848488000A448A4000048EC4D1
:10D9400080000000048800000EC0000000000800F5
:10D9500001224488100C9252524C048C84848E1CF8
:10D96000824C901E1EC244924C06CA525FE21FF0C7
:10D970001EC13E02448ED12E1FE24488100ED12ECD
:10D98000D12E0ED12EC488000800080000048004A7
:10D99000880244880482000EC00EC00804824488B5
:10D9A0000ED126C0040ED135B36C0C925ED2521C3F
:10D9B000925C925C0ED010100E1C9252525C1ED0E3
:10D9C0001C901E1ED01C90100ED013712E12525E91
:10D9D000D2521C8808081C1FE242524C1254981460
:10D9E00092101010101E113B75B131113935B37101
:10D9F0000C9252524C1C925C90100C92524C861C11
:10DA0000925C92510ED00C825C1FE484848412528A
:10DA100052524C1131312A44113135BB7112524CE2
:10DA20009252112A4484841EC488101E0EC808080D
:10DA30000E10080482410EC242424E048A40000089
:10DA4000000000001F0804800000000ED2524F109A
:10DA5000101C925C000ED0100E02424ED24E0C9260
:10DA60005C900E06C81C88080ED24EC24C10101CCA
:10DA700092520800080808024002424C1014981400
:10DA8000920808080806001B75B131001C9252521A
:10DA9000000C92524C001C925C90000ED24EC200C0
:10DAA0000ED010100006C8049808080EC80700120F
:10DAB00052524F0011312A4400113135BB00124C33
:10DAC0008C9200112A4498001EC4881E06C48C84BF
:10DAD00086080808080818080C881800000C8360DD
:10DAE0000000000001000000020000000300000030
:10DAF0000400000005000000060000000700000010
:10DB000008000000090000000A0000000B000000EF
:10DB10000C0000000D0000000E0000000F000000CF
:10DB200010000000120000001400000016000000A9
:10DB3000180000001A0000001C0000001E00000079
:10DB40002000000023000000260000002900000043
:10DB50002C0000002F000000320000003600000002
:10DB60003A0000003E0000004200000046000000B5
:10DB70004B00000050000000550000005A0000005B
:10DB800061000000680000006F00000076000000E7
:10DB90007D000000840000008B0000009200000067
:10DBA00099000000A0000000A7000000AE000000E7
:10DBB000B5000000BC000000C3000000CA00000067
:10DBC000D1000000D8000000DF000000E6000000E7
:10DBD000ED000000F4000000FB000000FF0000006A
:10DBE00030DC0000154200003BDC0000B1470000C3
:10DBF00045DC0000D943000052DC00002146000053
:10DC000059DC00007146000062DC0000C1460000E3
:10DC10006EDC0000B94500007FDC000049440000D4
:10DC20008CDC000049450000646973706C61790008
:10DC30006C696768744C6576656C006D62446973E5
:10DC4000706C6179006D62446973706C61794F66C4
:10DC500066006D62506C6F74006D62556E706C6F13
:10DC600074006D62447261775368617065006D6223
:10DC70005368617065466F724C6574746572006EAE
:10DC8000656F506978656C53656E64006E656F50A2
:10DC90006978656C53657450696E004E6F742065C9
:10DCA0006E6F75676820726F6F6D206576656E2088
:10DCB000616674657220636F6D70616374696F6E05
:10DCC00000436F6D70616374656420466C617368B6
:10DCD00020636F64652073746F72650A2564206227
:10DCE000797465732075736564202825642525295A
:10DCF000206F6620256400426164207265636F7244
:10DD00006420666F756E6420647572696E67206941
:10DD10006E697469616C697A6174696F6E002564FB
:10DD20002025642025642028256420776F72647381
:10DD300029002564207265636F7264732C2025644A
:10DD400020776F7264732C206D61784944202564BC
:10DD50002C20636F6D70616374696F6E20637963EB
:10DD60006C657320256400526573746F726564205E
:10DD700025642073637269707473005374617274E4
:10DD8000656400726164696F000000001CDE0000C1
:10DD90008151000029DE00001D54000039DE000022
:10DDA0009D53000047DE0000B155000052DE000028
:10DDB000A951000062DE00003152000076DE000052
:10DDC0001952000085DE00009357000091DE00002C
:10DDD000115700009ADE0000B5560000A5DE0000D5
:10DDE000FD550000B0DE000039560000B9DE00002D
:10DDF0006D560000C2DE0000B9510000D1DE000007
:10DE000099510000DADE0000C95100006E6F6E65A6
:10DE1000006F746865720070616972006469736193
:10DE2000626C65526164696F006D657373616765EB
:10DE30005265636569766564007061636B657452F1
:10DE4000656365697665007061636B657453656EC3
:10DE500064007265636569766564496E74656765BB
:10DE6000720072656365697665644D657373616799
:10DE7000655479706500726563656976656453748D
:10DE800072696E670073656E64496E74656765726A
:10DE90000073656E64506169720073656E645374DB
:10DEA00072696E67007365744368616E6E656C00BD
:10DEB00073657447726F757000736574506F776522
:10DEC00072007369676E616C537472656E67746813
:10DED000006465766963654944006C6173744D65DF
:10DEE0007373616765494400556E6B6E6F776E2082
:10DEF0007072696D6974697665205B25733A257364
:10DF00005D00000000000000963007772C610EEEE7
:10DF1000BA51099919C46D078FF46A7035A563E980
:10DF2000A395649E3288DB0EA4B8DC791EE9D5E0A7
:10DF300088D9D2972B4CB609BD7CB17E072DB8E7A6
:10DF4000911DBF906410B71DF220B06A4871B9F3FB
:10DF5000DE41BE847DD4DA1AEBE4DD6D51B5D4F434
:10DF6000C785D38356986C13C0A86B647AF962FD99
:10DF7000ECC9658A4F5C0114D96C0663633D0FFAE6
:10DF8000F50D088DC8206E3B5E10694CE44160D5EC
:10DF9000727167A2D1E4033C47D4044BFD850DD2D6
:10DFA0006BB50AA5FAA8B5356C98B242D6C9BBDBE9
:10DFB00040F9BCACE36CD832755CDF45CF0DD6DCE4
:10DFC000593DD1ABAC30D9263A00DE518051D7C88B
:10DFD0001661D0BFB5F4B42123C4B3569995BACF16
:10DFE0000FA5BDB89EB802280888055FB2D90CC637
:10DFF00024E90BB1877C6F2F114C6858AB1D61C1B0
:10E000003D2D66B69041DC760671DB01BC20D298CE
:10E010002A10D5EF8985B1711FB5B606A5E4BF9F5B
:10E0200033D4B8E8A2C9077834F9000F8EA809964E
:10E0300018980EE1BB0D6A7F2D3D6D08976C6491B9
:10E04000015C63E6F4516B6B62616C1CD8306585D2
:10E050004E0062F2ED95066C7BA5011BC1F40882AF
:10E0600057C40FF5C6D9B06550E9B712EAB8BE8BF0
:10E070007C88B9FCDF1DDD62492DDA15F37CD38C79
:10E08000654CD4FB5861B24DCE51B53A7400BCA377
:10E09000E230BBD441A5DF4AD795D83D6DC4D1A4A9
:10E0A000FBF4D6D36AE96943FCD96E34468867AD80
:10E0B000D0B860DA732D0444E51D03335F4C0AAA1F
:10E0C000C97C0DDD3C710550AA41022710100BBE22
:10E0D00086200CC925B56857B3856F2009D466B969
:10E0E0009FE461CE0EF9DE5E98C9D9292298D0B09E
:10E0F000B4A8D7C7173DB359810DB42E3B5CBDB74B
:10E10000AD6CBAC02083B8EDB6B3BF9A0CE2B603CB
:10E110009AD2B1743947D5EAAF77D29D1526DB0480
:10E120008316DC73120B63E3843B64943E6A6D0DCB
:10E13000A85A6A7A0BCF0EE49DFF099327AE000A16
:10E14000B19E077D44930FF0D2A3088768F2011EA9
:10E15000FEC206695D5762F7CB67658071366C1940
:10E16000E7066B6E761BD4FEE02BD3895A7ADA1061
:10E17000CC4ADD676FDFB9F9F9EFBE8E43BEB71742
:10E18000D58EB060E8A3D6D67E93D1A1C4C2D838CC
:10E1900052F2DF4FF167BBD16757BCA6DD06B53F32
:10E1A0004B36B248DA2B0DD84C1B0AAFF64A033671
:10E1B000607A0441C3EF60DF55DF67A8EF8E6E31F0
:10E1C00079BE69468CB361CB1A8366BCA0D26F2539
:10E1D00036E2685295770CCC03470BBBB916022286
:10E1E0002F260555BE3BBAC5280BBDB2925AB42B9B
:10E1F000046AB35CA7FFD7C231CFD0B58B9ED92CB0
:10E200001DAEDE5BB0C2649B26F263EC9CA36A7514
:10E210000A936D02A906099C3F360EEB85670772CB
:10E2200013570005824ABF95147AB8E2AE2BB17B32
:10E23000381BB60C9B8ED2920DBED5E5B7EFDC7CB9
:10E2400021DFDB0BD4D2D38642E2D4F1F8B3DD6810
:10E250006E83DA1FCD16BE815B26B9F6E177B06F0B
:10E260007747B718E65A0888706A0FFFCA3B0666F8
:10E270005C0B0111FF9E658F69AE62F8D3FF6B6185
:10E2800045CF6C1678E20AA0EED20DD75483044E27
:10E29000C2B30339612667A7F71660D04D476949B5
:10E2A000DB776E3E4A6AD1AEDC5AD6D9660BDF40C8
:10E2B000F03BD83753AEBCA9C59EBBDE7FCFB2477B
:10E2C000E9FFB5301CF2BDBD8AC2BACA3093B35360
:10E2D000A6A3B4240536D0BA9306D7CD2957DE5469
:10E2E000BF67D9232E7A66B3B84A61C4021B685D42
:10E2F000942B6F2A37BE0BB4A18E0CC31BDF055ABB
:10E300008DEF022D416C6C207461736B73207374FC
:10E310006F707065640076313133002025732025DD
:10E3200073004D656D6F727920636C656172656411
:10E33000004E6F2066726565207461736B20656E98
:10E340007472696573000000B8E30000316D00006D
:10E35000C5E3000059670000D1E30000016D000033
:10E36000D7E30000116D0000DDE30000216D000027
:10E37000E3E30000C56A0000F9E300008D670000D8
:10E3800003E400008D6D00000BE40000E16A000072
:10E3900014E400004969000020E400006568000002
:10E3A00029E40000B168000031E40000196A0000AF
:10E3B00073656E736F727300616363656C65726120
:10E3C00074696F6E0074656D7065726174757265E5
:10E3D0000074696C74580074696C74590074696CC9
:10E3E000745A00736574416363656C65726F6D6523
:10E3F00074657252616E676500746F75636852650B
:10E400006164006932635265616400693263577206
:10E410006974650073706945786368616E6765004B
:10E420007370695365747570007265616444485413
:10E43000006D6963726F70686F6E6500B8E400000C
:10E44000196E0000C6E40000296E0000D3E400004D
:10E450001D6E0000DCE400002D6E0000E6E400000C
:10E46000316E0000EFE40000356E0000F4E40000BF
:10E47000396E0000F9E400003D6E000005E5000083
:10E48000416E00000CE50000456E000015E500003F
:10E49000496E00001AE500004D6E000025E5000001
:10E4A000516E00002FE50000216E000039E50000EC
:10E4B000256E000074667400656E61626C65446967
:10E4C00073706C6179007365744261636B6C69672A
:10E4D0006874006765745769647468006765744898
:10E4E000656967687400736574506978656C006C61
:10E4F000696E65007265637400726F756E64656441
:10E500005265637400636972636C6500747269615B
:10E510006E676C65007465787400746674546F750A
:10E520006368656400746674546F7563685800743A
:10E530006674546F7563685900746674546F7563BC
:10E54000685072657373757265007661727300004E
:10E5500070E50000E17200007AE50000C172000081
:10E5600083E500009D7200008FE500002B72000023
:10E57000766172457869737473007661724E616D6D
:10E580006564007365745661724E616D65640076F2
:10E5900061724E616D65466F72496E6465780057B1
:10E5A000656C636F6D6520746F204D6963726F4297
:10E5B0006C6F636B732100705F73706920213D2065
:10E5C0004E554C4C002F686F6D652F6769742F2E68
:10E5D000706C6174666F726D696F2F7061636B61CF
:10E5E0006765732F6672616D65776F726B2D6172EF
:10E5F0006475696E6F6E6F726469636E7266352FD3
:10E600006C69627261726965732F5350492F535060
:10E61000492E63707000535049436C6173733A3AEA
:10E62000535049436C617373284E52465F535049AF
:10E630005F547970652A2C2075696E74385F742C6C
:10E640002075696E74385F742C2075696E74385F3C
:10E650007429000000000000000000006974000040
:10E66000257400004B740000557400005F740000B6
:10E6700049740000030000000200000001000000D7
:10E680000400000005000000110000000C00000064
:10E690000B000000120000000A000000060000004D
:10E6A0001A0000001400000017000000160000000F
:10E6B0001500000010000000FFFFFFFFFFFFFFFF3D
:10E6C000000000001E0000001900000018000000FB
:10E6D0000700000008000000090000000D00000015
:10E6E0000E0000000F0000001C0000001B000000D6
:10E6F0001D000000130000000000000000000000EA
:10E700005578000089800000D5780000E978000085
:10E71000DF7800005178000045780000F5780000AF
:10E7200071780000417800000000000000003043D4
:10E7300000000000000030C373717274000000001C
:10E74000FB21F93FFB2109407CD91240FB211940F4
:10E750007A6A1F407CD92240BBFD2540FB2129401D
:10E760003A462C407A6A2F405C4731407CD932408F
:10E770009C6B3440BBFD3540DB8F3740FB2139407B
:10E780001BB43A403A463C405AD83D407A6A3F4032
:10E790004C7E40405C4741406C1042407CD9424036
:10E7A0008CA243409C6B4440AC344540BBFD45408B
:10E7B000CBC64640DB8F4740EB584840FB214940E1
:10E7C00083F9A200444E6E00FC291500D1572700A2
:10E7D000DD34F50062DBC0003C99950041904300B8
:10E7E0006351FE00BBDEAB00B761C5003A6E24008A
:10E7F000D24D42004906E00009EA2E001C92D100E9
:10E80000EB1DFE0029B11C00E83EA700F535820093
:10E8100044BB2E009CE98400B4267000417E5F005A
:10E82000D6913900538339009CF439008B5F840002
:10E8300028F9BD00F81F3B00DEFF97000F98050088
:10E84000112FEF000A5A8B006D1F6D00CF7E36002E
:10E8500009CB2700464FB7009E663F002DEA5F00B8
:10E86000BA277500E5EBC7003D7BF100F7390700DB
:10E8700092528A00FB6BEA001FB15F00085D8D00B9
:10E88000300356007BFC4600F0AB6B0020BCCF0091
:10E8900036F49A00E3A91D005E619100081BE600B2
:10E8A00085996500A0145F008D40680080D8FF0046
:10E8B00027734D0006063100CA561500C9A873001B
:10E8C0007BE260006B8CC00000000040FB21F93F40
:10E8D000000000002D44743E000000809846F83C83
:10E8E0000000006051CC783B00000080831BF039B1
:10E8F0000000004020257A38000000802282E336A4
:10E90000000000001DF36935020000000300000054
:10E910000400000006000000009D0000AA9C00000A
:10E92000AA9C0000D89D0000A69C0000A69C0000A8
:10E93000CE9D0000D89D0000A69C0000CE9D00004A
:10E94000A69C0000D89D0000DC9D0000DC9D00001E
:10E95000DC9D0000E49D0000DCA700004EA6000046
:10E9600092A60000F6A5000092A6000082A7000073
:10E9700092A60000F6A500004EA600004EA60000DC
:10E9800082A70000F6A50000EEA50000EEA500009D
:10E99000EEA5000090A7000004AF000006AE000046
:10E9A00006AE000024B1000000AE000000AE000082
:10E9B0000CB1000024B1000000AE00000CB100005A
:10E9C00000AE000024B100001AB100001AB100002E
:10E9D0001AB1000028B100002C2066756E637469BE
:10E9E0006F6E3A2000617373657274696F6E2022D6
:10E9F000257322206661696C65643A2066696C65DE
:10EA000020222573222C206C696E652025642573D5
:10EA100025730A0090000020232D302B2000686C05
:10EA20004C00656667454647003031323334353631
:10EA3000373839414243444546003031323334356A
:10EA40003637383961626364656600000000000093
:10EA500000000000000000000000000000000000B6
:10EA600000000000000000000000000000000000A6
:10EA70000000000000000000000000000000000096
:10EA80000000000000000000000000000000000086
:10EA90000000000000000000000000000000000076
:10EAA000000000000000000000000000504F53492B
:10EAB000580000202020202020202020282828283E
:10EAC000282020202020202020202020202020203E
:10EAD000202020881010101010101010101010108E
:10EAE000101010040404040404040404041010109E
:10EAF000101010104141414141410101010101014A
:10EB000001010101010101010101010101011010D7
:10EB1000101010104242424242420202020202021D
:10EB200002020202020202020202020202021010A9
:10EB30001010200000000000000000000000000095
:10EB400000000000000000000000000000000000C5
:10EB500000000000000000000000000000000000B5
:10EB600000000000000000000000000000000000A5
:10EB70000000000000000000000000000000000095
:10EB80000000000000000000000000000000000085
:10EB90000000000000000000000000000000000075
:10EBA0000000000000000000000000000000000065
:08EBB00000000000000000005D
:08EBB8005015FF7F0100000071
:10EBC000FFFFFFFFE803000001000000E803DC0591
:10EBD000DC05DC05DC050000FFFFFFFFFFFFFFFF9A
:10EBE0001800000019FCFFFFFFFFFFFF02000000FC
:10EBF00040420F00FF0000000024F400020000006B
:10EC000003000000FFFFFFFF000000000100000004
:10EC10000000020001000000FFFFFFFF00000000F5
:10EC2000020000000000040002000000FFFFFFFFE0
:10EC300000000000030000000000080003000000C6
:10EC40000A00000008000000010000009000002001
:10EC5000000000006CEA00008CEA00004CEA0000B2
:10EC600000000000000000000000000000000000A4
:10EC70000000000000000000000000000000000094
:10EC80000000000000000000000000000000000084
:10EC90000000000000000000000000000000000074
:10ECA0000000000000000000000000000000000064
:10ECB0004300000000000000000000000000000011
:10ECC0000000000000000000000000000000000044
:10ECD00043000000000000000000000000000000F1
:10ECE0000000000000000000000000000000000024
:10ECF00043000000000000000000000000000000D1
:10ED00000000000000000000000000000000000003
:10ED100043000000000000000000000000000000B0
:10ED200000000000000000000000000000000000E3
:10ED30004300000000000000000000000000000090
:10ED400000000000000000000000000000000000C3
:10ED50004300000000000000000000000000000070
:10ED600000000000000000000000000000000000A3
:10ED70004300000000000000000000000000000050
:10ED80000000000000000000000000000000000083
:10ED900031D0000049CA000000000000B2EA0000C3
:10EDA0007AD2000013D7000013D7000013D7000059
:10EDB00013D7000013D7000013D7000013D70000AB
:10EDC00013D7000013D70000FFFFFFFFFFFFFFFF77
:10EDD000FFFFFFFFFFFF00000100415343494900CF
:10EDE0000000000000000000000000000000000023
:10EDF00000000000000000000000415343494900AA
:10EE00000000000000000000000000000000000002
:10EE1000000000000000000000000000E900000009
:10EE2000F573000049770000A17B0000C1000000DD
:04000003000077E59D
:00000001FF
